:10000000F4FB0220990100008956010041560100CD
:100010004156010041560100415601004156010080
:100020004156010041560100415601008956010028
:1000300089560100415601001971010069730100E0
:100040008956010089560100895601008956010030
:100050008956010089560100895601008956010020
:100060008956010089560100895601008956010010
:100070008956010089560100895601008956010000
:1000800089560100895601008956010089560100F0
:1000900089560100895601008956010089560100E0
:1000A000295001003D5001006151010085520100BD
:1000B0008956010089560100895601000975010021
:1000C0008956010025770100895601004179010018
:1000D00089560100417A0100895601000150010052
:1000E0008956010089560100895601008956010090
:1000F0008956010089560100895601008956010080
:10010000F906FF1F6111FF1F895601008956010082
:1001100089560100BD62010089560100895601001F
:10012000895601008956010089560100895601004F
:10013000895601008956010089560100895601003F
:100140008956010089560100417B01008956010052
:10015000417C010089560100895601008956010041
:1001600089560100155001005150010089560100C7
:1001700089560100895601008956010089560100FF
:10018000895601007150010089560100895601000D
:1001900089560100895601005B4B4CF220524DF606
:1001A000281010B51A80188000BF00BF574C15F0FA
:1001B0006FFA4FF030612160554B564A5649A360A3
:1001C0004FF47000E260554C0860236813F48072AD
:1001D00004D153484FF4A85102602160514C237858
:1001E000190704D594F800C04CF0080222704E495B
:1001F0004E4C4F4B2A2008704E498B4204D254F883
:10020000040F43F8040BF8E74B4A4C4800248242A1
:1002100002D242F8044BFAE7494B4A4A002452F80A
:10022000240043F824000134662CF8D1464C474999
:100230004FF0800E04F801EB8C42FBD1444C454B4F
:100240003F4A1A60A4F5805C8A202421A0222070F5
:100250008CF801108CF800209CF806309A07FBD52A
:100260009CF80600C406FBD43B4CA1793A4B01F044
:100270000C02082AF9D10320462418715C7199797F
:100280008806FCD5344A9079334B4106FBD5334A76
:100290004FF08274092120201460516018709C79FD
:1002A00004F00C020C2AFAD12D4B2E4C2E49196069
:1002B0002E482F4B206000220721626044F8041C66
:1002C000C4F80C3D62B615F097FA15480468E207C9
:1002D00005D5284815F07EFA2749284A0A60284B98
:1002E0001878430609D5244C244922688A4204D14F
:1002F000204815F06FFA0023236019F0F5FC15F083
:10030000CDF915F0EFF8FEE70E20054030800440EF
:10031000823F04000100002B88ED00E010D0034074
:1003200014D0034002D0074000E00740DC35020053
:10033000F806FF1F202AFF1F202AFF1F946AFF1FB5
:100340000002FF1F0000000000E400E056E400E0AF
:100350000050064008ED00E00040064044800440A4
:100360000480044014E000E0C0100500BFD4010088
:10037000000020203F316C671CE00340A5C3945A65
:1003800000F00740FFFFFFFFFFFFFFFFFFFFFFFF42
:10039000FFFFFFFFFFFFFFFFFFFFFFFFFFFFFFFF6D
:1003A000FFFFFFFFFFFFFFFFFFFFFFFFFFFFFFFF5D
:1003B000FFFFFFFFFFFFFFFFFFFFFFFFFFFFFFFF4D
:1003C000FFFFFFFFFFFFFFFFFFFFFFFFFFFFFFFF3D
:1003D000FFFFFFFFFFFFFFFFFFFFFFFFFFFFFFFF2D
:1003E000FFFFFFFFFFFFFFFFFFFFFFFFFFFFFFFF1D
:1003F000FFFFFFFFFFFFFFFFFFFFFFFFFFFFFFFF0D
:10040000FFFFFFFFFFFFFFFFFFFFFFFFDEF9FFFF23
:1004100010B5054C237833B9044B13B10448AFF33E
:1004200000800123237010BD202AFF1F0000000060
:10043000D8350200084B10B51BB108490848AFF386
:1004400000800848036803B910BD074B002BFBD0A0
:10045000BDE81040184700BF00000000242AFF1F1D
:10046000D8350200202AFF1F00000000704700BF9F
:10047000704700BFD0F888328169027DF0B4D0F8AF
:1004800084620F69114C00EBC30501339E4298BF93
:1004900000232D6A00EBC30C2F804D26C0F8883254
:1004A000DCF81C0006FB0244225C02F01F031F2B39
:1004B00009D017064ABFCF68102727F0100743F06E
:1004C0004005CF600D60F0BC704700BFB02A02004D
:1004D000034B586810B101680A681047704700BFA5
:1004E000EC64FF1F034B986810B101680A6810475D
:1004F000704700BFEC64FF1F034BD86810B1016860
:100500000A681047704700BFEC64FF1F034B18696F
:1005100010B101680A681047704700BFEC64FF1F04
:10052000034B586910B101680A681047704700BF53
:10053000EC64FF1F034B986910B101680A6810470B
:10054000704700BFEC64FF1F034BD86910B101680E
:100550000A681047704700BFEC64FF1F034B186A1E
:1005600010B101680A681047704700BFEC64FF1FB4
:10057000034B586A10B101680A681047704700BF02
:10058000EC64FF1F034B986A10B101680A681047BA
:10059000704700BFEC64FF1F034BD86A10B10168BD
:1005A0000A681047704700BFEC64FF1F034B186BCD
:1005B00010B101680A681047704700BFEC64FF1F64
:1005C000034B586B10B101680A681047704700BFB1
:1005D000EC64FF1F034B986B10B101680A68104769
:1005E000704700BFEC64FF1F034BD86B10B101686C
:1005F0000A681047704700BFEC64FF1F034B186C7C
:1006000010B101680A681047704700BFEC64FF1F13
:10061000034B586C10B101680A681047704700BF5F
:10062000EC64FF1F034B986C10B101680A68104717
:10063000704700BFEC64FF1F034BD86C10B101681A
:100640000A681047704700BFEC64FF1F034B186D2A
:1006500010B101680A681047704700BFEC64FF1FC3
:10066000034B586D10B101680A681047704700BF0E
:10067000EC64FF1F034B986D10B101680A681047C6
:10068000704700BFEC64FF1F034BD86D10B10168C9
:100690000A681047704700BFEC64FF1F034B186ED9
:1006A00010B101680A681047704700BFEC64FF1F73
:1006B000034B586E10B101680A681047704700BFBD
:1006C000EC64FF1F034B986E10B101680A68104775
:1006D000704700BFEC64FF1F034BD86E10B1016878
:1006E0000A681047704700BFEC64FF1F034B186F88
:1006F00010B101680A681047704700BFEC64FF1F23
:10070000034B586F10B101680A681047704700BF6B
:10071000EC64FF1F034B986F10B101680A68104723
:10072000704700BFEC64FF1F034BD86F10B1016826
:100730000A681047704700BFEC64FF1F034BD3F8F3
:10074000800010B101680A6810477047EC64FF1F11
:10075000034BD3F8840010B101680A681047704752
:10076000EC64FF1F034BD3F8880010B101680A68DE
:1007700010477047EC64FF1F034BD3F88C0010B197
:1007800001680A6810477047EC64FF1F034BD3F8F9
:10079000900010B101680A6810477047EC64FF1FB1
:1007A000034BD3F8940010B101680A6810477047F2
:1007B000EC64FF1F034BD3F8980010B101680A687E
:1007C00010477047EC64FF1F034BD3F89C0010B137
:1007D00001680A6810477047EC64FF1F034BD3F8A9
:1007E000A00010B101680A6810477047EC64FF1F51
:1007F000034BD3F8A40010B101680A681047704792
:10080000EC64FF1F034BD3F8A80010B101680A681D
:1008100010477047EC64FF1F034BD3F8AC0010B1D6
:1008200001680A6810477047EC64FF1F034BD3F858
:10083000B00010B101680A6810477047EC64FF1FF0
:10084000034BD3F8B40010B101680A681047704731
:10085000EC64FF1F034BD3F8B80010B101680A68BD
:1008600010477047EC64FF1F034BD3F8BC0010B176
:1008700001680A6810477047EC64FF1F034BD3F808
:10088000C00010B101680A6810477047EC64FF1F90
:10089000034BD3F8C40010B101680A6810477047D1
:1008A000EC64FF1F034BD3F8C80010B101680A685D
:1008B00010477047EC64FF1F034BD3F8CC0010B116
:1008C00001680A6810477047EC64FF1F034BD3F8B8
:1008D000D00010B101680A6810477047EC64FF1F30
:1008E000034BD3F8D40010B101680A681047704771
:1008F000EC64FF1F034BD3F8D80010B101680A68FD
:1009000010477047EC64FF1F034BD3F8DC0010B1B5
:1009100001680A6810477047EC64FF1F034BD3F867
:10092000E00010B101680A6810477047EC64FF1FCF
:10093000034BD3F8E40010B101680A681047704710
:10094000EC64FF1F034BD3F8E80010B101680A689C
:1009500010477047EC64FF1F034BD3F8EC0010B155
:1009600001680A6810477047EC64FF1F4368074A34
:10097000D8B211F0FF0F52F830304FF0010014BF21
:1009800083F8800083F80001704700BFFC2E02004E
:10099000C9B2007915F036BB08B5007915F024FB13
:1009A00008BD00BF374B1B6830B42BB193F87010F3
:1009B000C27819B9162A3FD030BC704793F87140FD
:1009C0001CB9162A3CD030BC704702F1FF3C0179BB
:1009D000BCF1160FF0D801A050F82CF06B0A000003
:1009E000550A0000B9090000B9090000B909000062
:1009F000B9090000B9090000B9090000B9090000EF
:100A0000B9090000B9090000B9090000B9090000DE
:100A1000B9090000B9090000B9090000B9090000CE
:100A2000B9090000B9090000B9090000B9090000BE
:100A3000410A00004D0A000093F87150002DC4D106
:100A4000012183F8701083F87110B5E7002083F856
:100A50007100B1E70C4A43F2864543F6CC0400200E
:100A600083F8720050551151A6E7074A43F2864CAD
:100A700043F6D005002483F8724002F80C4051512F
:100A80009AE700BFC02AFF1FF82AFF1F90F86430C2
:100A9000002B43D010B48268334C92F802C0334923
:100AA0000CF0FE039370026E13792370046E2279AA
:100AB0000A708368D978090618D4DC78220615D420
:100AC00093F803C05FEA0C6410D4DA7811060DD4F1
:100AD000D9780A060AD4DC78240607D493F803C030
:100AE0005FEA0C6102D4DA781206E3D5016E204B7E
:100AF0000C791C7081680222CA70846894F802C064
:100B00000CF0C703A370836842F21071DA78920682
:100B100005D4002480F864405DF8044B7047DC780D
:100B2000A406F6D593F803C05FEA8C62F1D5DA78B3
:100B30009406EED5DC78A206EBD593F803C05FEA05
:100B40008C64E6D5DA789206E3D5DC78A406E0D5A5
:100B50000839DBD1997000BF83688021997000BF8C
:100B600001220273D5E700BF1F8000401A800040B9
:100B70001C800040D0F884328BB390F814C0184920
:100B800070B4D0F88852846900EB8C0200EBC50089
:100B9000D268C56920684D2606FB0C1C53099900D4
:100BA0001CF8055001F1604606F5614C02F01F0289
:100BB000012305F01F0140F0400003FA02F61F294F
:100BC0002060CCF8006009D02D064ABFE5681025EA
:100BD00025F0100541F04002E560226070BC7047CE
:100BE000B02A020038B5437B85689C1E012CEA7848
:100BF000A97902D90223EB7038BD5FFA82FC5FEA63
:100C0000CC642AD45FEA4C632DD4CBB213F0500FDE
:100C1000044612D0A87940F05002AA71A568A979BB
:100C200001F0DF03AB71A0680222C27025690DB12B
:100C3000606DA8470221A5686173636D3F2B04D8DE
:100C4000581C606523442A791A75A97941F050032C
:100C5000AB71A4680225E57038BD1022EA705FEA26
:100C60004C621CD5856800214165816595F806C0F8
:100C70004CF02003AB718468C025A57081680A79A7
:100C8000530880F85C308C7944F050058D71816890
:100C90004222CA7084680323A279437338BD8568F1
:100CA000A97941F05002AA7180680224C47038BD4D
:100CB000B5EEC00AF1EE10FA2DE9F04700F1F08030
:100CC000FDEEC07ADFF8E4C1F8EEE70A17EE903ADD
:100CD00030EE600A00F1FF3E00248CFB0321DA179E
:100CE000C2EBA1088CFB08254FEAE876C6EBA50508
:100CF0008CFB0527E917C1EBA7068CFB0629F21729
:100D0000C2EBA90708EB880A05EB8509A3EB4A03A8
:100D100006EB860207EB8701A8EB490AA6EB410127
:100D20003033A5EB42020AF130098EF8013001F1AF
:100D3000300A3032611C0EF10103B8F1000F12D0FD
:100D40000C4683F801900B46013165B10C468EF8D4
:100D5000032001313EB19C1CD91C0EF804AF3B4668
:100D60000FB10C46B9E75FEA61087ED0461802462B
:100D700016F801CD077802F801CB08F1FF35804461
:100D80009045377005F007036FD0BBB3012B2DD012
:100D9000022B25D0032B1DD0042B15D0052B0DD0F5
:100DA000062B05D0157816F8019D02F8019B3570C9
:100DB000137816F801AD02F801AB3370157816F808
:100DC00001CD02F801CB3570137816F8017D02F8D9
:100DD000017B3370157816F8013D02F8013B357040
:100DE000157816F8019D02F8019B357016F801ADD3
:100DF000177802F801AB9045377036D0134616F8D5
:100E0000015C177803F8015B06F8017C557816F849
:100E1000027C577006F8025C5D7816F803EC83F8E4
:100E200001E006F8035CD37816F8047CD77006F866
:100E3000043C92F804C016F8055C157106F805CC60
:100E4000537916F8067C577106F8063C92F806901E
:100E500016F8075C957106F8079C16F8083DD779D7
:100E6000D371083290453770C8D1B2EE041A60EEE3
:100E7000011A0E4EBDEEE12A044412EE103A86FB32
:100E80000328DA17C2EBA80A0AEB8A05A3EB450789
:100E900030372E2600234654A770E370BDE8F08754
:100EA0002D230370B1EE400A013009E767666666DC
:100EB00001380B463A2800F25C82DFE810F053025A
:100EC0004C0245023E0237023002290222021B0276
:100ED000AE01A701A001990192018B0184017D015E
:100EE00076016F01680161015A0153014C0145010E
:100EF0003E0137013001290122011B0113010B01C1
:100F00000301FB00F300EB00E300DB00D300CB00A8
:100F1000C300BB00B300AB00A3009B0093008B0099
:100F200083007B0073006B0063005B0053004B0089
:100F300043003B00BC48BD49C0F8EC201A463B20AA
:100F400014F0C8BBB848BA49C0F8E8201A463A209D
:100F500014F0C0BBB448B749C0F8E4201A463920A1
:100F600014F0B8BBB048B449C0F8E0201A463820A5
:100F700014F0B0BBAC48B149C0F8DC201A463720A9
:100F800014F0A8BBA848AE49C0F8D8201A463620AD
:100F900014F0A0BBA448AB49C0F8D4201A463520B1
:100FA00014F098BBA048A849C0F8D0201A463420B5
:100FB00014F090BB9C48A549C0F8CC201A463320B9
:100FC00014F088BB9848A249C0F8C8201A463220BD
:100FD00014F080BB94489F49C0F8C4201A463120C1
:100FE00014F078BB90489C49C0F8C0201A463020C5
:100FF00014F070BB8C489949C0F8BC201A462F20C9
:1010000014F068BB88489649C0F8B8201A462E20CC
:1010100014F060BB84489349C0F8B4201A462D20D0
:1010200014F058BB80489049C0F8B0201A462C20D4
:1010300014F050BB7C488D49C0F8AC201A462B20D8
:1010400014F048BB78488A49C0F8A8201A462A20DC
:1010500014F040BB74488749C0F8A4201A462920E0
:1010600014F038BB70488449C0F8A0201A462820E4
:1010700014F030BB6C488149C0F89C201A462720E8
:1010800014F028BB68487E49C0F898201A462620EC
:1010900014F020BB64487B49C0F894201A462520F0
:1010A00014F018BB60487849C0F890201A462420F4
:1010B00014F010BB5C487549C0F88C201A462320F8
:1010C00014F008BB58487249C0F888201A462220FC
:1010D00014F000BB54486F49C0F884201A46212000
:1010E00014F0F8BA50486C49C0F880201A46202005
:1010F00014F0F0BA4C486949C2671A461F2014F030
:10110000E9BA4948664982671A461E2014F0E2BAD5
:101110004548644942671A461D2014F0DBBA42482C
:10112000614902671A461C2014F0D4BA3E485F4950
:10113000C2661A461B2014F0CDBA3B485C49826651
:101140001A461A2014F0C6BA37485A4942661A4657
:10115000192014F0BFBA3448574902661A461820BD
:1011600014F0B8BA30485549C2651A46172014F031
:10117000B1BA2D48524982651A46162014F0AABA0F
:101180002948504942651A46152014F0A3BA26484A
:101190004D4902651A46142014F09CBA22484B4966
:1011A000C2641A46132014F095BA1F484849826455
:1011B0001A46122014F08EBA1B48464942641A4659
:1011C000112014F087BA1848434902641A461020C7
:1011D00014F080BA14484149C2631A460F2014F033
:1011E00079BA11483E4982631A460E2014F072BA49
:1011F0000D483C4942631A460D2014F06BBA0A4868
:10120000394902631A460C2014F064BA064837497B
:10121000C2621A460B2014F05DBA03483449826258
:101220001A460A2014F056BAEC64FF1F5909000050
:1012300045090000310900001D09000009090000EE
:10124000F5080000E1080000CD080000B908000022
:10125000A5080000910800007D0800006908000052
:1012600055080000410800002D0800001908000082
:1012700005080000F1070000DD070000C9070000B5
:10128000B5070000A10700008D07000079070000E6
:1012900065070000510700003D0700002907000016
:1012A0001507000001070000ED060000D906000048
:1012B000C5060000B10600009D060000890600007A
:1012C00075060000610600004D06000039060000AA
:1012D0002506000011060000FD050000E9050000DC
:1012E000D5050000C1050000AD050000990500000E
:1012F000850500001F48204942621A46092014F063
:10130000E9B91C481D4902621A46082014F0E2B9E6
:1013100018481B49C2611A46072014F0DBB915486A
:10132000184982611A46062014F0D4B911481649AA
:1013300042611A46052014F0CDB90E4813490261E6
:101340001A46042014F0C6B90A481149C2601A4668
:10135000032014F0BFB907480E4982601A460220E4
:1013600014F0B8B903480C4942601A46012014F041
:10137000B1B97047EC64FF1F710500005D05000006
:101380004905000035050000210500000D0500009D
:10139000F9040000E5040000D104000008B513467C
:1013A00040680A461946FFF783FD08BD826810B4FD
:1013B00042F210730446D17888060AD5D0788106A7
:1013C00007D592F803C05FEA8C6002D5D178890610
:1013D0002BD4B0239370A26842F2107392F803C02A
:1013E0005FEA8C601BD4D178890618D4D078800647
:1013F00015D492F803C05FEA8C6110D4D1788806C6
:101400000DD4D07881060AD492F803C05FEA8C60CC
:1014100005D4D178890602D4083BDFD115E0D47811
:10142000C4F340105DF8044B7047D0788006D0D5E7
:1014300092F803C05FEA8C61CBD5D1788806C8D515
:10144000D0788106C5D5083BB5D1937000BFA2689E
:101450008020907000BF0121184621735DF8044B75
:10146000704700BF3C2370B5037191F864608260DF
:1014700004460D460160002E04F0B6828B6842F2ED
:101480001070DD782D0623D4DE78320620D493F850
:1014900003C05FEA0C661BD4DA78150618D4DD7831
:1014A0002A0615D4DE78360612D493F803C05FEA14
:1014B0000C650DD4DA7812060AD40838E1D1987098
:1014C00000BF88688022827000BF01230B7328E070
:1014D0000220D8708D68AB7843F01006AE70886833
:1014E000002202718A6842F21070D578AB0708D4E6
:1014F00092F803C05FEA8C7603D4D3789E0741F15B
:101500008B83D57802205FFA85FCD0701CF0100226
:1015100045F034805FEACC7505F1238089680225A7
:10152000CD7021688B6842F21070DE78320602F1CD
:101530002584DD782E0602F1218493F803C05FEA4A
:101540000C6602F11B84DA78150602F11784DE7846
:10155000320602F11384DD782E0602F10F8493F82F
:1015600003C05FEA0C6502F10984DA78120602F121
:1015700005840838D9D1987000BF886880228270AD
:1015800000BF01230B7321688D68AE7806F0C70099
:10159000A8708B6842F2107093F803C05FEA8C6504
:1015A00002F18985256895F86410002902F0B2855A
:1015B000AB6842F21071D878000602F1B183DE7890
:1015C000320602F1AD8393F803C05FEA0C6002F1CA
:1015D000A783DA78120602F1A383D878060602F10F
:1015E0009F83DE78300602F19B8393F803C05FEAA5
:1015F0000C6202F19583DA78160602F191830839BC
:10160000D9D1997000BFA96880228A7000BF0123D8
:101610002B7321688B6842F21070DE78320602F17B
:101620005183DD782E0602F14D8393F803C05FEA03
:101630000C6202F14783DA78160602F14383DE7802
:10164000350602F13F83DD782A0602F13B8393F8E9
:1016500003C05FEA0C6602F13583DA78150602F101
:1016600031830838D9D1987000BF88688022827091
:1016700000BF01230B7321688D68AE7806F0C700A8
:10168000A8708B6842F2107093F803C05FEA8C6513
:1016900002F1A584256895F86410002902F0CE8433
:1016A000AB6842F21071D878000602F1DD82DE7874
:1016B000320602F1D98293F803C05FEA0C6002F1AE
:1016C000D382DA78120602F1CF82D878060602F1C8
:1016D000CB82DE78300602F1C78293F803C05FEA5E
:1016E0000C6202F1C182DA78160602F1BD82083975
:1016F000D9D1997000BFA96880228A7000BF0123E8
:101700002B7321688B6842F21070DE78320602F18A
:101710007D82DD782E0602F1798293F803C05FEABC
:101720000C6202F17382DA78160602F16F82DE78BB
:10173000350602F16B82DD782A0602F1678293F8A2
:1017400003C05FEA0C6602F16182DA78150602F1E5
:101750005D820838D9D1987000BF88688022827075
:1017600000BF01230B7321688D68AE7806F0C700B7
:10177000A8708B6842F2107093F803C05FEA8C6522
:1017800002F1C183256895F86410002902F0EA830C
:10179000AB6842F21071D878000602F10982DE7857
:1017A000320602F1058293F803C05FEA0C6002F191
:1017B000FF81DA78120602F1FB81D878060602F181
:1017C000F781DE78300602F1F38193F803C05FEA17
:1017D0000C6202F1ED81DA78160602F1E98108392E
:1017E000D9D1997000BFA96880228A7000BF0123F7
:1017F0002B7321688B6842F21070DE78320602F19A
:10180000A981DD782E0602F1A58193F803C05FEA75
:101810000C6202F19F81DA78160602F19B81DE7874
:10182000350602F19781DD782A0602F1938193F85B
:1018300003C05FEA0C6602F18D81DA78150602F1C9
:1018400089810838D9D1987000BF88688022827059
:1018500000BF01230B7321688D68AE7806F0C700C6
:10186000A8708B6842F2107093F803C05FEA8C6531
:1018700002F1DD82256895F86410002902F00683E4
:10188000AB6842F21071D878000602F13581DE783B
:10189000320602F1318193F803C05FEA0C6002F175
:1018A0002B81DA78120602F12781D878060602F138
:1018B0002381DE78300602F11F8193F803C05FEACE
:1018C0000C6202F11981DA78160602F115810839E5
:1018D000D9D1997000BFA96880228A7000BF012306
:1018E0002B7321688B6842F21070DE78320602F1A9
:1018F000D580DD782E0602F1D18093F803C05FEA2F
:101900000C6202F1CB80DA78160602F1C780DE782D
:10191000350602F1C380DD782A0602F1BF8093F814
:1019200003C05FEA0C6602F1B980DA78150602F1AD
:10193000B5800838D9D1987000BF8868802282703D
:1019400000BF01230B7321688D68AE7806F0C700D5
:10195000A8708B6842F2107093F803C05FEA8C6540
:1019600002F15985256895F86410002902F08285F6
:10197000AB6842F21071D878000602F16180DE781F
:10198000320602F15D8093F803C05FEA0C6002F159
:101990005780DA78120602F15380D878060602F1F1
:1019A0004F80DE78300602F14B8093F803C05FEA87
:1019B0000C6202F14580DA78160602F1418008399E
:1019C000D9D1997000BFA96880228A7000BF012315
:1019D0002B7321688B6842F21070DE78320602F1B8
:1019E0000180DD782E0601F1FD8793F803C05FEAE0
:1019F0000C6201F1F787DA78160601F1F387DE78D9
:101A0000350601F1EF87DD782A0601F1EB8793F8BF
:101A100003C05FEA0C6601F1E587DA78150601F18B
:101A2000E1870838D9D1987000BF88688022827019
:101A300000BF01230B7321688D68AE7806F0C700E4
:101A4000A8708B6842F2107093F803C05FEA8C654F
:101A500002F17584256895F86410002902F09E84CF
:101A6000AB6842F21071D878000601F18D87DE78FC
:101A7000320601F1898793F803C05FEA0C6001F137
:101A80008387DA78120601F17F87D878060601F19C
:101A90007B87DE78300601F1778793F803C05FEA31
:101AA0000C6201F17187DA78160601F16D87083949
:101AB000D9D1997000BFA96880228A7000BF012324
:101AC0002B7321688B6842F21070DE78320601F1C8
:101AD0002D87DD782E0601F1298793F803C05FEA90
:101AE0000C6201F12387DA78160601F11F87DE7890
:101AF000350601F11B87DD782A0601F1178793F877
:101B000003C05FEA0C6601F11187DA78150601F16E
:101B10000D870838D9D1987000BF886880228270FC
:101B200000BF01230B7321688D68AE7806F0C700F3
:101B3000A8708B6842F2107093F803C05FEA8C655E
:101B400002F19183256895F86410002902F0BA83A8
:101B5000AB6842F21071D878000601F1B986DE78E0
:101B6000320601F1B58693F803C05FEA0C6001F11B
:101B7000AF86DA78120601F1AB86D878060601F155
:101B8000A786DE78300601F1A38693F803C05FEAEA
:101B90000C6201F19D86DA78160601F19986083902
:101BA000D9D1997000BFA96880228A7000BF012333
:101BB0002B7321688B6842F21070DE78320601F1D7
:101BC0005986DD782E0601F1558693F803C05FEA49
:101BD0000C6201F14F86DA78160601F14B86DE7849
:101BE000350601F14786DD782A0601F1438693F830
:101BF00003C05FEA0C6601F13D86DA78150601F153
:101C000039860838D9D1987000BF886880228270E0
:101C100000BF01230B7321688D68AE7806F0C70002
:101C2000A8708B6842F2107093F803C05FEA8C656D
:101C300002F1AD82256895F86410002902F0D68281
:101C4000AB6842F21071D878000601F1E585DE78C4
:101C5000320601F1E18593F803C05FEA0C6001F1FF
:101C6000DB85DA78120601F1D785D878060601F10E
:101C7000D385DE78300601F1CF8593F803C05FEAA3
:101C80000C6201F1C985DA78160601F1C5850839BB
:101C9000D9D1997000BFA96880228A7000BF012342
:101CA0002B7321688B6842F21070DE78320601F1E6
:101CB0008585DD782E0601F1818593F803C05FEA02
:101CC0000C6201F17B85DA78160601F17785DE7802
:101CD000350601F17385DD782A0601F16F8593F8E9
:101CE00003C05FEA0C6601F16985DA78150601F137
:101CF00065850838D9D1987000BF886880228270C5
:101D000000BF01230B7321688D68AE7806F0C70011
:101D1000A8708B6842F2107093F803C05FEA8C657C
:101D200002F12985256895F86410002902F0528592
:101D3000AB6842F21071D878000601F11185DE78A7
:101D4000320601F10D8593F803C05FEA0C6001F1E2
:101D50000785DA78120601F10385D878060601F1C5
:101D6000FF84DE78300601F1FB8493F803C05FEA5C
:101D70000C6201F1F584DA78160601F1F184083974
:101D8000D9D1997000BFA96880228A7000BF012351
:101D90002B7321688B6842F21070DE78320601F1F5
:101DA000B184DD782E0601F1AD8493F803C05FEABB
:101DB0000C6201F1A784DA78160601F1A384DE78BB
:101DC000350601F19F84DD782A0601F19B8493F8A2
:101DD00003C05FEA0C6601F19584DA78150601F11B
:101DE00091840838D9D1987000BF886880228270A9
:101DF00000BF01230B7321688D68AE7806F0C70021
:101E0000A8708B6842F2107093F803C05FEA8C658B
:101E100002F14584256895F86410002902F06E846B
:101E2000AB6842F21071D878000601F13D84DE788B
:101E3000320601F1398493F803C05FEA0C6001F1C6
:101E40003384DA78120601F12F84D878060601F17E
:101E50002B84DE78300601F1278493F803C05FEA13
:101E60000C6201F12184DA78160601F11D8408392B
:101E7000D9D1997000BFA96880228A7000BF012360
:101E80002B7321688B6842F21070DE78320601F104
:101E9000DD83DD782E0601F1D98393F803C05FEA74
:101EA0000C6201F1D383DA78160601F1CF83DE7874
:101EB000350601F1CB83DD782A0601F1C78393F85B
:101EC00003C05FEA0C6601F1C183DA78150601F1FF
:101ED000BD830838D9D1987000BF8868802282708D
:101EE00000BF01230B7321688D68AE7806F0C70030
:101EF000A8708B6842F2107093F803C05FEA8C659B
:101F000002F16183256895F86410002902F08A8344
:101F1000AB6842F21071D878000601F16983DE786F
:101F2000320601F1658393F803C05FEA0C6001F1AA
:101F30005F83DA78120601F15B83D878060601F137
:101F40005783DE78300601F1538393F803C05FEACC
:101F50000C6201F14D83DA78160601F149830839E4
:101F6000D9D1997000BFA96880228A7000BF01236F
:101F70002B7321688B6842F21070DE78320601F113
:101F80000983DD782E0601F1058393F803C05FEA2B
:101F90000C6201F1FF82DA78160601F1FB82DE782D
:101FA000350601F1F782DD782A0601F1F38293F814
:101FB00003C05FEA0C6601F1ED82DA78150601F1E3
:101FC000E9820838D9D1987000BF88688022827071
:101FD00000BF01230B7321688D68AE7806F0C7003F
:101FE000A8708B6842F2107093F803C05FEA8C65AA
:101FF00002F17D82256895F86410002902F0A6821E
:10200000AB6842F21071D878000601F19582DE7853
:10201000320601F1918293F803C05FEA0C6001F18E
:102020008B82DA78120601F18782D878060601F1F0
:102030008382DE78300601F17F8293F803C05FEA85
:102040000C6201F17982DA78160601F1758208399D
:10205000D9D1997000BFA96880228A7000BF01237E
:102060002B7321688B6842F21070DE78320601F122
:102070003582DD782E0601F1318293F803C05FEAE4
:102080000C6201F12B82DA78160601F12782DE78E4
:10209000350601F12382DD782A0601F11F8293F8CB
:1020A00003C05FEA0C6601F11982DA78150601F1C6
:1020B00015820838D9D1987000BF88688022827054
:1020C00000BF01230B7321688D68AE7806F0C7004E
:1020D000A8708B6842F2107093F803C05FEA8C65B9
:1020E00002F1F984256895F86410002902F0228530
:1020F000AB6842F21071D878000601F1C181DE7838
:10210000320601F1BD8193F803C05FEA0C6001F172
:10211000B781DA78120601F1B381D878060601F1A9
:10212000AF81DE78300601F1AB8193F803C05FEA3E
:102130000C6201F1A581DA78160601F1A181083956
:10214000D9D1997000BFA96880228A7000BF01238D
:102150002B7321688B6842F21070DE78320601F131
:102160006181DD782E0601F15D8193F803C05FEA9D
:102170000C6201F15781DA78160601F15381DE789D
:10218000350601F14F81DD782A0601F14B8193F884
:1021900003C05FEA0C6601F14581DA78150601F1AA
:1021A00041810838D9D1987000BF88688022827038
:1021B00000BF01230B7321688D68AE7806F0C7005D
:1021C000A8708B6842F2107093F803C05FEA8C65C8
:1021D00002F11584256895F86410002902F03E8408
:1021E000AB6842F21071D878000601F1ED80DE781C
:1021F000320601F1E98093F803C05FEA0C6001F157
:10220000E380DA78120601F1DF80D878060601F162
:10221000DB80DE78300601F1D78093F803C05FEAF7
:102220000C6201F1D180DA78160601F1CD8008390F
:10223000D9D1997000BFA96880228A7000BF01239C
:102240002B7321688B6842F21070DE78320601F140
:102250008D80DD782E0601F1898093F803C05FEA56
:102260000C6201F18380DA78160601F17F80DE7856
:10227000350601F17B80DD782A0601F1778093F83D
:1022800003C05FEA0C6601F17180DA78150601F18E
:102290006D800838D9D1987000BF8868802282701C
:1022A00000BF01230B7321688D68AE7806F0C7006C
:1022B000A8708B6842F2107093F803C05FEA8C65D7
:1022C00002F13183256895F86410002902F05A83E1
:1022D000AB6842F21071D878000601F11980DE78FF
:1022E000320601F1158093F803C05FEA0C6001F13A
:1022F0000F80DA78120601F10B80D878060601F11A
:102300000780DE78300601F1038093F803C05FEAAE
:102310000C6200F1FD87DA78160600F1F9870839BA
:10232000D9D1997000BFA96880228A7000BF0123AB
:102330002B7321688B6842F21070DE78320600F150
:10234000B987DD782E0600F1B58793F803C05FEA00
:102350000C6200F1AF87DA78160600F1AB87DE7801
:10236000350600F1A787DD782A0600F1A38793F8E8
:1023700003C05FEA0C6600F19D87DA78150600F16C
:1023800099870838D9D1987000BF886880228270F8
:1023900000BF01230B7321688D68AE7806F0C7007B
:1023A000A8708B6842F2107093F803C05FEA8C65E6
:1023B00002F14D82256895F86410002902F07682BA
:1023C000AB6842F21071D878000600F14587DE78DC
:1023D000320600F1418793F803C05FEA0C6000F118
:1023E0003B87DA78120600F13787D878060600F1C5
:1023F0003387DE78300600F12F8793F803C05FEA59
:102400000C6200F12987DA78160600F12587083971
:10241000D9D1997000BFA96880228A7000BF0123BA
:102420002B7321688B6842F21070DE78320600F15F
:10243000E586DD782E0600F1E18693F803C05FEAB9
:102440000C6200F1DB86DA78160600F1D786DE78BA
:10245000350600F1D386DD782A0600F1CF8693F8A1
:1024600003C05FEA0C6600F1C986DA78150600F150
:10247000C5860838D9D1987000BF886880228270DC
:1024800000BF01230B7321688D68AE7806F0C7008A
:10249000A8708B6842F2107093F803C05FEA8C65F5
:1024A00002F1C684256895F86410002902F0EF84D3
:1024B000AB6842F21071D878000600F17186DE78C0
:1024C000320600F16D8693F803C05FEA0C6000F1FC
:1024D0006786DA78120600F16386D878060600F17E
:1024E0005F86DE78300600F15B8693F803C05FEA12
:1024F0000C6200F15586DA78160600F1518608392B
:10250000D9D1997000BFA96880228A7000BF0123C9
:102510002B7321688B6842F21070DE78320600F16E
:102520001186DD782E0600F10D8693F803C05FEA70
:102530000C6200F10786DA78160600F10386DE7871
:10254000350600F1FF85DD782A0600F1FB8593F85A
:1025500003C05FEA0C6600F1F585DA78150600F134
:10256000F1850838D9D1987000BF886880228270C0
:1025700000BF01230B7321688D68AE7806F0C70099
:10258000A8708B6842F2107093F803C05FEA8C6504
:1025900002F1E383256895F86410002902F00C84A9
:1025A000AB6842F21071D878000600F19D85DE78A4
:1025B000320600F1998593F803C05FEA0C6000F1E0
:1025C0009385DA78120600F18F85D878060600F137
:1025D0008B85DE78300600F1878593F803C05FEACB
:1025E0000C6200F18185DA78160600F17D850839E4
:1025F000D9D1997000BFA96880228A7000BF0123D9
:102600002B7321688B6842F21070DE78320600F17D
:102610003D85DD782E0600F1398593F803C05FEA29
:102620000C6200F13385DA78160600F12F85DE782A
:10263000350600F12B85DD782A0600F1278593F811
:1026400003C05FEA0C6600F12185DA78150600F117
:102650001D850838D9D1987000BF886880228270A3
:1026600000BF01230B7321688D68AE7806F0C700A8
:10267000A8708B6842F2107093F803C05FEA8C6513
:1026800002F10083256895F86410002902F029837F
:10269000AB6842F21071D878000600F1C984DE7888
:1026A000320600F1C58493F803C05FEA0C6000F1C4
:1026B000BF84DA78120600F1BB84D878060600F1F0
:1026C000B784DE78300600F1B38493F803C05FEA84
:1026D0000C6200F1AD84DA78160600F1A98408399D
:1026E000D9D1997000BFA96880228A7000BF0123E8
:1026F0002B7321688B6842F21070DE78320600F18D
:102700006984DD782E0600F1658493F803C05FEAE2
:102710000C6200F15F84DA78160600F15B84DE78E3
:10272000350600F15784DD782A0600F1538493F8CA
:1027300003C05FEA0C6600F14D84DA78150600F1FB
:1027400049840838D9D1987000BF88688022827087
:1027500000BF01230B7321688D68AE7806F0C700B7
:10276000A8708B6842F2107093F803C05FEA8C6522
:1027700002F11D82256895F86410002902F0468256
:10278000AB6842F21071D878000600F1F683DE786B
:10279000320600F1F28393F803C05FEA0C6000F1A7
:1027A000EC83DA78120600F1E883D878060600F1A7
:1027B000E483DE78300600F1E08393F803C05FEA3B
:1027C0000C6200F1DA83DA78160600F1D683083954
:1027D000D9D1997000BFA96880228A7000BF0123F7
:1027E0002B7321688B6842F21070DE78320600F19C
:1027F0009783DD782E0600F1938393F803C05FEA98
:102800000C6200F18D83DA78160600F18983DE7898
:10281000350600F18583DD782A0600F1818393F87F
:1028200003C05FEA0C6600F17B83DA78150600F1DD
:1028300077830838D9D1987000BF88688022827069
:1028400000BF01230B7321688D68AE7806F0C700C6
:10285000A8708B6842F2107093F803C05FEA8C6531
:1028600002F18B84256895F86410002902F0B48485
:10287000AB6842F21071D878000600F12483DE784C
:10288000320600F1208393F803C05FEA0C6000F188
:102890001A83DA78120600F11683D878060600F15A
:1028A0001283DE78300600F10E8393F803C05FEAEE
:1028B0000C6200F10883DA78160600F10483083907
:1028C000D9D1997000BFA96880228A7000BF012306
:1028D0002B7321688B6842F21070DE78320600F1AB
:1028E000C582DD782E0600F1C18293F803C05FEA4D
:1028F0000C6200F1BB82DA78160600F1B782DE784E
:10290000350600F1B382DD782A0600F1AF8293F834
:1029100003C05FEA0C6600F1A982DA78150600F1BF
:10292000A5820838D9D1987000BF8868802282704B
:1029300000BF01230B7321688D68AE7806F0C700D5
:10294000A8708B6842F2107093F803C05FEA8C6540
:1029500002F1AF83256895F86410002902F0D8834E
:10296000AB6842F21071D878000600F15282DE782E
:10297000320600F14E8293F803C05FEA0C6000F16A
:102980004882DA78120600F14482D878060600F10F
:102990004082DE78300600F13C8293F803C05FEAA3
:1029A0000C6200F13682DA78160600F132820839BC
:1029B000D9D1997000BFA96880228A7000BF012315
:1029C0002B7321688B6842F21070DE78320600F1BA
:1029D000F381DD782E0600F1EF8193F803C05FEA02
:1029E0000C6200F1E981DA78160600F1E581DE7803
:1029F000350600F1E181DD782A0600F1DD8193F8EA
:102A000003C05FEA0C6600F1D781DA78150600F1A1
:102A1000D3810838D9D1987000BF8868802282702D
:102A200000BF01230B7321688D68AE7806F0C700E4
:102A3000A8708B6842F2107093F803C05FEA8C654F
:102A400002F1CC82256895F86410002902F0F58225
:102A5000AB6842F21071D878000600F18081DE7810
:102A6000320600F17C8193F803C05FEA0C6000F14C
:102A70007681DA78120600F17281D878060600F1C4
:102A80006E81DE78300600F16A8193F803C05FEA58
:102A90000C6200F16481DA78160600F16081083971
:102AA000D9D1997000BFA96880228A7000BF012324
:102AB0002B7321688B6842F21070DE78320600F1C9
:102AC0002181DD782E0600F11D8193F803C05FEAB5
:102AD0000C6200F11781DA78160600F11381DE78B6
:102AE000350600F10F81DD782A0600F10B8193F89D
:102AF00003C05FEA0C6600F10581DA78150600F183
:102B000001810838D9D1987000BF8868802282700E
:102B100000BF01230B7321688D68AE7806F0C700F3
:102B2000A8708B6842F2107093F803C05FEA8C655E
:102B300002F1E981256895F86410002902F01282FB
:102B4000AB6842F21071D878000600F1AE80DE78F2
:102B5000320600F1AA8093F803C05FEA0C6000F12E
:102B6000A480DA78120600F1A080D878060600F179
:102B70009C80DE78300600F1988093F803C05FEA0D
:102B80000C6200F19280DA78160600F18E80083926
:102B9000D9D1997000BFA96880228A7000BF012333
:102BA0002B7321688B6842F21070DE7832064FD4A6
:102BB000DD782E064CD493F803C05FEA0C6247D44C
:102BC000DA78160644D4DE78350641D4DD782A0654
:102BD0003ED493F803C05FEA0C6639D4DA78150660
:102BE00036D40838E1D1987000BF8868802282709E
:102BF00000BF01230B7321688D68AE7806F0C70013
:102C0000A8708B6842F2107093F803C05FEA8C657D
:102C100001F1E280204670BDD678B5073EF571AC73
:102C2000D578AB073EF56DAC92F803C05FEA8C76C1
:102C30003EF567ACD3789D073EF563ACD678B30715
:102C40003EF55FAC08387EF450AC9070FEF738BCAF
:102C50000220D8708E68B37843F01005B57088688C
:102C6000AF2202718A6842F21070D678B5070BD491
:102C700092F803C05FEA8C7306D4D3789B0703D421
:102C8000D578AE0743F15584D67802205FFA86FCEA
:102C9000D0701CF0100243F0C1875FEACC7603F1DC
:102CA000CC8789680226CE70A5E70221D970A86872
:102CB000837843F010068670A96800220A71AA681A
:102CC00042F21071D07883070BD492F803C05FEA08
:102CD0008C7606D4D378980703D4D678B30743F11B
:102CE0001084D07802215FFA80FCD1701CF01002B1
:102CF00043F0A9875FEACC7003F1B487AD68022086
:102D0000E8704EE70220D8708E68B37843F0100563
:102D1000B5708868A72202718A6842F21070D6786E
:102D2000B5070BD492F803C05FEA8C7306D4D3784E
:102D30009B0703D4D578AE0743F1CB83D678022026
:102D40005FFA86FCD0701CF0100243F03D875FEA0A
:102D5000CC7603F1488789680226CE70DBE6022133
:102D6000D970A868837843F010068670A96800229D
:102D70000A71AA6842F21071D07883070BD492F8D6
:102D800003C05FEA8C7606D4D378980703D4D6784C
:102D9000B30743F18683D07802215FFA80FCD170BB
:102DA0001CF0100243F025875FEACC7003F13087F6
:102DB000AD680220E8707CE60220D8708E68B37897
:102DC00043F01005B5708868A42202718A6842F247
:102DD0001070D678B5070BD492F803C05FEA8C73F5
:102DE00006D4D3789B0703D4D578AE0743F141834B
:102DF000D67802205FFA86FCD0701CF0100243F0F7
:102E000037875FEACC7603F1428789680226CE7065
:102E100009E60221D970A868837843F0100686700D
:102E2000A96800220A71AA6842F21071D07883075B
:102E30000BD492F803C05FEA8C7606D4D378980757
:102E400003D4D678B30743F1FC82D07802215FFA2D
:102E500080FCD1701CF0100243F01F875FEACC7039
:102E600003F12A87AD680220E870AAE50220D87035
:102E70008E68B37843F01005B570886840220271FF
:102E80008A6842F21070D678B5070BD492F803C066
:102E90005FEA8C7306D4D3789B0703D4D578AE074A
:102EA00043F1B782D67802205FFA86FCD0701CF01E
:102EB000100243F007875FEACC7603F11287896836
:102EC0000226CE7037E50221D970A868837843F0D6
:102ED00010068670A96800220A71AA6842F2107171
:102EE000D07883070BD492F803C05FEA8C7606D4BF
:102EF000D378980703D4D678B30743F17282D07899
:102F000002215FFA80FCD1701CF0100243F0EF86C2
:102F10005FEACC7003F1FA86AD680220E870D8E46D
:102F20000220D8708E68B37843F01005B5708868B9
:102F3000DB2202718A6842F21070D678B5070BD492
:102F400092F803C05FEA8C7306D4D3789B0703D44E
:102F5000D578AE0743F12D82D67802205FFA86FC41
:102F6000D0701CF0100243F0B9835FEACC7603F115
:102F7000C48389680226CE7065E40221D970A868EE
:102F8000837843F010068670A96800220A71AA6847
:102F900042F21071D07883070BD492F803C05FEA35
:102FA0008C7606D4D378980703D4D678B30743F148
:102FB000E881D07802215FFA80FCD1701CF0100209
:102FC00043F023835FEACC7003F12E83AD680220C7
:102FD000E87006E40220D8708E68B37843F01005DC
:102FE000B5708868F12202718A6842F21070D67852
:102FF000B5070BD492F803C05FEA8C7306D4D3787C
:103000009B0703D4D578AE0743F1A381D67802207D
:103010005FFA86FCD0701CF0100243F035835FEA43
:10302000CC7603F1408389680226CE70FFF793BB0C
:103030000221D970A868837843F010068670A968C9
:1030400000220A71AA6842F21071D07883070BD46B
:1030500092F803C05FEA8C7606D4D378980703D43D
:10306000D678B30743F15D81D07802215FFA80FC06
:10307000D1701CF0100243F01C835FEACC7003F1A6
:103080002783AD680220E870FFF733BB0220D870B9
:103090008E68B37843F01005B5708868D922027144
:1030A0008A6842F21070D678B5070BD492F803C044
:1030B0005FEA8C7306D4D3789B0703D4D578AE0728
:1030C00043F11781D67802205FFA86FCD0701CF09D
:1030D000100243F021865FEACC7603F12C868968E2
:1030E0000226CE70FFF7BFBA0221D970A868837894
:1030F00043F010068670A96800220A71AA6842F29D
:103100001071D07883070BD492F803C05FEA8C76F5
:1031100006D4D378980703D4D678B30743F1D18087
:10312000D07802215FFA80FCD1701CF0100243F0CD
:1031300008865FEACC7003F11386AD680220E87060
:10314000FFF75FBA0220D8708E68B37843F010059D
:10315000B5708868FF2202718A6842F21070D678D2
:10316000B5070BD492F803C05FEA8C7306D4D3780A
:103170009B0703D4D578AE0743F18B80D678022025
:103180005FFA86FCD0701CF0100243F0EF855FEA16
:10319000CC7603F1FA8589680226CE70FFF7EBB989
:1031A0000221D970A868837843F010068670A96858
:1031B00000220A71AA6842F21071D07883070BD4FA
:1031C00092F803C05FEA8C7606D4D378980703D4CC
:1031D000D678B30743F14580D07802215FFA80FCAE
:1031E000D1701CF0100243F03A825FEACC7003F118
:1031F0004582AD680220E870FFF78BB90220D870D5
:103200008E68B37843F01005B5708868812202712A
:103210008A6842F21070D678B5070BD492F803C0D2
:103220005FEA8C7306D4D3789B0703D4D578AE07B6
:1032300042F1FF87D67802205FFA86FCD0701CF03E
:10324000100243F0F3825FEACC7603F1FE828968D4
:103250000226CE70FFF717B90221D970A8688378CB
:1032600043F010068670A96800220A71AA6842F22B
:103270001071D07883070BD492F803C05FEA8C7684
:1032800006D4D378980703D4D678B30742F1B98728
:10329000D07802215FFA80FCD1701CF0100243F05C
:1032A000DA825FEACC7003F1E582AD680220E87053
:1032B000FFF7B7B80220D8708E68B37843F01005D6
:1032C000B5708868122202718A6842F21070D6784E
:1032D000B5070BD492F803C05FEA8C7306D4D37899
:1032E0009B0703D4D578AE0742F17387D6780220C6
:1032F0005FFA86FCD0701CF0100243F06D825FEA2A
:10330000CC7603F1788289680226CE70FFF743B845
:103310000221D970A868837843F010068670A968E6
:1033200000220A71AA6842F21071D07883070BD488
:1033300092F803C05FEA8C7606D4D378980703D45A
:10334000D678B30742F12D87D07802215FFA80FC4E
:10335000D1701CF0100243F054825FEACC7003F18C
:103360005F82AD680220E870FEF7E3BF0220D870EC
:103370008E68B37843F01005B5708868DA22027160
:103380008A6842F21070D678B5070BD492F803C061
:103390005FEA8C7306D4D3789B0703D4D578AE0745
:1033A00042F1E786D67802205FFA86FCD0701CF0E6
:1033B000100243F065825FEACC7603F1708289687F
:1033C0000226CE70FEF76FBF0221D970A8688378FD
:1033D00043F010068670A96800220A71AA6842F2BA
:1033E0001071D07883070BD492F803C05FEA8C7613
:1033F00006D4D378980703D4D678B30742F1A186D0
:10340000D07802215FFA80FCD1701CF0100243F0EA
:103410004C825FEACC7003F15782AD680220E870FD
:10342000FEF70FBF0220D8708E68B37843F0100506
:10343000B5708868C82202718A6842F21070D67826
:10344000B5070BD492F803C05FEA8C7306D4D37827
:103450009B0703D4D578AE0742F15B86D67802206D
:103460005FFA86FCD0701CF0100243F033825FEAF2
:10347000CC7603F13E8289680226CE70FEF79BBEB1
:103480000221D970A868837843F010068670A96875
:1034900000220A71AA6842F21071D07883070BD417
:1034A00092F803C05FEA8C7606D4D378980703D4E9
:1034B000D678B30742F11586D07802215FFA80FCF6
:1034C000D1701CF0100243F01A825FEACC7003F155
:1034D0002582AD680220E870FEF73BBE0220D8705E
:1034E0008E68B37843F01005B5708868A122027128
:1034F0008A6842F21070D678B5070BD492F803C0F0
:103500005FEA8C7306D4D3789B0703D4D578AE07D3
:1035100042F1CF85D67802205FFA86FCD0701CF08D
:10352000100243F027835FEACC7603F13283896887
:103530000226CE70FEF7C7BD0221D970A868837835
:1035400043F010068670A96800220A71AA6842F248
:103550001071D07883070BD492F803C05FEA8C76A1
:1035600006D4D378980703D4D678B30742F1898577
:10357000D07802215FFA80FCD1701CF0100243F079
:103580000E835FEACC7003F11983AD680220E87006
:10359000FEF767BD0220D8708E68B37843F010053F
:1035A000B5708868012202718A6842F21070D6787C
:1035B000B5070BD492F803C05FEA8C7306D4D378B6
:1035C0009B0703D4D578AE0742F14385D678022015
:1035D0005FFA86FCD0701CF0100243F0A1825FEA13
:1035E000CC7603F1AC8289680226CE70FEF7F3BC7C
:1035F0000221D970A868837843F010068670A96804
:1036000000220A71AA6842F21071D07883070BD4A5
:1036100092F803C05FEA8C7606D4D378980703D477
:10362000D678B30742F1FD84D07802215FFA80FC9E
:10363000D1701CF0100243F088825FEACC7003F175
:103640009382AD680220E870FEF793BC0220D87028
:103650008E68B37843F01005B57088682022027137
:103660008A6842F21070D678B5070BD492F803C07E
:103670005FEA8C7306D4D3789B0703D4D578AE0762
:1036800042F1B784D67802205FFA86FCD0701CF035
:10369000100243F0F1815FEACC7603F1FC81896886
:1036A0000226CE70FEF71FBC0221D970A86883786D
:1036B00043F010068670A96800220A71AA6842F2D7
:1036C0001071D07883070BD492F803C05FEA8C7630
:1036D00006D4D378980703D4D678B30742F171841F
:1036E000D07802215FFA80FCD1701CF0100243F008
:1036F000D8815FEACC7003F1E381AD680220E87005
:10370000FEF7BFBB0220D8708E68B37843F0100577
:10371000B5708868142202718A6842F21070D678F7
:10372000B5070BD492F803C05FEA8C7306D4D37844
:103730009B0703D4D578AE0742F12B84D6780220BC
:103740005FFA86FCD0701CF0100243F0BF815FEA84
:10375000CC7603F1CA8189680226CE70FEF74BBB96
:103760000221D970A868837843F010068670A96892
:1037700000220A71AA6842F21071D07883070BD434
:1037800092F803C05FEA8C7606D4D378980703D406
:10379000D678B30742F1E583D07802215FFA80FC46
:1037A000D1701CF0100243F0A6815FEACC7003F1E7
:1037B000B181AD680220E870FEF7EBBA0220D87044
:1037C0008E68B37843F01005B57088688D22027159
:1037D0008A6842F21070D678B5070BD492F803C00D
:1037E0005FEA8C7306D4D3789B0703D4D578AE07F1
:1037F00042F19F83D67802205FFA86FCD0701CF0DD
:10380000100243F0BB805FEACC7603F1C680896882
:103810000226CE70FEF777BA0221D970A8688378A5
:1038200043F010068670A96800220A71AA6842F265
:103830001071D07883070BD492F803C05FEA8C76BE
:1038400006D4D378980703D4D678B30742F15983C6
:10385000D07802215FFA80FCD1701CF0100243F096
:10386000A2805FEACC7003F1AD80AD680220E87001
:10387000FEF717BA0220D8708E68B37843F01005AF
:10388000B5708868402202718A6842F21070D6785A
:10389000B5070BD492F803C05FEA8C7306D4D378D3
:1038A0009B0703D4D578AE0742F11383D678022064
:1038B0005FFA86FCD0701CF0100243F035805FEA9E
:1038C000CC7603F1408089680226CE70FEF7A3B95A
:1038D0000221D970A868837843F010068670A96821
:1038E00000220A71AA6842F21071D07883070BD4C3
:1038F00092F803C05FEA8C7606D4D378980703D495
:10390000D678B30742F1CD82D07802215FFA80FCED
:10391000D1701CF0100243F01C805FEACC7003F100
:103920002780AD680220E870FEF743B90220D87006
:103930008E68B37843F01005B57088680022027174
:103940008A6842F21070D678B5070BD492F803C09B
:103950005FEA8C7306D4D3789B0703D4D578AE077F
:1039600042F18782D67802205FFA86FCD0701CF084
:10397000100243F02D805FEACC7603F1388089682D
:103980000226CE70FEF7CFB80221D970A8688378DE
:1039900043F010068670A96800220A71AA6842F2F4
:1039A0001071D07883070BD492F803C05FEA8C764D
:1039B00006D4D378980703D4D678B30742F141826E
:1039C000D07802215FFA80FCD1701CF0100243F025
:1039D00014805FEACC7003F11F80AD680220E870AC
:1039E000FEF76FB80220D8708E68B37843F01005E8
:1039F000B5708868D32202718A6842F21070D67856
:103A0000B5070BD492F803C05FEA8C7306D4D37861
:103A10009B0703D4D578AE0742F1FB81D67802200C
:103A20005FFA86FCD0701CF0100242F0FB875FEA60
:103A3000CC7603F1068089680226CE70FDF7FBBFC5
:103A40000221D970A868837843F010068670A968AF
:103A500000220A71AA6842F21071D07883070BD451
:103A600092F803C05FEA8C7606D4D378980703D423
:103A7000D678B30742F1B581D07802215FFA80FC95
:103A8000D1701CF0100242F0E2875FEACC7002F1C4
:103A9000ED87AD680220E870FDF79BBF0220D8706B
:103AA0008E68B37843F01005B57088683F220271C4
:103AB0008A6842F21070D678B5070BD492F803C02A
:103AC0005FEA8C7306D4D3789B0703D4D578AE070E
:103AD00042F16F81D67802205FFA86FCD0701CF02C
:103AE000100242F04F865FEACC7602F15A8689686E
:103AF0000226CE70FDF727BF0221D970A86883780F
:103B000043F010068670A96800220A71AA6842F282
:103B10001071D07883070BD492F803C05FEA8C76DB
:103B200006D4D378980703D4D678B30742F1298115
:103B3000D07802215FFA80FCD1701CF0100242F0B4
:103B400036865FEACC7002F14186AD680220E870EB
:103B5000FDF7C7BE0220D8708E68B37843F0100519
:103B6000B5708868A82202718A6842F21070D6780F
:103B7000B5070BD492F803C05FEA8C7306D4D378F0
:103B80009B0703D4D578AE0742F1E380D6780220B4
:103B90005FFA86FCD0701CF0100242F0C9855FEA23
:103BA000CC7602F1D48589680226CE70FDF753BE2B
:103BB0000221D970A868837843F010068670A9683E
:103BC00000220A71AA6842F21071D07883070BD4E0
:103BD00092F803C05FEA8C7606D4D378980703D4B2
:103BE000D678B30742F19D80D07802215FFA80FC3D
:103BF000D1701CF0100242F0B0855FEACC7002F187
:103C0000BB85AD680220E870FDF7F3BD0220D870D7
:103C10008E68B37843F01005B57088688022027111
:103C20008A6842F21070D678B5070BD492F803C0B8
:103C30005FEA8C7306D4D3789B0703D4D578AE079C
:103C400042F15780D67802205FFA86FCD0701CF0D3
:103C5000100242F09B845FEACC7602F1A684896868
:103C60000226CE70FDF77FBD0221D970A868837847
:103C700043F010068670A96800220A71AA6842F211
:103C80001071D07883070BD492F803C05FEA8C766A
:103C900006D4D378980703D4D678B30742F11180BD
:103CA000D07802215FFA80FCD1701CF0100242F043
:103CB00082845FEACC7002F18D84AD680220E870E6
:103CC000FDF71FBD0220D8708E68B37843F0100551
:103CD000B5708868D52202718A6842F21070D67871
:103CE000B5070BD492F803C05FEA8C7306D4D3787F
:103CF0009B0703D4D578AE0741F1CB87D678022055
:103D00005FFA86FCD0701CF0100242F069845FEA12
:103D1000CC7602F1748489680226CE70FDF7ABBCC4
:103D20000221D970A868837843F010068670A968CC
:103D300000220A71AA6842F21071D07883070BD46E
:103D400092F803C05FEA8C7606D4D378980703D440
:103D5000D678B30741F18587D07802215FFA80FCDD
:103D6000D1701CF0100242F0CE845FEACC7002F1F8
:103D7000D984AD680220E870FDF74BBC0220D870F2
:103D80008E68B37843F01005B5708868AE22027172
:103D90008A6842F21070D678B5070BD492F803C047
:103DA0005FEA8C7306D4D3789E0703D4D578AD0729
:103DB00041F13F87D67802205FFA86FCD0701CF074
:103DC000100242F037845FEACC7602F142848968BF
:103DD0000226CE70FDF7D7BBDA7892067EF51AAFD1
:103DE000DD78AE067EF516AFDE78B5067EF512AF4D
:103DF00093F803C05FEA8C627EF50CAFDA78960622
:103E00007EF508AFDD78AD067EF504AFDE78B2064C
:103E10007EF500AF08387EF4F7AE987000BF8B686F
:103E20008020987000BF01220A73204670BDDA78A6
:103E300092067DF51FADDD78AE067DF51BADDE7813
:103E4000B5067DF517AD93F803C05FEA8C627DF58A
:103E500011ADDA7896067DF50DADDD78AD067DF510
:103E600009ADDE78B2067DF505AD08387DF4FCAC11
:103E7000987000BF8B688020987000BF2568012271
:103E80000A7395F8641000297DF4FAAC2846267967
:103E9000FDF78CFA002801F07385A86890F802E01D
:103EA0004EF030038370AA6842F21071D078830616
:103EB00001F1388592F803C05FEA8C6001F1328528
:103EC00092F803E05FEA8E6001F12C85D3789B06BF
:103ED00001F12885D078800601F1248592F803C08D
:103EE0005FEA8C6301F11E8592F803E05FEA8E6061
:103EF00001F11885D3789B0601F114850839D5D1D5
:103F0000917001F036BDDA7892067DF53BACDD7834
:103F1000AE067DF537ACDE78B5067DF533AC93F8AB
:103F200003C05FEA8C627DF52DACDA7896067DF5EC
:103F300029ACDD78AD067DF525ACDE78B2067DF5E1
:103F400021AC08387DF418AC987000BF8B688020D5
:103F5000987000BF256801220A7395F86410002943
:103F60007DF416AC28462679FDF720FA002801F0EA
:103F70003885A86890F802E04EF030038370AA6894
:103F800042F21071D078830601F1FD8492F803C0EB
:103F90005FEA8C6001F1F78492F803E05FEA8E60DB
:103FA00001F1F184D3789B0601F1ED84D07880068D
:103FB00001F1E98492F803C05FEA8C6301F1E384C4
:103FC00092F803E05FEA8E6001F1DD84D3789B060E
:103FD00001F1D9840839D5D1917001F0FBBCDA78B0
:103FE00092067DF557ABDD78AE067DF553ABDE78F6
:103FF000B5067DF54FAB93F803C05FEA8C627DF5A3
:1040000049ABDA7896067DF545ABDD78AD067DF5F2
:1040100041ABDE78B2067DF53DAB08387DF434ABBC
:10402000987000BF8B688020987000BF25680122BF
:104030000A7395F8641000297DF432AB284626797E
:10404000FDF7B4F9002801F0C085A86890F802E0F7
:104050004EF030038370AA6842F21071D078830664
:1040600001F1858592F803C05FEA8C6001F17F85DC
:1040700092F803E05FEA8E6001F17985D3789B06C0
:1040800001F17585D078800601F1718592F803C041
:104090005FEA8C6301F16B8592F803E05FEA8E6062
:1040A00001F16585D3789B0601F161850839D5D189
:1040B000917001F083BDDA7892067DF573AADD7800
:1040C000AE067DF56FAADE78B5067DF56BAA93F88E
:1040D00003C05FEA8C627DF565AADA7896067DF505
:1040E00061AADD78AD067DF55DAADE78B2067DF5C4
:1040F00059AA08387DF450AA987000BF8B688020B8
:10410000987000BF256801220A7395F86410002991
:104110007DF44EAA28462679FDF748F9002801F0DB
:104120008585A86890F802E04EF030038370AA6895
:1041300042F21071D078830601F14A8592F803C0EB
:104140005FEA8C6001F1448592F803E05FEA8E60DB
:1041500001F13E85D3789B0601F13A85D07880063F
:1041600001F1368592F803C05FEA8C6301F1308576
:1041700092F803E05FEA8E6001F12A85D3789B060E
:1041800001F126850839D5D1917001F048BDDA7862
:1041900092067DF54FADDD78AE067DF54BADDE7850
:1041A000B5067DF547AD93F803C05FEA8C627DF5F7
:1041B00041ADDA7896067DF53DADDD78AD067DF54D
:1041C00039ADDE78B2067DF535AD08387DF42CAD1D
:1041D000987000BF8B688020987000BF256801220E
:1041E0000A7395F8641000297DF42AAD28462679D3
:1041F000FDF7DCF8002801F08684A86890F802E05A
:104200004EF030038370AA6842F21071D0788306B2
:1042100001F14B8492F803C05FEA8C6001F14584A0
:1042200092F803E05FEA8E6001F13F84D3789B0649
:1042300001F13B84D078800601F1378492F803C005
:104240005FEA8C6301F1318492F803E05FEA8E60EB
:1042500001F12B84D3789B0601F127840839D5D14D
:10426000917001F049BCDA7892067DF56BACDD788F
:10427000AE067DF567ACDE78B5067DF563AC93F8E8
:1042800003C05FEA8C627DF55DACDA7896067DF559
:1042900059ACDD78AD067DF555ACDE78B2067DF51E
:1042A00051AC08387DF448AC987000BF8B68802012
:1042B000987000BF256801220A7395F864100029E0
:1042C0007DF446AC28462679FDF770F8002801F009
:1042D0004B84A86890F802E04EF030038370AA681F
:1042E00042F21071D078830601F1108492F803C075
:1042F0005FEA8C6001F10A8492F803E05FEA8E6065
:1043000001F10484D3789B0601F10084D078800603
:1043100001F1FC8392F803C05FEA8C6301F1F6833C
:1043200092F803E05FEA8E6001F1F083D3789B0698
:1043300001F1EC830839D5D1917001F00EBCDA7827
:1043400092067DF587ABDD78AE067DF583ABDE7832
:10435000B5067DF57FAB93F803C05FEA8C627DF50F
:1043600079ABDA7896067DF575ABDD78AD067DF52F
:1043700071ABDE78B2067DF56DAB08387DF464ABC9
:10438000987000BF8B688020987000BF256801225C
:104390000A7395F8641000297DF462AB28462679EB
:1043A000FDF704F8002801F0C581A86890F802E044
:1043B0004EF030038370AA6842F21071D078830601
:1043C00001F18A8192F803C05FEA8C6001F1848177
:1043D00092F803E05FEA8E6001F17E81D3789B065C
:1043E00001F17A81D078800601F1768192F803C0DC
:1043F0005FEA8C6301F1708192F803E05FEA8E60FE
:1044000001F16A81D3789B0601F166810839D5D123
:10441000917001F088B9DA7892067DF5A3AADD786B
:10442000AE067DF59FAADE78B5067DF59BAA93F8CA
:1044300003C05FEA8C627DF595AADA7896067DF571
:1044400091AADD78AD067DF58DAADE78B2067DF500
:1044500089AA08387DF480AA987000BF8B688020F4
:10446000987000BF256801220A7395F8641000292E
:104470007DF47EAA28462679FCF798FF002801F0F3
:104480008A81A86890F802E04EF030038370AA6831
:1044900042F21071D078830601F14F8192F803C087
:1044A0005FEA8C6001F1498192F803E05FEA8E6077
:1044B00001F14381D3789B0601F13F81D0788006DA
:1044C00001F13B8192F803C05FEA8C6301F1358111
:1044D00092F803E05FEA8E6001F12F81D3789B06AA
:1044E00001F12B810839D5D1917001F04DB9DA78FD
:1044F00092067DF57FADDD78AE067DF57BADDE788D
:10450000B5067DF577AD93F803C05FEA8C627DF563
:1045100071ADDA7896067DF56DADDD78AD067DF589
:1045200069ADDE78B2067DF565AD08387DF45CAD29
:10453000987000BF8B688020987000BF25680122AA
:104540000A7395F8641000297DF45AAD284626793F
:10455000FCF72CFF002801F08B80A86890F802E09F
:104560004EF030038370AA6842F21071D07883064F
:1045700001F1508092F803C05FEA8C6001F14A803B
:1045800092F803E05FEA8E6001F14480D3789B06E5
:1045900001F14080D078800601F13C8092F803C0A0
:1045A0005FEA8C6301F1368092F803E05FEA8E6087
:1045B00001F13080D3789B0601F12C800839D5D1E8
:1045C000917001F04EB8DA7892067DF59BACDD78FB
:1045D000AE067DF597ACDE78B5067DF593AC93F825
:1045E00003C05FEA8C627DF58DACDA7896067DF5C6
:1045F00089ACDD78AD067DF585ACDE78B2067DF55B
:1046000081AC08387DF478AC987000BF8B6880204E
:10461000987000BF256801220A7395F8641000297C
:104620007DF476AC28462679FCF7C0FE002801F020
:104630005080A86890F802E04EF030038370AA68BA
:1046400042F21071D078830601F1158092F803C010
:104650005FEA8C6001F10F8092F803E05FEA8E6000
:1046600001F10980D3789B0601F10580D07880069E
:1046700001F1018092F803C05FEA8C6300F1FB87CF
:1046800092F803E05FEA8E6000F1F587D3789B062D
:1046900000F1F1870839D5D1917001F013B8DA78BB
:1046A00092067DF5B7ABDD78AE067DF5B3ABDE786F
:1046B000B5067DF5AFAB93F803C05FEA8C627DF57C
:1046C000A9ABDA7896067DF5A5ABDD78AD067DF56C
:1046D000A1ABDE78B2067DF59DAB08387DF494ABD6
:1046E000987000BF8B688020987000BF25680122F9
:1046F0000A7395F8641000297DF492AB2846267958
:10470000FCF754FE002801F0D980A86890F802E078
:104710004EF030038370AA6842F21071D07883069D
:1047200001F19E8092F803C05FEA8C6001F19880ED
:1047300092F803E05FEA8E6001F19280D3789B06E5
:1047400001F18E80D078800601F18A8092F803C052
:104750005FEA8C6301F1848092F803E05FEA8E6087
:1047600001F17E80D3789B0601F17A800839D5D19A
:10477000917001F09CB8DA7892067DF5D3AADD78C5
:10478000AE067DF5CFAADE78B5067DF5CBAA93F807
:1047900003C05FEA8C627DF5C5AADA7896067DF5DE
:1047A000C1AADD78AD067DF5BDAADE78B2067DF53D
:1047B000B9AA08387DF4B0AA987000BF8B68802031
:1047C000987000BF256801220A7395F864100029CB
:1047D0007DF4AEAA28462679FCF7E8FD002801F012
:1047E0009E80A86890F802E04EF030038370AA68BB
:1047F00042F21071D078830601F1638092F803C011
:104800005FEA8C6001F15D8092F803E05FEA8E6000
:1048100001F15780D3789B0601F15380D078800650
:1048200001F14F8092F803C05FEA8C6301F1498087
:1048300092F803E05FEA8E6001F14380D3789B0633
:1048400001F13F800839D5D1917001F061B8DA7873
:1048500092067DF5AFADDD78AE067DF5ABADDE78C9
:10486000B5067DF5A7AD93F803C05FEA8C627DF5D0
:10487000A1ADDA7896067DF59DADDD78AD067DF5C6
:1048800099ADDE78B2067DF595AD08387DF48CAD36
:10489000987000BF8B688020987000BF2568012247
:1048A0000A7395F8641000297DF48AAD28462679AC
:1048B000FCF77CFD002800F09F87A86890F802E0D4
:1048C0004EF030038370AA6842F21071D0788306EC
:1048D00000F1648792F803C05FEA8C6000F15E87A4
:1048E00092F803E05FEA8E6000F15887D3789B0668
:1048F00000F15487D078800600F1508792F803C009
:104900005FEA8C6300F14A8792F803E05FEA8E6009
:1049100000F14487D3789B0600F140870839D5D150
:10492000917000F062BFDA7892067DF5CBACDD784D
:10493000AE067DF5C7ACDE78B5067DF5C3AC93F861
:1049400003C05FEA8C627DF5BDACDA7896067DF532
:10495000B9ACDD78AD067DF5B5ACDE78B2067DF597
:10496000B1AC08387DF4A8AC987000BF8B6880208B
:10497000987000BF256801220A7395F86410002919
:104980007DF4A6AC28462679FCF710FD002800F03F
:104990006487A86890F802E04EF030038370AA683C
:1049A00042F21071D078830600F1298792F803C093
:1049B0005FEA8C6000F1238792F803E05FEA8E6083
:1049C00000F11D87D3789B0600F11987D078800607
:1049D00000F1158792F803C05FEA8C6300F10F873E
:1049E00092F803E05FEA8E6000F10987D3789B06B6
:1049F00000F105870839D5D1917000F027BFDA782A
:104A000092067DF5E7ABDD78AE067DF5E3ABDE78AB
:104A1000B5067DF5DFAB93F803C05FEA8C627DF5E8
:104A2000D9ABDA7896067DF5D5ABDD78AD067DF5A8
:104A3000D1ABDE78B2067DF5CDAB08387DF4C4ABE2
:104A4000987000BF8B688020987000BF2568012295
:104A50000A7395F8641000297DF4C2AB28462679C4
:104A6000FCF7A4FC002800F0DD84A86890F802E0C0
:104A70004EF030038370AA6842F21071D07883063A
:104A800000F1A28492F803C05FEA8C6000F19C847C
:104A900092F803E05FEA8E6000F19684D3789B067B
:104AA00000F19284D078800600F18E8492F803C0E1
:104AB0005FEA8C6300F1888492F803E05FEA8E601D
:104AC00000F18284D3789B0600F17E840839D5D129
:104AD000917000F0A0BCDA7892067DF503ABDD782A
:104AE000AE067DF5FFAADE78B5067DF5FBAA93F844
:104AF00003C05FEA8C627DF5F5AADA7896067DF54B
:104B0000F1AADD78AD067DF5EDAADE78B2067DF579
:104B1000E9AA08387DF4E0AA987000BF8B6880206D
:104B2000987000BF256801220A7395F86410002967
:104B30007DF4DEAA28462679FCF738FC002800F030
:104B4000A284A86890F802E04EF030038370AA684F
:104B500042F21071D078830600F1678492F803C0A6
:104B60005FEA8C6000F1618492F803E05FEA8E6096
:104B700000F15B84D3789B0600F15784D0788006DF
:104B800000F1538492F803C05FEA8C6300F14D8416
:104B900092F803E05FEA8E6000F14784D3789B06C9
:104BA00000F143840839D5D1917000F065BCDA7802
:104BB00092067DF5DFADDD78AE067DF5DBADDE7806
:104BC000B5067DF5D7AD93F803C05FEA8C627DF53D
:104BD000D1ADDA7896067DF5CDADDD78AD067DF503
:104BE000C9ADDE78B2067DF5C5AD08387DF4BCAD43
:104BF000987000BF8B688020987000BF25680122E4
:104C00000A7395F8641000297DF4BAAD2846267918
:104C1000FCF7CCFB002800F0A383A86890F802E022
:104C20004EF030038370AA6842F21071D078830688
:104C300000F1688392F803C05FEA8C6000F1628340
:104C400092F803E05FEA8E6000F15C83D3789B0604
:104C500000F15883D078800600F1548392F803C0A5
:104C60005FEA8C6300F14E8392F803E05FEA8E60A6
:104C700000F14883D3789B0600F144830839D5D1ED
:104C8000917066E3DA7892067DF5FCACDD78AE06CD
:104C90007DF5F8ACDE78B5067DF5F4AC93F803C08D
:104CA0005FEA8C627DF5EEACDA7896067DF5EAACCB
:104CB000DD78AD067DF5E6ACDE78B2067DF5E2ACDA
:104CC00008387DF4D9AC987000BF8B68802098704C
:104CD00000BF256801220A7395F8641000297DF44D
:104CE000D7AC28462679FCF761FB002800F06983E1
:104CF000A86890F802E04EF030038370AA6842F290
:104D00001071D078830600F12E8392F803C05FEA19
:104D10008C6000F1288392F803E05FEA8E6000F176
:104D20002283D3789B0600F11E83D078800600F1A1
:104D30001A8392F803C05FEA8C6300F1148392F83F
:104D400003E05FEA8E6000F10E83D3789B0600F1EA
:104D50000A830839D5D191702CE3DA7892067DF573
:104D600019ACDD78AE067DF515ACDE78B5067DF5BF
:104D700011AC93F803C05FEA8C627DF50BACDA7876
:104D800096067DF507ACDD78AD067DF503ACDE78E3
:104D9000B2067DF5FFAB08387DF4F6AB987000BF26
:104DA0008B688020987000BF256801220A7395F8EF
:104DB000641000297DF4F4AB28462679FCF7F6FA56
:104DC000002800F0F383A86890F802E04EF030036A
:104DD0008370AA6842F21071D078830600F1B8831C
:104DE00092F803C05FEA8C6000F1B28392F803E0AE
:104DF0005FEA8E6000F1AC83D3789B0600F1A88354
:104E0000D078800600F1A48392F803C05FEA8C6337
:104E100000F19E8392F803E05FEA8E6000F19883D0
:104E2000D3789B0600F194830839D5D19170B6E30D
:104E3000DA7892067DF536ABDD78AE067DF532ABDD
:104E4000DE78B5067DF52EAB93F803C05FEA8C6281
:104E50007DF528ABDA7896067DF524ABDD78AD06D6
:104E60007DF520ABDE78B2067DF51CAB08387DF40D
:104E700013AB987000BF8B688020987000BF2568C6
:104E800001220A7395F8641000297DF411AB2846BD
:104E90002679FCF78BFA002800F0B983A86890F80F
:104EA00002E04EF030038370AA6842F21071D078AD
:104EB000830600F17E8392F803C05FEA8C6000F104
:104EC000788392F803E05FEA8E6000F17283D37812
:104ED0009B0600F16E83D078800600F16A8392F819
:104EE00003C05FEA8C6300F1648392F803E05FEA39
:104EF0008E6000F15E83D3789B0600F15A830839F7
:104F0000D5D191707CE3DA7892067DF513AEDD7829
:104F1000AE067DF50FAEDE78B5067DF50BAE93F8E7
:104F200003C05FEA8C627DF505AEDA7896067DF502
:104F300001AEDD78AD067DF5FDADDE78B2067DF51E
:104F4000F9AD08387DF4F0AD987000BF8B68802013
:104F5000987000BF256801220A7395F86410002933
:104F60007DF4EEAD28462679FCF720FA002800F003
:104F7000BB82A86890F802E04EF030038370AA6804
:104F800042F21071D078830600F1808292F803C05B
:104F90005FEA8C6000F17A8292F803E05FEA8E604B
:104FA00000F17482D3789B0600F17082D07880067D
:104FB00000F16C8292F803C05FEA8C6300F16682B4
:104FC00092F803E05FEA8E6000F16082D3789B067E
:104FD00000F15C820839D5D191707EE2DA789206D0
:104FE0007DF530ADDD78AE067DF52CADDE78B5060D
:104FF0007DF528AD93F803C05FEA8C627DF522ADA4
:10500000DA7896067DF51EADDD78AD067DF51AAD34
:10501000DE78B2067DF516AD08387DF40DAD9870DA
:1050200000BF8B688020987000BF256801220A733A
:1050300095F8641000297DF40BAD28462679FCF71D
:10504000B5F9002800F08182A86890F802E04EF0DF
:1050500030038370AA6842F21071D078830600F1A1
:10506000468292F803C05FEA8C6000F1408292F8B9
:1050700003E05FEA8E6000F13A82D3789B0600F18C
:105080003682D078800600F1328292F803C05FEA5F
:105090008C6300F12C8292F803E05FEA8E6000F1ED
:1050A0002682D3789B0600F122820839D5D19170EF
:1050B00044E2DA7892067DF54DACDD78AE067DF5FA
:1050C00049ACDE78B5067DF545AC93F803C05FEAE0
:1050D0008C627DF53FACDA7896067DF53BACDD78E9
:1050E000AD067DF537ACDE78B2067DF533AC083819
:1050F0007DF42AAC987000BF8B688020987000BF48
:10510000256801220A7395F8641000297DF428AC03
:1051100028462679FCF74AF9002800F0BF80A868E5
:1051200090F802E04EF030038370AA6842F21071EA
:10513000D078830600F1848092F803C05FEA8C6027
:105140007ED492F803E05FEA8E6079D4D3789B0630
:1051500076D4D078800673D492F803C05FEA8C636B
:105160006ED492F803E05FEA8E6069D4D3789B0630
:1051700066D40839DCD1917089E0DA7892067DF541
:1051800071ABDD78AE067DF56DABDE78B5067DF5ED
:1051900069AB93F803C05FEA8C627DF563ABDA78A4
:1051A00096067DF55FABDD78AD067DF55BABDE7811
:1051B000B2067DF557AB08387DF44EAB987000BF52
:1051C0008B688020987000BF256801220A7395F8CB
:1051D000641000297DF44CAB28462679FCF7E6F8EC
:1051E000002800F08C80A86890F802E04EF03003B0
:1051F0008370AA6842F21071D078830651D492F875
:1052000003C05FEA8C604CD492F803E05FEA8E60E2
:1052100047D4D3789B0644D4D078800641D492F802
:1052200003C05FEA8C633CD492F803E05FEA8E60CF
:1052300037D4D3789B0634D40839DDD1917057E048
:105240007600F1B21171AB6842F21072D878810722
:1052500024D4DE78B60721D493F803C05FEA8C70BB
:105260001CD493F803E05FEA8E7117D4D9788E07C7
:1052700014D4D878800711D4DE78B1070ED493F80F
:1052800003C05FEA8C7609D4083ADFD19A7000BF78
:10529000AB6880229A7000BF012129732568FDF751
:1052A0005FBB7600F1B21171AB6842F21072D87830
:1052B000810724D4DE78B60721D493F803C05FEACF
:1052C0008C701CD493F803E05FEA8E7117D4D97800
:1052D0008E0714D4D878800711D4DE78B1070ED4A5
:1052E00093F803C05FEA8C7609D4083ADFD19A704C
:1052F00000BFAB6880229A7000BF01212973256826
:10530000FDF7B6BA7600F1B21171AB6842F21072D5
:10531000D878810724D4DE78B60721D493F803C067
:105320005FEA8C701CD493F803E05FEA8E7117D4A7
:10533000D9788E0714D4D878800711D4DE78B107D5
:105340000ED493F803C05FEA8C7609D4083ADFD113
:105350009A7000BFAB6880229A7000BF0121297348
:105360002568FDF70DBA7600F1B21171AB6842F213
:105370001072D878810724D4DE78B60721D493F848
:1053800003C05FEA8C701CD493F803E05FEA8E716F
:1053900017D4D9788E0714D4D878800711D4DE7842
:1053A000B1070ED493F803C05FEA8C7609D4083AAB
:1053B000DFD19A7000BFAB6880229A7000BF0121D4
:1053C00029732568FDF764B97600F1B21171AB68F5
:1053D00042F21072D878810724D4DE78B60721D43F
:1053E00093F803C05FEA8C701CD493F803E05FEA83
:1053F0008E7117D4D9788E0714D4D878800711D439
:10540000DE78B1070ED493F803C05FEA8C7609D436
:10541000083ADFD19A7000BFAB6880229A7000BF53
:10542000012129732568FCF7DBBE7600F1B211710A
:10543000AB6842F21072D878810724D4DE78B607C0
:1054400021D493F803C05FEA8C701CD493F803E076
:105450005FEA8E7117D4D9788E0714D4D878800774
:1054600011D4DE78B1070ED493F803C05FEA8C76CE
:1054700009D4083ADFD19A7000BFAB6880229A70D5
:1054800000BF012129732568FCF732BE7600F1B216
:105490001171AB6842F21072D878810724D4DE789B
:1054A000B60721D493F803C05FEA8C701CD493F83C
:1054B00003E05FEA8E7117D4D9788E0714D4D878B8
:1054C000800711D4DE78B1070ED493F803C05FEAE9
:1054D0008C7609D4083ADFD19A7000BFAB6880227D
:1054E0009A7000BF012129732568FDF729BB76005A
:1054F000F1B21171AB6842F21072D878810724D4EE
:10550000DE78B60721D493F803C05FEA8C701CD410
:1055100093F803E05FEA8E7117D4D9788E0714D41C
:10552000D878800711D4DE78B1070ED493F803C081
:105530005FEA8C7609D4083ADFD19A7000BFAB6875
:1055400080229A7000BF012129732568FDF780BA77
:105550007600F1B21171AB6842F21072D87881070F
:1055600024D4DE78B60721D493F803C05FEA8C70A8
:105570001CD493F803E05FEA8E7117D4D9788E07B4
:1055800014D4D878800711D4DE78B1070ED493F8FC
:1055900003C05FEA8C7609D4083ADFD19A7000BF65
:1055A000AB6880229A7000BF012129732568FCF73F
:1055B000F7BF7600F1B21171AB6842F21072D87881
:1055C000810724D4DE78B60721D493F803C05FEABC
:1055D0008C701CD493F803E05FEA8E7117D4D978ED
:1055E0008E0714D4D878800711D4DE78B1070ED492
:1055F00093F803C05FEA8C7609D4083ADFD19A7039
:1056000000BFAB6880229A7000BF01212973256812
:10561000FCF74EBF7600F1B21171AB6842F2107226
:10562000D878810724D4DE78B60721D493F803C054
:105630005FEA8C701CD493F803E05FEA8E7117D494
:10564000D9788E0714D4D878800711D4DE78B107C2
:105650000ED493F803C05FEA8C7609D4083ADFD100
:105660009A7000BFAB6880229A7000BF0121297335
:105670002568FCF7C5BC7600F1B21171AB6842F247
:105680001072D878810724D4DE78B60721D493F835
:1056900003C05FEA8C701CD493F803E05FEA8E715C
:1056A00017D4D9788E0714D4D878800711D4DE782F
:1056B000B1070ED493F803C05FEA8C7609D4083A98
:1056C000DFD19A7000BFAB6880229A7000BF0121C1
:1056D00029732568FCF71CBC7600F1B21171AB6828
:1056E00042F21072D878810724D4DE78B60721D42C
:1056F00093F803C05FEA8C701CD493F803E05FEA70
:105700008E7117D4D9788E0714D4D878800711D425
:10571000DE78B1070ED493F803C05FEA8C7609D423
:10572000083ADFD19A7000BFAB6880229A7000BF40
:10573000012129732568FCF793B97600F1B2117144
:10574000AB6842F21072D878810724D4DE78B607AD
:1057500021D493F803C05FEA8C701CD493F803E063
:105760005FEA8E7117D4D9788E0714D4D878800761
:1057700011D4DE78B1070ED493F803C05FEA8C76BB
:1057800009D4083ADFD19A7000BFAB6880229A70C2
:1057900000BF012129732568FCF7EAB87600F1B251
:1057A0001171AB6842F21072D878810724D4DE7888
:1057B000B60721D493F803C05FEA8C701CD493F829
:1057C00003E05FEA8E7117D4D9788E0714D4D878A5
:1057D000800711D4DE78B1070ED493F803C05FEAD6
:1057E0008C7609D4083ADFD19A7000BFAB6880226A
:1057F0009A7000BF012129732568FCF7E1BD76008E
:10580000F1B21171AB6842F21072D878810724D4DA
:10581000DE78B60721D493F803C05FEA8C701CD4FD
:1058200093F803E05FEA8E7117D4D9788E0714D409
:10583000D878800711D4DE78B1070ED493F803C06E
:105840005FEA8C7609D4083ADFD19A7000BFAB6862
:1058500080229A7000BF012129732568FCF738BDAA
:105860007600F1B21171AB6842F21072D8788107FC
:1058700024D4DE78B60721D493F803C05FEA8C7095
:105880001CD493F803E05FEA8E7117D4D9788E07A1
:1058900014D4D878800711D4DE78B1070ED493F8E9
:1058A00003C05FEA8C7609D4083ADFD19A7000BF52
:1058B000AB6880229A7000BF012129732568FCF72C
:1058C000AFBA7600F1B21171AB6842F21072D878BB
:1058D000810724D4DE78B60721D493F803C05FEAA9
:1058E0008C701CD493F803E05FEA8E7117D4D978DA
:1058F0008E0714D4D878800711D4DE78B1070ED47F
:1059000093F803C05FEA8C7609D4083ADFD19A7025
:1059100000BFAB6880229A7000BF012129732568FF
:10592000FCF706BA7600F1B21171AB6842F2107260
:10593000D878810724D4DE78B60721D493F803C041
:105940005FEA8C701CD493F803E05FEA8E7117D481
:10595000D9788E0714D4D878800711D4DE78B107AF
:105960000ED493F803C05FEA8C7609D4083ADFD1ED
:105970009A7000BFAB6880229A7000BF0121297322
:105980002568FBF77DBF7600F1B21171AB6842F27A
:105990001072D878810724D4DE78B60721D493F822
:1059A00003C05FEA8C701CD493F803E05FEA8E7149
:1059B00017D4D9788E0714D4D878800711D4DE781C
:1059C000B1070ED493F803C05FEA8C7609D4083A85
:1059D000DFD19A7000BFAB6880229A7000BF0121AE
:1059E00029732568FBF7D4BE0846FBF7DFFC0028C7
:1059F00058D0AA68907840F030019170AB6842F2BC
:105A00001071DE78B60620D493F803C05FEA8C608C
:105A10001BD493F803E05FEA8E6616D4DA7890061A
:105A200013D4D878820610D4DE78B6060DD493F855
:105A300003C05FEA8C6008D493F803E05FEA8E62EB
:105A400003D40839DDD1997025E078211971AB684C
:105A500042F21072D878810724D4DE78B60721D4B8
:105A600093F803C05FEA8C761CD493F803E05FEAF6
:105A70008E7017D4D978890714D4D878860711D4B2
:105A8000DE78B0070ED493F803C05FEA8C7109D4B6
:105A9000083ADFD19A7000BFAB6880229A7000BFCD
:105AA000012129732168FBF7E9BC7600F1B211717D
:105AB000AB6842F21072D878810724D4DE78B6073A
:105AC00021D493F803C05FEA8C701CD493F803E0F0
:105AD0005FEA8E7117D4D9788E0714D4D8788007EE
:105AE00011D4DE78B1070ED493F803C05FEA8C7648
:105AF00009D4083ADFD19A7000BFAB6880229A704F
:105B000000BF012129732568FCF79AB87600F1B22D
:105B10001171AB6842F21072D878810724D4DE7814
:105B2000B60721D493F803C05FEA8C701CD493F8B5
:105B300003E05FEA8E7117D4D9788E0714D4D87831
:105B4000800711D4DE78B1070ED493F803C05FEA62
:105B50008C7609D4083ADFD19A7000BFAB688022F6
:105B60009A7000BF012129732568FBF7F1BF760009
:105B7000F1B21171AB6842F21072D878810724D467
:105B8000DE78B60721D493F803C05FEA8C701CD48A
:105B900093F803E05FEA8E7117D4D9788E0714D496
:105BA000D878800711D4DE78B1070ED493F803C0FB
:105BB0005FEA8C7609D4083ADFD19A7000BFAB68EF
:105BC00080229A7000BF012129732568FBF768BD08
:105BD0007600F1B21171AB6842F21072D878810789
:105BE00024D4DE78B60721D493F803C05FEA8C7022
:105BF0001CD493F803E05FEA8E7117D4D9788E072E
:105C000014D4D878800711D4DE78B1070ED493F875
:105C100003C05FEA8C7609D4083ADFD19A7000BFDE
:105C2000AB6880229A7000BF012129732568FBF7B9
:105C3000BFBCD678B3073EF5BDA892F803C05FEAB3
:105C40008C763EF5B7A8D3789D073EF5B3A8D578F6
:105C5000AB073EF5AFA808387EF49DA89070FBF71F
:105C60008BBCD07886073EF577A892F803C05FEA30
:105C70008C703EF571A8D3789B073EF56DA8D67859
:105C8000B6073EF569A808397EF457A89170FBF76E
:105C9000B9BCD678B5073EF531A892F803C05FEAE3
:105CA0008C733EF52BA8D3789E073EF527A8D578B0
:105CB000AD073EF523A808387EF411A89070FBF7D5
:105CC000D3BCD07886073DF5EBAF92F803C05FEA0E
:105CD0008C703DF5E5AFD3789B073DF5E1AFD67805
:105CE000B6073DF5DDAF08397DF4CBAF9170FBF71A
:105CF00001BDD678B5073DF5A5AF92F803C05FEAC0
:105D00008C733DF59FAFD3789E073DF59BAFD5785B
:105D1000AD073DF597AF08387DF485AF9070FBF780
:105D20001BBDD07886073DF55FAF92F803C05FEAF0
:105D30008C703DF559AFD3789B073DF555AFD678BC
:105D4000B6073DF551AF08397DF43FAF9170FBF7D1
:105D500049BDD678B5073DF519AF92F803C05FEAA3
:105D60008C733DF513AFD3789E073DF50FAFD57813
:105D7000AD073DF50BAF08387DF4F9AE9070FBF739
:105D800063BDD07886073DF5D3AE92F803C05FEAD5
:105D90008C703DF5CDAED3789B073DF5C9AED67876
:105DA000B6073DF5C5AE08397DF4B3AE9170FBF78B
:105DB00091BDD678B5073DF58DAE92F803C05FEA88
:105DC0008C733DF587AED3789E073DF583AED578CD
:105DD000AD073DF57FAE08387DF46DAE9070FBF7F2
:105DE000ABBDD07886073DF547AE92F803C05FEAB9
:105DF0008C703DF541AED3789B073DF53DAED6782E
:105E0000B6073DF539AE08397DF427AE9170FBF742
:105E1000D9BDD678B5073DF501AE92F803C05FEA6B
:105E20008C733DF5FBADD3789E073DF5F7ADD57886
:105E3000AD073DF5F3AD08387DF4E1AD9070FBF7AB
:105E4000F3BDD07886073DF5BBAD92F803C05FEA9D
:105E50008C703DF5B5ADD3789B073DF5B1ADD678E7
:105E6000B6073DF5ADAD08397DF49BAD9170FBF7FC
:105E700021BED678B5073DF575AD92F803C05FEA4F
:105E80008C733DF56FADD3789E073DF56BADD5783E
:105E9000AD073DF567AD08387DF455AD9070FBF763
:105EA0003BBED07886073DF52FAD92F803C05FEA80
:105EB0008C703DF529ADD3789B073DF525ADD6789F
:105EC000B6073DF521AD08397DF40FAD9170FBF7B4
:105ED00069BED678B5073DF5E9AC92F803C05FEA34
:105EE0008C733DF5E3ACD3789E073DF5DFACD578F8
:105EF000AD073DF5DBAC08387DF4C9AC9070FBF71D
:105F000083BED07886073DF5A3AC92F803C05FEA64
:105F10008C703DF59DACD3789B073DF599ACD67858
:105F2000B6073DF595AC08397DF483AC9170FBF76D
:105F3000B1BED678B5073DF55DAC92F803C05FEA17
:105F40008C733DF557ACD3789E073DF553ACD578AF
:105F5000AD073DF54FAC08387DF43DAC9070FBF7D4
:105F6000CBBED07886073DF517AC92F803C05FEA48
:105F70008C703DF511ACD3789B073DF50DACD67810
:105F8000B6073DF509AC08397DF4F7AB9170FBF726
:105F9000F9BED678B5073DF5D1AB92F803C05FEAFC
:105FA0008C733DF5CBABD3789E073DF5C7ABD57869
:105FB000AD073DF5C3AB08387DF4B1AB9070FBF78E
:105FC00013BFD07886073DF58BAB92F803C05FEA2C
:105FD0008C703DF585ABD3789B073DF581ABD678CA
:105FE000B6073DF57DAB08397DF46BAB9170FBF7DF
:105FF00041BFD678B5073DF545AB92F803C05FEADF
:106000008C733DF53FABD3789E073DF53BABD57820
:10601000AD073DF537AB08387DF425AB9070FBF745
:106020005BBFD07886073DF5FFAA92F803C05FEA10
:106030008C703DF5F9AAD3789B073DF5F5AAD67883
:10604000B6073DF5F1AA08397DF4DFAA9170FBF798
:1060500089BFD678B5073DF5B9AA92F803C05FEAC3
:106060008C733DF5B3AAD3789E073DF5AFAAD578DA
:10607000AD073DF5ABAA08387DF499AA9070FBF7FF
:10608000A3BFD07886073DF573AA92F803C05FEAF4
:106090008C703DF56DAAD3789B073DF569AAD6783B
:1060A000B6073DF565AA08397DF453AA9170FBF750
:1060B000D1BFD678B5073DF52DAA92F803C05FEAA7
:1060C0008C733DF527AAD3789E073DF523AAD57892
:1060D000AD073DF51FAA08387DF40DAA9070FBF7B7
:1060E000EBBFD07886073DF5E7A992F803C05FEAD9
:1060F0008C703DF5E1A9D3789B073DF5DDA9D678F5
:10610000B6073DF5D9A908397DF4C7A99170FCF708
:1061100019B8D678B5073DF5A1A992F803C05FEA92
:106120008C733DF59BA9D3789E073DF597A9D5784B
:10613000AD073DF593A908387DF481A99070FCF76F
:1061400033B8D07886073DF55BA992F803C05FEAC3
:106150008C703DF555A9D3789B073DF551A9D678AC
:10616000B6073DF54DA908397DF43BA99170FCF7C0
:1061700061B8D678B5073DF515A992F803C05FEA76
:106180008C733DF50FA9D3789E073DF50BA9D57803
:10619000AD073DF507A908387DF4F5A89070FCF728
:1061A0007BB8D07886073DF5CFA892F803C05FEAA8
:1061B0008C703DF5C9A8D3789B073DF5C5A8D67866
:1061C000B6073DF5C1A808397DF4AFA89170FCF77A
:1061D000A9B8D678B5073DF589A892F803C05FEA5B
:1061E0008C733DF583A8D3789E073DF57FA8D578BD
:1061F000AD073DF57BA808387DF469A89070FCF7E1
:10620000C3B8D07886073DF543A892F803C05FEA8B
:106210008C703DF53DA8D3789B073DF539A8D6781D
:10622000B6073DF535A808397DF423A89170FCF731
:10623000F1B8D678B5073CF5FDAF92F803C05FEA38
:106240008C733CF5F7AFD3789E073CF5F3AFD57868
:10625000AD073CF5EFAF08387CF4DDAF9070FCF78C
:106260000BB9D07886073CF5B7AF92F803C05FEA68
:106270008C703CF5B1AFD3789B073CF5ADAFD678C9
:10628000B6073CF5A9AF08397CF497AF9170FCF7DD
:1062900039B9D678B5073CF571AF92F803C05FEA1B
:1062A0008C733CF56BAFD3789E073CF567AFD57820
:1062B000AD073CF563AF08387CF451AF9070FCF744
:1062C00053B9D07886073CF52BAF92F803C05FEA4C
:1062D0008C703CF525AFD3789B073CF521AFD67881
:1062E000B6073CF51DAF08397CF40BAF9170FCF795
:1062F00081B9D678B5073CF5E5AE92F803C05FEA00
:106300008C733CF5DFAED3789E073CF5DBAED578D9
:10631000AD073CF5D7AE08387CF4C5AE9070FCF7FD
:106320009BB9D07886073CF59FAE92F803C05FEA30
:106330008C703CF599AED3789B073CF595AED6783A
:10634000B6073CF591AE08397CF47FAE9170FCF74E
:10635000C9B9D678B5073CF559AE92F803C05FEAE3
:106360008C733CF553AED3789E073CF54FAED57891
:10637000AD073CF54BAE08387CF439AE9070FCF7B5
:10638000E3B9D07886073CF514AE92F803C05FEA13
:106390008C703CF50EAED3789B073CF50AAED678F0
:1063A000B6073CF506AE08397CF4F4AD9170FCF705
:1063B00011BAD678B5073CF5CFAD92F803C05FEAC5
:1063C0008C733CF5C9ADD3789E073CF5C5ADD57847
:1063D000AD073CF5C1AD08387CF4AFAD9070FCF76B
:1063E0002BBAD07886073CF58AAD92F803C05FEAF5
:1063F0008C703CF584ADD3789B073CF580ADD678A6
:10640000B6073CF57CAD08397CF46AAD9170FCF7B9
:1064100059BAD678B5073CF545AD92F803C05FEAA6
:106420008C733CF53FADD3789E073CF53BADD578FA
:10643000AD073CF537AD08387CF425AD9070FCF71E
:1064400073BAD07886073CF500AD92F803C05FEAD6
:106450008C703CF5FAACD3789B073CF5F6ACD6785B
:10646000B6073CF5F2AC08397CF4E0AC9170FCF76F
:10647000A1BAD678B5073CF5BBAC92F803C05FEA89
:106480008C733CF5B5ACD3789E073CF5B1ACD578B0
:10649000AD073CF5ADAC08387CF49BAC9070FCF7D4
:1064A000BBBAD07886073CF576AC92F803C05FEAB9
:1064B0008C703CF570ACD3789B073CF56CACD6780F
:1064C000B6073CF568AC08397CF456AC9170FCF723
:1064D000E9BAD678B5073CF531AC92F803C05FEA6B
:1064E0008C733CF52BACD3789E073CF527ACD57864
:1064F000AD073CF523AC08387CF411AC9070FCF788
:1065000003BBD07886073CF5ECAB92F803C05FEA9A
:106510008C703CF5E6ABD3789B073CF5E2ABD678C4
:10652000B6073CF5DEAB08397CF4CCAB9170FCF7D8
:1065300031BBD678B5073CF5A7AB92F803C05FEA4C
:106540008C733CF5A1ABD3789E073CF59DABD57819
:10655000AD073CF599AB08387CF487AB9070FCF73D
:1065600043BB8B680126DE7000BF8D680873AA707C
:1065700000BF8B6880269E70FAF7D0BF8868102213
:10658000C27000BF03208D680022EFE788681022E8
:10659000C27000BF8E68032000220873B27000BF73
:1065A0008B6880259D70FDF75ABB8B680125DD70D7
:1065B00000BF8E68F1E7A9681022CA7000BFA86802
:1065C000032100222973827000BFAB6880269E7071
:1065D000FDF773BBAB680126DE7000BFA868F1E76A
:1065E00088681022C27000BF8E68032000220873E2
:1065F000B27000BF8B6880259D70FDF78CBB8B68E7
:106600000125DD7000BF8E68F1E7A9681022CA700D
:1066100000BFA868032100222973827000BFAB6805
:1066200080269E70FCF7D2BCAB680126DE7000BFEE
:10663000A868F1E788681022C27000BF8E68032046
:1066400000220873B27000BF8B6880259D70FDF733
:10665000BEBB8B680125DD7000BF8E68F1E7A968BD
:106660001022CA7000BFA86803210022297382701B
:1066700000BFAB6880269E70FCF7BBBDAB680126EF
:10668000DE7000BFA868F1E788681022C27000BF02
:106690008E68032000220873B27000BF8B688025CB
:1066A0009D70FCF7C0BC8B680125DD7000BF8E6853
:1066B000F1E7A9681022CA7000BFA8680321002270
:1066C0002973827000BFAB6880269E70FCF7D9BC2E
:1066D000AB680126DE7000BFA868F1E78868102269
:1066E000C27000BF8E68032000220873B27000BF22
:1066F0008B6880259D70FCF73CBC8B680125DD70A4
:1067000000BF8E68F1E7A9681022CA7000BFA868B0
:10671000032100222973827000BFAB6880269E701F
:10672000FDF727BBAB680126DE7000BFA868F1E764
:1067300088681022C27000BF8E6803200022087390
:10674000B27000BF8B6880259D70FDF72CBA8B68F6
:106750000125DD7000BF8E68F1E7A9681022CA70BC
:1067600000BFA868032100222973827000BFAB68B4
:1067700080269E70FDF745BAAB680126DE7000BF2B
:10678000A868F1E788681022C27000BF8E680320F5
:1067900000220873B27000BF8B6880259D70FDF7E2
:1067A000A6B98B680125DD7000BF8E68F1E7A96886
:1067B0001022CA7000BFA8680321002229738270CA
:1067C00000BFAB6880269E70FDF7BFB9AB6801269D
:1067D000DE7000BFA868F1E788681022C27000BFB1
:1067E0008E68032000220873B27000BF8B6880257A
:1067F0009D70FCF788BD8B680125DD7000BF8E6839
:10680000F1E7A9681022CA7000BFA868032100221E
:106810002973827000BFAB6880269E70FCF7A1BD13
:10682000AB680126DE7000BFA868F1E78868102217
:10683000C27000BF8E68032000220873B27000BFD0
:106840008B6880259D70FCF702BD8B680125DD708B
:1068500000BF8E68F1E7A9681022CA7000BFA8685F
:10686000032100222973827000BFAB6880269E70CE
:10687000FCF71BBDAB680126DE7000BFA868F1E71E
:1068800088681022C27000BF8E680320002208733F
:10689000B27000BF8B6880259D70FCF790BD8B683F
:1068A0000125DD7000BF8E68F1E7A9681022CA706B
:1068B00000BFA868032100222973827000BFAB6863
:1068C00080269E70FCF7A9BDAB680126DE7000BF74
:1068D000A868F1E788681022C27000BF8E680320A4
:1068E00000220873B27000BF8B6880259D70FCF792
:1068F000C2BD8B680125DD7000BF8E68F1E7A96815
:106900001022CA7000BFA868032100222973827078
:1069100000BFAB6880269E70FCF7DBBDAB6801262C
:10692000DE7000BFA868F1E788681022C27000BF5F
:106930008E68032000220873B27000BF8B68802528
:106940009D70FCF7C0BF8B680125DD7000BF8E68AD
:10695000F1E7A9681022CA7000BFA86803210022CD
:106960002973827000BFAB6880269E70FCF7D9BF88
:10697000AB680126DE7000BFA868F1E788681022C6
:10698000C27000BF8E68032000220873B27000BF7F
:106990008B6880259D70FCF73ABF8B680125DD7000
:1069A00000BF8E68F1E7A9681022CA7000BFA8680E
:1069B000032100222973827000BFAB6880269E707D
:1069C000FCF753BFAB680126DE7000BFA868F1E793
:1069D00088681022C27000BF8E68032000220873EE
:1069E000B27000BF8B6880259D70FCF7C8BF8B68B4
:1069F0000125DD7000BF8E68F1E7A9681022CA701A
:106A000000BFA868032100222973827000BFAB6811
:106A100080269E70FCF7E1BFAB680126DE7000BFE8
:106A2000A868F1E788681022C27000BF8E68032052
:106A300000220873B27000BF8B6880259D70FCF740
:106A4000FABF8B680125DD7000BF8E68F1E7A96889
:106A50001022CA7000BFA868032100222973827027
:106A600000BFAB6880269E70FDF713B8AB680126A7
:106A7000DE7000BFA868F1E788681022C27000BF0E
:106A80008E68032000220873B27000BF8B688025D7
:106A90009D70FCF704BE8B680125DD7000BF8E6819
:106AA000F1E7A9681022CA7000BFA868032100227C
:106AB0002973827000BFAB6880269E70FCF71DBEF4
:106AC000AB680126DE7000BFA868F1E78868102275
:106AD000C27000BF8E68032000220873B27000BF2E
:106AE0008B6880259D70FCF736BE8B680125DD70B4
:106AF00000BF8E68F1E7A9681022CA7000BFA868BD
:106B0000032100222973827000BFAB6880269E702B
:106B1000FCF74FBEAB680126DE7000BFA868F1E746
:106B200088681022C27000BF8E680320002208739C
:106B3000B27000BF8B6880259D70FCF754BD8B68D8
:106B40000125DD7000BF8E68F1E7A9681022CA70C8
:106B500000BFA868032100222973827000BFAB68C0
:106B600080269E70FCF76DBDAB680126DE7000BF0D
:106B7000A868F1E788681022C27000BF8E68032001
:106B800000220873B27000BF8B6880259D70FCF7EF
:106B9000CEBC8B680125DD7000BF8E68F1E7A96867
:106BA0001022CA7000BFA8680321002229738270D6
:106BB00000BFAB6880269E70FCF7E7BCAB6801267F
:106BC000DE7000BFA868F1E788681022C27000BFBD
:106BD0008E68032000220873B27000BF8B68802586
:106BE0009D70FCF7B8B88B680125DD7000BF8E681A
:106BF000F1E7A9681022CA7000BFA868032100222B
:106C00002973827000BFAB6880269E70FCF7D0B8F5
:106C1000AB680126DE7000BFA868F1E78868102223
:106C2000C27000BF8E68032000220873B27000BFDC
:106C30008B6880259D70FCF734B88B680125DD706A
:106C400000BF8E68F1E7A9681022CA7000BFA8686B
:106C5000032100222973827000BFAB6880269E70DA
:106C6000FCF74CB8AB680126DE7000BFA868F1E7FE
:106C700088681022C27000BF8E680320002208734B
:106C8000B27000BF8B6880259D70FCF7BEB88B6822
:106C90000125DD7000BF8E68F1E7A9681022CA7077
:106CA00000BFA868032100222973827000BFAB686F
:106CB00080269E70FCF7D6B8AB680126DE7000BF58
:106CC000A868F1E788681022C27000BF8E680320B0
:106CD00000220873B27000BF8B6880259D70FCF79E
:106CE000EEB88B680125DD7000BF8E68F1E7A968FA
:106CF0001022CA7000BFA868032100222973827085
:106D000000BFAB6880269E70FCF706B9AB68012611
:106D1000DE7000BFA868F1E788681022C27000BF6B
:106D20008E68032000220873B27000BF8B68802534
:106D30009D70FCF7D4B98B680125DD7000BF8E68AB
:106D4000F1E7A9681022CA7000BFA86803210022D9
:106D50002973827000BFAB6880269E70FCF7EDB986
:106D6000AB680126DE7000BFA868F1E788681022D2
:106D7000C27000BF8E68032000220873B27000BF8B
:106D80008B6880259D70FCF706BA8B680125DD7045
:106D900000BF8E68F1E700BFD0ED047A90ED056A80
:106DA00090ED037AD0ED026A30EE670A77EE660A5C
:106DB000E6EE007AF4EEE70AF1EE10FAC0ED047A9E
:106DC00020DD36EEA77A80ED037AD0ED001A90ED43
:106DD000062A90ED010A76EEA12AF0EE613A37EE2E
:106DE000623AE3EE023AF4EEC03AF1EE10FA08D558
:106DF000F4EEE31AF1EE10FA54BFB0EE610AB0EE11
:106E0000630A704737EE261AB4EEE71AF1EE10FA6D
:106E100044BF37EEE67A80ED037AD6E7F8B5837B98
:106E20000446002B00F0FF810568067B95F864009E
:106E3000002800F0A783AB6842F21071D8780206F0
:106E400023D4DF783F0620D493F803C05FEA0C60B8
:106E50001BD4DA78120618D4D878070615D4DF7850
:106E6000380612D493F803C05FEA0C620DD4DA78C6
:106E700017060AD40839E1D1997000BFA9688022A9
:106E80008A7000BF01232B7325E00221D970A86806
:106E9000837843F010078770A96800220A71AA68F6
:106EA00042F21071D078800705D492F803C05FEAEF
:106EB0008C7340F1BF81D07802215FFA80FCD170E1
:106EC0001CF0100242F090805FEACC7701F15F87FE
:106ED000AD680220E87021688B6842F21070DF789C
:106EE0003D0623D4DD782A0620D493F803C05FEA58
:106EF0000C621BD4DA78170618D4DF783D0615D457
:106F0000DD782A0612D493F803C05FEA0C670DD42B
:106F1000DA7815060AD40838E1D1987000BF88687D
:106F20008022827000BF01230B7328E00220D870FA
:106F30008F68BB7843F01005BD70886881220271AC
:106F40008A6842F21070D778BF0708D492F803C05D
:106F50005FEA8C7503D4D3789B0740F1F882D77829
:106F600002205FFA87FCD0701CF0100242F02D80E6
:106F70005FEACC7302F18E8089680227CF702168A6
:106F80008D68AF7807F0C700A8708B6842F2107068
:106F900093F803C05FEA8C6700F19581256895F846
:106FA0006410002900F0BE81AB6842F21071D878FD
:106FB000020616D4DF783F0613D493F803C05FEAC5
:106FC0000C600ED4DA7812060BD4D878070608D4F1
:106FD000DF78380605D493F803C05FEA0C6240F10D
:106FE0003A820221D970A868837843F0100787702D
:106FF000A96800220A71AA6842F21071D07880074D
:1070000008D492F803C05FEA8C7303D4D37898074E
:1070100040F18282D07802215FFA80FCD1701CF0AE
:10702000100241F0F8875FEACC7702F12D80AD685D
:107030000220E87021688B6842F21070DF783D060C
:1070400016D4DD782A0613D493F803C05FEA0C62E5
:107050000ED4DA7817060BD4DF783D0608D4DD7835
:107060002A0605D493F803C05FEA0C6740F1E38178
:107070000220D8708F68BB7843F01005BD708A6815
:1070800016718A6842F21070D778BF0708D492F858
:1070900003C05FEA8C7503D4D3789B0740F121824B
:1070A000D77802205FFA87FCD0701CF0100241F004
:1070B000C1875FEACC7301F1DB8789680227CF7053
:1070C00021688D68AF7807F0C700A8708B6842F21E
:1070D000107093F803C05FEA8C6700F1CA802568DE
:1070E000617B95F8647000290CBFA626A726002FA7
:1070F00001F0E385AB6842F21071D878020616D42D
:10710000DF783F0613D493F803C05FEA0C600ED417
:10711000DA7812060BD4D878070608D4DF78380658
:1071200005D493F803C05FEA0C6240F17481022138
:10713000D970A868837843F010078770A968002287
:107140000A71AA6842F21071D078800708D492F8C8
:1071500003C05FEA8C7303D4D378980740F1A6810B
:10716000D07802215FFA80FCD1701CF0100241F04F
:1071700043875FEACC7701F19387AD680220E8701E
:1071800021688B6842F21070DF783D0616D4DD78F6
:107190002A0613D493F803C05FEA0C620ED4DA789F
:1071A00017060BD4DF783D0608D4DD782A0605D40F
:1071B00093F803C05FEA0C6740F11D810220D8708C
:1071C0008F68BB7843F01005BD708A6816718A68B5
:1071D00042F21070D678B30708D4D778BF0705D429
:1071E00092F803C05FEA8C7640F14581D3780220A3
:1071F000DDB2D07015F0100241F02B87EE0701F1DF
:107200003D8789680227CF7021688E68B27802F0C6
:10721000C707B7708B6842F21070DD78AD0600F1D9
:10722000BE800021A173256895F86470002F00F0DE
:107230000C82F8BDD37898073FF53DAED778BB07F1
:107240003FF539AED07887073FF535AE92F803C0E9
:107250005FEA8C703FF52FAED3789B073FF52BAEDE
:10726000D778BF073FF527AE08397FF41BAE917082
:1072700003E6DA7895067FF532AFDD78AF067FF565
:107280002EAFDF78BD067FF52AAF93F803C05FEA23
:107290008C627FF524AFDA7897067FF520AFDD7832
:1072A000AD067FF51CAFDF78BA067FF518AF08385A
:1072B0007FF40FAF987000BF8B688020987000BF7C
:1072C00001220A730BE7DA7895067FF567AEDD7861
:1072D000AF067FF563AEDF78BD067FF55FAE93F84E
:1072E00003C05FEA8C627FF559AEDA7897067FF5C6
:1072F00055AEDD78AD067FF551AEDF78BA067FF585
:107300004DAE08387FF444AE987000BF8B68802083
:10731000987000BF256801220A7395F8641000294F
:107320007FF442AE28462779FAF740F8002801F0AA
:10733000C184A86890F802E04EF030038370AA6818
:1073400042F21071D078800601F1868492F803C071
:107350005FEA8C6301F1808492F803E05FEA8E605B
:1073600001F17A84D3789B0601F17684D078800687
:1073700001F1728492F803C05FEA8C6301F16C84BE
:1073800092F803E05FEA8E6001F16684D3789B0691
:1073900001F162840839D5D1917001F084BCDE78A6
:1073A000B2067FF53EAF93F803C05FEA8C627FF5CB
:1073B00038AFDA7897067FF534AFDF78BE067FF511
:1073C00030AFDD78AD067FF52CAFDE78B2067FF505
:1073D00028AF93F803C05FEA8C677FF522AF0838C7
:1073E0007FF41BAF987000BF8B688020987000BF3F
:1073F00001220A7315E7DA7815063FF5DFAE083883
:107400007FF4C2AE987000BF8B688020987000BF78
:1074100001250D73F8E6DA7817063FF588AE0839CE
:107420007FF46BAE997000BFA96880228A7000BF9C
:1074300001232B73A4E6DA7815063FF519AE083858
:107440007FF4FCAD987000BF88688022827000BF16
:1074500001230B7334E6DA7817063FF5C2AD08391D
:107460007FF4A5AD997000BFA96880228A7000BF23
:1074700001232B73DEE5D3789D073FF5B7AED578B2
:10748000AB073FF5B3AED678B7073FF5AFAED778C9
:10749000BE073FF5ABAE92F803C05FEA8C753FF5CF
:1074A000A5AE08387FF496AE9070ACE7D778BB07EE
:1074B0003FF556AED07887073FF552AE92F803C03D
:1074C0005FEA8C703FF54CAED3789B073FF548AE32
:1074D000D778BF073FF544AE08397FF435AE9170D9
:1074E000A1E7D578AF073FF5DBADD778BD073FF50E
:1074F000D7AD92F803C05FEA8C733FF5D1ADD37876
:107500009F073FF5CDADD578AD073FF5C9AD08383C
:107510007FF4BAAD907096E7D778BB073FF57AADA8
:10752000D07887073FF576AD92F803C05FEA8C709C
:107530003FF570ADD3789B073FF56CADD778BF07AB
:107540003FF568AD08397FF459AD91708BE7D57878
:10755000AF073FF504ADD778BD073FF500AD92F812
:1075600003C05FEA8C733FF5FAACD3789F073FF511
:10757000F6ACD578AD073FF5F2AC08387FF4E3AC54
:107580009070CBE428462779F9F710FF002859D0EE
:10759000AA68917841F030039370AA6842F21071A2
:1075A000D078800620D492F803C05FEA8C631BD4A5
:1075B00092F803E05FEA8E6016D4D3789B0613D46A
:1075C000D078800610D492F803C05FEA8C630BD4A5
:1075D00092F803E05FEA8E6006D4D3789B0603D46A
:1075E0000839DDD1917026E07F00F9B21171AB68E6
:1075F00042F21072D878800724D4DF78B90721D4FA
:1076000093F803C05FEA8C701CD493F803E05FEA40
:107610008E7117D4D9788F0714D4D878800711D4F5
:10762000DF78B9070ED493F803C05FEA8C7709D4EA
:10763000083ADFD19A7000BFAB6880229A7000BF11
:10764000012129732568FFF7F6BB28462679F9F74B
:10765000ADFE002838D0A86890F802E04EF0300364
:107660008370AA6842F21071D778BB0600F16F836D
:10767000D078870600F16B8392F803C05FEA8C63D1
:1076800000F1658392F803E05FEA8E6700F15F83A3
:10769000D378980600F15B83D778BB0600F1578357
:1076A000D078870600F1538392F803C05FEA8C60BC
:1076B00000F14D830839D7D1917000BFAB688022AB
:1076C0009A7000BF01262E7321688B6842F21070F9
:1076D000DD782A0600F16983DF783F0600F16583D3
:1076E00093F803E05FEA0E6600F15F8393F803C04E
:1076F0005FEA0C6500F15983DA78120600F15583D0
:10770000DE78370600F15183DD782E0600F14D83D7
:10771000DF783D0600F149830838D9D1987000BF61
:107720008B688020987000BF01260E7321688B68DB
:1077300042F21070DF783F0600F13F8693F803E0D5
:107740005FEA0E6600F1398693F803C05FEA0C65C4
:1077500000F13386DA78120600F12F86DD782F06E5
:1077600000F12B86DE78360600F12786DF783D06AD
:1077700000F1238693F803E05FEA0E6200F11D86B4
:107780000838D7D1987000BF8B688020987000BFF0
:1077900001250D7321688E68B27802F0C707B770B3
:1077A0008B6842F21070DD78AE0600F148862568DD
:1077B00095F86410002900F07386AB6842F21071EE
:1077C000D878000600F1B785DF783A0600F1B38576
:1077D00093F803C05FEA0C6000F1AD8593F803E015
:1077E0005FEA0E6200F1A785DA78170600F1A3853B
:1077F000DE78360600F19F85D878000600F19B857B
:10780000DF783A0600F197850839D9D1997000BF21
:10781000AB688021997000BF01262E7321688B68A8
:1078200042F21070DF783D0600F1438593F803C003
:107830005FEA0C6200F13D8593F803E05FEA0E65B4
:1078400000F13785DA78120600F13385DD782F06EE
:1078500000F12F85DE78360600F12B85DF783D06B6
:1078600000F1278593F803C05FEA0C6200F12185DF
:107870000838D7D1987000BF8B688020987000BFFF
:1078800001250D7321688E68B27802F0C707B770C2
:107890008B6842F21070DD78AD0600F1298725680B
:1078A00095F86410002900F05487AB6842F210711B
:1078B000D878020600F1BB84DF783F0600F1B78478
:1078C00093F803E05FEA0E6000F1B18493F803C01F
:1078D0005FEA0C6200F1AB84DA78170600F1A78446
:1078E000DE78360600F1A384D878000600F19F8484
:1078F000DF783A0600F19B840839D9D1997000BF2E
:10790000AB688021997000BF01262E7321688B68B7
:1079100042F21070DF783F0600F1478493F803E0ED
:107920005FEA0E6600F1418493F803C05FEA0C65DC
:1079300000F13B84DA78120600F13784DD782F06F7
:1079400000F13384DE78360600F12F84DF783D06BF
:1079500000F12B8493F803E05FEA0E6200F12584C6
:107960000838D7D1987000BF8B688020987000BF0E
:1079700001250D7321688E68B27802F0C707B770D1
:107980008B6842F21070DD78AE0600F1248725681E
:1079900095F86410002900F04F87AB6842F210712F
:1079A000D878000600F1C183DF783A0600F1BD8384
:1079B00093F803C05FEA0C6000F1B78393F803E02B
:1079C0005FEA0E6200F1B183DA78170600F1AD8349
:1079D000DE78360600F1A983D878000600F1A58389
:1079E000DF783A0600F1A1830839D9D1997000BF38
:1079F000AB688021997000BF01262E7321688B68C7
:107A000042F21070DF783D0600F14F8393F803C017
:107A10005FEA0C6200F1498393F803E05FEA0E65C8
:107A200000F14383DA78120600F13F83DD782F06F8
:107A300000F13B83DE78360600F13783DF783D06C0
:107A400000F1338393F803C05FEA0C6200F12D83E9
:107A50000838D7D1987000BF8B688020987000BF1D
:107A600001250D7321688E68B27802F0C707B770E0
:107A70008B6842F21070DD78AD0600F15385256801
:107A800095F86410002900F07E85AB6842F2107111
:107A9000D878020600F1C982DF783F0600F1C5827E
:107AA00093F803E05FEA0E6000F1BF8293F803C031
:107AB0005FEA0C6200F1B982DA78170600F1B5824C
:107AC000DE78360600F1B182D878000600F1AD828A
:107AD000DF783A0600F1A9820839D9D1997000BF40
:107AE000AB688021997000BF01262E7321688B68D6
:107AF00042F21070DF783F0600F1578293F803E0FE
:107B00005FEA0E6600F1518293F803C05FEA0C65EC
:107B100000F14B82DA78120600F14782DD782F06F9
:107B200000F14382DE78360600F13F82DF783D06C1
:107B300000F13B8293F803E05FEA0E6200F13582C8
:107B40000838D7D1987000BF8B688020987000BF2C
:107B500001250D7321688E68B27802F0C707B770EF
:107B60008B6842F21070DD78AE0600F14E85256814
:107B700095F86410002900F07985AB6842F2107125
:107B8000D878000600F1D181DF783A0600F1CD8186
:107B900093F803C05FEA0C6000F1C78193F803E03B
:107BA0005FEA0E6200F1C181DA78170600F1BD814B
:107BB000DE78360600F1B981D878000600F1B5818B
:107BC000DF783A0600F1B1810839D9D1997000BF48
:107BD000AB688021997000BF01262E7321688B68E5
:107BE00042F21070DF783D0600F15F8193F803C028
:107BF0005FEA0C6200F1598193F803E05FEA0E65D9
:107C000000F15381DA78120600F14F81DD782F06FA
:107C100000F14B81DE78360600F14781DF783D06C2
:107C200000F1438193F803C05FEA0C6200F13D81EB
:107C30000838D7D1987000BF8B688020987000BF3B
:107C400001250D7321688E68B27802F0C707B770FE
:107C50008B6842F21070DD78AD0600F12F86256842
:107C600095F86410002900F05A86AB6842F2107152
:107C7000D878020600F1D980DF783F0600F1D58080
:107C800093F803E05FEA0E6000F1CF8093F803C041
:107C90005FEA0C6200F1C980DA78170600F1C5804E
:107CA000DE78360600F1C180D878000600F1BD808C
:107CB000DF783A0600F1B9800839D9D1997000BF50
:107CC000AB688021997000BF01262E73236893F85A
:107CD0006470002F7FF4ADAAA5689A68DD664FF442
:107CE00080641C6742F2107092F803E05FEA0E674E
:107CF00000F1568692F803C05FEA0C6600F15086E8
:107D0000D1780C0600F14C86D678310600F1488611
:107D1000D7783F0600F14486D478260600F14086E5
:107D200092F803E05FEA0E6400F13A8692F803C02D
:107D30005FEA0C6100F134860838D5D1907000BF3D
:107D400098688021817000BF01241C73F8BD760003
:107D5000F1B21171AB6842F21072DF78B8073FF5EB
:107D6000B3ACD87881073FF5AFACDE78B0073FF50C
:107D7000ABAC93F803E05FEA8E713FF5A5AC93F8E6
:107D800003C05FEA8C773FF59FACD9788E073FF54B
:107D90009BACDF78B8073FF597ACD87881073FF503
:107DA00093AC083AD9D19A7087E40220D8708A68D7
:107DB000937843F0100696708D6800272F718A68BB
:107DC00042F2107092F803E05FEA8E761ED492F8C9
:107DD00003C05FEA8C7519D4D3789B0716D4D67884
:107DE000B70713D4D578AE0710D4D778BD070DD414
:107DF00092F803E05FEA8E7308D492F803C05FEA5A
:107E00008C7703D40838DDD1907088E4D3780220D1
:107E1000DEB2D07016F0100240F0E287F30700F1F6
:107E2000D28789680225CD7080E40221D970AA68C2
:107E3000937843F010069670A86840270771AA68E7
:107E400042F2107192F803E05FEA8E761ED492F847
:107E500003C05FEA8C7019D4D3789F0716D4D67804
:107E6000B60713D4D078800710D4D778BB070DD4C9
:107E700092F803E05FEA8E7708D492F803C05FEAD5
:107E80008C7603D40839DDD1917018E7D3780221BC
:107E9000DEB2D17016F0100241F05980F30701F103
:107EA0001F80AD680220E87010E70220D8708A6851
:107EB000937843F0100595708E68072737718A68AC
:107EC00042F2107092F803E05FEA8E731ED492F8CB
:107ED00003C05FEA8C7719D4D3789F0716D4D5787E
:107EE000AE0713D4D678B50710D4D778BB070DD416
:107EF00092F803E05FEA8E7708D492F803C05FEA55
:107F00008C7603D40838DDD1907094E6D3780220C3
:107F1000DDB2D07015F0100240F0D287EE0700F10C
:107F2000C28789680227CF708CE60221D970AA68BF
:107F3000937843F010069670A86800270771AA6826
:107F400042F2107192F803C05FEA8C731ED492F86B
:107F500003E05FEA8E7719D4D3789F0716D4D678DA
:107F6000B60713D4D078800710D4D778BB070DD4C8
:107F700092F803C05FEA8C7708D492F803E05FEAD6
:107F80008E7603D40839DDD1917020E6D3780221B2
:107F9000DEB2D17016F0100240F09A87F60700F1B9
:107FA0003687AD680220E87018E60220D8708A682B
:107FB000937843F0100595708E68002737718A68B2
:107FC00042F2107092F803C05FEA8C751ED492F8EA
:107FD00003E05FEA8E7319D4D3789F0716D4D5785F
:107FE000AE0713D4D678B50710D4D778BB070DD415
:107FF00092F803C05FEA8C7708D492F803E05FEA56
:108000008E7603D40838DDD190709CE5D3780220B9
:10801000DDB2D07015F0100240F01387EF0700F1C9
:10802000038789680227CF7094E50221D970AA6876
:10803000937843F010069670A86800270771AA6825
:1080400042F2107192F803E05FEA8E761ED492F845
:1080500003C05FEA8C7019D4D3789F0716D4D67802
:10806000B60713D4D078800710D4D778BB070DD4C7
:1080700092F803E05FEA8E7708D492F803C05FEAD3
:108080008C7603D40839DDD1917028E5D3780221AC
:10809000DEB2D17016F0100240F0AA86F30700F1AC
:1080A000FC86AD680220E87020E50220D8708A685E
:1080B000937843F0100595708E68222737718A688F
:1080C00042F2107092F803E05FEA8E731ED492F8C9
:1080D00003C05FEA8C7719D4D3789F0716D4D5787C
:1080E000AE0713D4D678B50710D4D778BB070DD414
:1080F00092F803E05FEA8E7708D492F803C05FEA53
:108100008C7603D40838DDD19070A4E4D3780220B3
:10811000DDB2D07015F0100240F0A886EE0700F135
:10812000988689680227CF709CE40221D970AA68DA
:10813000937843F010069670A86800270771AA6824
:1081400042F2107192F803C05FEA8C731ED492F869
:1081500003E05FEA8E7719D4D3789F0716D4D678D8
:10816000B60713D4D078800710D4D778BB070DD4C6
:1081700092F803C05FEA8C7708D492F803E05FEAD4
:108180008E7603D40839DDD1917030E4D3780221A2
:10819000DEB2D17016F0100240F07086F60700F1E2
:1081A000DE86AD680220E87028E40220D8708A6874
:1081B000937843F0100595708E687F2737718A6831
:1081C00042F2107092F803C05FEA8C751FD492F8E7
:1081D00003E05FEA8E731AD4D3789F0717D4D5785B
:1081E000AE0714D4D678B50711D4D778BB070ED410
:1081F00092F803C05FEA8C7709D492F803E05FEA53
:108200008E7604D40838DDD19070FFF7ACBBD378FC
:108210000220DDB2D07015F0100240F0B386EF07F7
:1082200000F1A38689680227CF70FFF7A3BB022164
:10823000D970AA68937843F010069670A868002752
:108240000771AA6842F2107192F803E05FEA8E7635
:108250001FD492F803C05FEA8C701AD4D3789F07BA
:1082600017D4D678B60714D4D078800711D4D7782D
:10827000BB070ED492F803E05FEA8E7709D492F838
:1082800003C05FEA8C7604D40839DDD19170FFF722
:1082900036BBD3780221DEB2D17016F0100240F066
:1082A0008385F30700F14D86AD680220E870FFF783
:1082B0002DBB0220D8708A68937843F01005957022
:1082C0008E68002737718A6842F2107092F803E0D6
:1082D0005FEA8E731FD492F803C05FEA8C771AD4DA
:1082E000D3789F0717D4D578AE0714D4D678B507BE
:1082F00011D4D778BB070ED492F803E05FEA8E77EB
:1083000009D492F803C05FEA8C7604D40838DDD132
:108310009070FFF7B0BAD3780220DDB2D07015F0BC
:10832000100240F0F785EE0700F1E7858968022723
:10833000CF70FFF7A7BA0221D970AA68937843F0EB
:1083400010069670A86800270771AA6842F210719B
:1083500092F803C05FEA8C731FD492F803E05FEADF
:108360008E771AD4D3789F0717D4D678B60714D44B
:10837000D078800711D4D778BB070ED492F803C009
:108380005FEA8C7709D492F803E05FEA8E7604D432
:108390000839DDD19170FFF73ABAD3780221DEB205
:1083A000D17016F0100240F0BD85F60700F1F2859D
:1083B000AD680220E870FFF731BA0220D8708A68F1
:1083C000937843F0100595708E68212737718A687D
:1083D00042F2107092F803C05FEA8C751FD492F8D5
:1083E00003E05FEA8E731AD4D3789F0717D4D57849
:1083F000AE0714D4D678B50711D4D778BB070ED4FE
:1084000092F803C05FEA8C7709D492F803E05FEA40
:108410008E7604D40838DDD19070FFF7B4B9D378E4
:108420000220DDB2D07015F0100240F0C685EF07D3
:1084300000F1B68589680227CF70FFF7ABB9DE7807
:10844000B5067FF5B4A993F803C05FEA8C657FF5A4
:10845000AEA993F803E05FEA8E627FF5A8A9DA7807
:1084600097067FF5A4A9DF78BE067FF5A0A9DD7881
:10847000AD067FF59CA9DE78B2067FF598A908388D
:108480007FF491A9987000BF8B688020987000BF1E
:10849000256801220A7395F8641000297FF48DA9DC
:1084A00028462679F8F782FF002838D0AF6897F879
:1084B00002C04CF03003BB70AA6842F21071D07851
:1084C000800600F10C83D778BB0600F1088392F890
:1084D00003E05FEA8E6000F1028392F803C05FEA76
:1084E0008C6300F1FC82D3789F0600F1F882D0788B
:1084F000800600F1F482D778BB0600F1F08292F892
:1085000003E05FEA8E6700F1EA820839D7D1917003
:1085100000BFAB6880229A7000BF01262E732568C9
:10852000FFF74BB9DE78B2067FF5A9AA93F803E00E
:108530005FEA8E657FF5A3AA93F803C05FEA8C62B9
:108540007FF59DAADA7897067FF599AADF78BE06AF
:108550007FF595AADD78AD067FF591AADE78B206A3
:108560007FF58DAA08387FF486AA987000BF8B68C3
:108570008020987000BF256801220A7395F8641066
:1085800000297FF482AA28462679F8F70FFF0028F1
:1085900038D0AF6897F802E04EF03003BB70AA689D
:1085A00042F21071D078830600F1C782D778BF06F7
:1085B00000F1C38292F803C05FEA8C6000F1BD82D3
:1085C00092F803E05FEA8E6300F1B782D3789F06EA
:1085D00000F1B382D078800600F1AF82D778BB0675
:1085E00000F1AB8292F803C05FEA8C6700F1A582CC
:1085F0000839D7D1917000BFAB6880229A7000BF54
:1086000001262E732568FFF740BADE78B5067FF5A0
:10861000AEAA93F803C05FEA8C657FF5A8AA93F829
:1086200003E05FEA8E627FF5A2AADA7897067FF50B
:108630009EAADF78BE067FF59AAADD78AD067FF5A3
:1086400096AADE78B2067FF592AA08387FF48BAA44
:10865000987000BF8B688020987000BF2568012249
:108660000A7395F8641000297FF487AA28462679B2
:10867000F8F79CFE002838D0AF6897F802C04CF09D
:108680003003BB70AA6842F21071D078800600F106
:108690008282D778BB0600F17E8292F803E05FEA1F
:1086A0008E6000F1788292F803C05FEA8C6300F17B
:1086B0007282D3789F0600F16E82D078800600F136
:1086C0006A82D778BB0600F1668292F803E05FEA1F
:1086D0008E6700F160820839D7D1917000BFAB6816
:1086E00080229A7000BF01262E732568FFF745BAD5
:1086F000DE78B2067FF5D3A893F803E05FEA8E65D3
:108700007FF5CDA893F803C05FEA8C627FF5C7A818
:10871000DA7897067FF5C3A8DF78BE067FF5BFA895
:10872000DD78AD067FF5BBA8DE78B2067FF5B7A889
:1087300008387FF4B0A8987000BF8B6880209870CC
:1087400000BF256801220A7395F8641000297FF4A0
:10875000ACA828462679F8F729FE002838D0AF685B
:1087600097F802E04EF03003BB70AA6842F2107135
:10877000D078830600F13D82D778BF0600F13982B8
:1087800092F803C05FEA8C6000F1338292F803E054
:108790005FEA8E6300F12D82D3789F0600F1298273
:1087A000D078800600F12582D778BB0600F12182BF
:1087B00092F803C05FEA8C6700F11B820839D7D1B9
:1087C000917000BFAB6880229A7000BF01262E73A3
:1087D0002568FFF76AB8DE78B5067FF5D8A893F864
:1087E00003C05FEA8C657FF5D2A893F803E05FEAE7
:1087F0008E627FF5CCA8DA7897067FF5C8A8DF7877
:10880000BE067FF5C4A8DD78AD067FF5C0A8DE788A
:10881000B2067FF5BCA808387FF4B5A8987000BFF1
:108820008B688020987000BF256801220A7395F834
:10883000641000297FF4B1A828462679F8F7B6FD20
:10884000002838D0AF6897F802C04CF03003BB70F6
:10885000AA6842F21071D078800600F1E580D778DE
:10886000BB0600F1E18092F803E05FEA8E6000F160
:10887000DB8092F803C05FEA8C6300F1D580D37887
:108880009F0600F1D180D078800600F1CD80D778A6
:10889000BB0600F1C98092F803E05FEA8E6700F141
:1088A000C3800839D7D1917000BFAB6880229A701D
:1088B00000BF01262E732568FFF76FB8DE78B20679
:1088C0007FF5CDA993F803E05FEA8E657FF5C7A930
:1088D00093F803C05FEA8C627FF5C1A9DA78970646
:1088E0007FF5BDA9DF78BE067FF5B9A9DD78AD06B5
:1088F0007FF5B5A9DE78B2067FF5B1A908387FF417
:10890000AAA9987000BF8B688020987000BF256866
:1089100001220A7395F8641000297FF4A6A928465D
:108920002679F8F743FD002837D0AF6897F802E0C2
:108930004EF03003BB70AA6842F21071D078830603
:1089400000F1A080D778BF0600F19C8092F803C0A8
:108950005FEA8C6000F1968092F803E05FEA8E6334
:1089600000F19080D3789F0600F18C80D07880064B
:1089700000F18880D778BB0600F1848092F803C0AC
:108980005FEA8C677ED40839D8D1917000BFAB689C
:1089900080229A7000BF01262E732568FFF765B903
:1089A0009079AB4E40F0500191719A681227D770C0
:1089B0009C68A07840F01001A1701A6E1168002028
:1089C000C871D2F800E001276C1C0C608F80CEF8D3
:1089D0000870146840F2FF3CA4F81EC01268E660FC
:1089E000A2F816C01E6E9F6831680437B7F1804F39
:1089F0000F618882887180F0C4813268012494609C
:108A000032681E6E934F00219161307938709C68F6
:108A100094F802C04CF00102A2709E682D78357166
:108A2000012783F86470F8BD7600F1B21171AB686C
:108A300042F21072D87887073FF53DAFDF78BE0766
:108A40003FF539AFDE78B7073FF535AF93F803C090
:108A50005FEA8C763FF52FAF93F803E05FEA8E7004
:108A60003FF529AFD97889073FF525AFD878870733
:108A70003FF521AFDF78BE073FF51DAF083AD9D1EA
:108A80009A7011E77600F1B21171AB6842F2107280
:108A9000D878800781D4DF78B9073FF57EAFDE78DC
:108AA000B7073FF57AAF93F803E05FEA8E763FF5BC
:108AB00074AF93F803C05FEA8C703FF56EAFD9785E
:108AC00089073FF56AAFD87887073FF566AFDF784B
:108AD000BE073FF562AF083ADAD19A7056E77600E2
:108AE000F1B21171AB6842F21072D87887073FF586
:108AF00016ADDF78BE073FF512ADDE78B7073FF55C
:108B00000EAD93F803C05FEA8C763FF508AD93F89D
:108B100003E05FEA8E703FF502ADD97889073FF533
:108B2000FEACD87887073FF5FAACDF78BE073FF593
:108B3000F6AC083AD9D19A70EAE47600F1B2117134
:108B4000AB6842F21072D87880073FF55BADDF78F2
:108B5000B9073FF557ADDE78B7073FF553AD93F84A
:108B600003E05FEA8E763FF54DAD93F803C05FEA10
:108B70008C703FF547ADD97889073FF543ADD8787C
:108B800087073FF53FADDF78BE073FF53BAD083ABD
:108B9000D9D19A702FE57600F1B21171AB6842F22B
:108BA0001072D87887073FF5A0ADDF78BE073FF594
:108BB0009CADDE78B7073FF598AD93F803C05FEA48
:108BC0008C763FF592AD93F803E05FEA8E703FF547
:108BD0008CADD97889073FF588ADD87887073FF500
:108BE00084ADDF78BE073FF580AD083AD9D19A70E1
:108BF00074E57600F1B21171AB6842F21072D87868
:108C000080073FF5E5ADDF78B9073FF5E1ADDE78E8
:108C1000B7073FF5DDAD93F803E05FEA8E763FF5E9
:108C2000D7AD93F803C05FEA8C703FF5D1ADD9782A
:108C300089073FF5CDADD87887073FF5C9ADDF7817
:108C4000BE073FF5C5AD083AD9D19A70B9E500BF66
:108C500001FCFFFF1B8000407F00F9B21171AB687F
:108C600042F21072D878800724D4DF78B90721D473
:108C700093F803C05FEA8C701CD493F803E05FEABA
:108C80008E7117D4D9788F0714D4D878800711D46F
:108C9000DF78B9070ED493F803C05FEA8C7709D464
:108CA000083ADFD19A7000BFAB6880229A7000BF8B
:108CB000012129732568FEF777B928462779F8F747
:108CC00075FB00285AD0A86890F802E04EF03003F7
:108CD0008370AA6842F21071D078800620D492F88E
:108CE00003C05FEA8C631BD492F803E05FEA8E60F6
:108CF00016D4D3789B0613D4D078800610D492F87B
:108D000003C05FEA8C630BD492F803E05FEA8E60E5
:108D100006D4D3789B0603D40839DDD1917026E0C0
:108D20007F00F9B21171AB6842F21072D8788007F7
:108D300024D4DF78B90721D493F803C05FEA8C709C
:108D40001CD493F803E05FEA8E7117D4D9788F07AB
:108D500014D4D878800711D4DF78B9070ED493F8EB
:108D600003C05FEA8C7709D4083ADFD19A7000BF5C
:108D7000AB6880229A7000BF012129732568FEF735
:108D8000B9B93268906800287FF43BAE36E6AB682C
:108D90000127DF7000BFA8682973827000BFAB682D
:108DA00080279F70FEF794B8A9681026CE7000BF88
:108DB000AB680321002229739A7000BFAF6880223C
:108DC000BA70FFF771BA8F680125FD7000BF8B681C
:108DD00008739A7000BF8F688022BA70FFF721B8BD
:108DE00088681026C67000BF03208B680022EFE75A
:108DF000A9681026CE7000BFAB680321002229733A
:108E00009A7000BFAF688022BA70FFF74AB9AF68A6
:108E10000120F87000BFAB6829739A7000BFAF687B
:108E20008022BA70FFF7BDB88E680127F77000BFC7
:108E30008B6808739A7000BF8E688022B270FFF74B
:108E4000F0B888681025C57000BF03208B68002229
:108E5000EFE78E680127F77000BF8B6808739A7080
:108E600000BF8E688022B270FFF75BB9886810255A
:108E7000C57000BF03208B680022EFE7A9681026A9
:108E8000CE7000BFAB680321002229739A7000BF27
:108E9000AF688022BA70FFF784B9AF680120F8701C
:108EA00000BFAB68ABE78E680127F77000BF8B6827
:108EB00008739A7000BF8E688022B270FFF731B8D5
:108EC00088681025C57000BF03208B680022EFE77B
:108ED000A9681026CE7000BF0321AB6800229BE773
:108EE000AF680120F87000BFAB6829739A7000BFAB
:108EF000AF688022BA70FEF7D4BF8E680127F77082
:108F000000BF8B6808739A7000BF8E688022B270B1
:108F1000FFF70CBA88681025C57000BF03208B6866
:108F20000022EFE7A9681026CE7000BFAB680321CE
:108F3000002229739A7000BFAF688022BA70FFF7D1
:108F400037BAAF680120F87000BFAB6833E7A96893
:108F50001026CE7000BF0321AB680022C5E7AF68C2
:108F60000120F87000BFAB688FE78E680127F770AB
:108F700000BF8B6808739A7000BF8E688022B27041
:108F8000FFF750B988681025C57000BF03208B68B3
:108F90000022EFE7AF680120F87000BFAB68C8E7B8
:108FA0008E680127F77000BF8B6808739A7000BF46
:108FB0008E688022B270FFF73DBA88681025C570B0
:108FC00000BF03208B680022EFE788681022C27080
:108FD00000BF8F68032000220873BA7000BF8B683F
:108FE00080259D70FDF7C8BFA9681022CA7000BF18
:108FF0000321A8680022CFE6A9681022CA7000BF2A
:10900000A868032100222973827000BFAB68802703
:109010009F70FEF7B2B8A9681022CA7000BFA86896
:10902000032100222973827000BFAB6880279F70E4
:10903000FDF7FDBF88681022C27000BF8F68032053
:1090400000220873BA7000BF8B6880259D70FEF700
:1090500034B888681025C57000BF8B6803200022D3
:1090600008739A7000BF8E688022B270FEF7C9B88C
:109070008B680125DD7000BF8F68E2E78E680127ED
:10908000F77000BF8B68EBE7AB680127DF7000BFAC
:10909000A868C7E78B680125DD7000BF8F689BE774
:1090A000AB680127DF7000BFA868ACE710B40368A5
:1090B00041681A7890F809C00C78037A14EA0C0F0A
:1090C00002EA03021DD0847A04F003010AB141F0E0
:1090D000040141F008039A1003F1FF3C8272BCF1D5
:1090E0000D0F0BD8DFE80CF021071B070A15212113
:1090F000150A071B0721C268531EC3605DF8044BA5
:109100007047817A01F00303002AE4D043F004039E
:10911000E1E7C3689C1EC4605DF8044B7047C168FA
:109120005DF8044B0231C1607047C4680134C4600B
:109130005DF8044B704700BF08B5034BD3F8EC0053
:10914000FFF7B4FF08BD00BFE463FF1F08B5034B82
:10915000D3F8E800FFF7AAFF08BD00BFE463FF1FD4
:1091600008B5034BD3F8E400FFF7A0FF08BD00BF2C
:10917000E463FF1F08B5034BD3F8E000FFF796FF49
:1091800008BD00BFE463FF1F08B5034BD3F8DC0044
:10919000FFF78CFF08BD00BFE463FF1F08B5034B5A
:1091A000D3F8D800FFF782FF08BD00BFE463FF1FBC
:1091B00008B5034BD3F8D400FFF778FF08BD00BF14
:1091C000E463FF1F08B5034BD3F8D000FFF76EFF31
:1091D00008BD00BFE463FF1F08B5034BD3F8CC0004
:1091E000FFF764FF08BD00BFE463FF1F08B5034B32
:1091F000D3F8C800FFF75AFF08BD00BFE463FF1FA4
:1092000008B5034BD3F8C400FFF750FF08BD00BFFB
:10921000E463FF1F08B5034BD3F8C000FFF746FF18
:1092200008BD00BFE463FF1F08B5034BD3F8BC00C3
:10923000FFF73CFF08BD00BFE463FF1F08B5034B09
:10924000D3F8B800FFF732FF08BD00BFE463FF1F8B
:1092500008B5034BD3F8B400FFF728FF08BD00BFE3
:10926000E463FF1F08B5034BD3F8B000FFF71EFF00
:1092700008BD00BFE463FF1F08B5034BD3F8AC0083
:10928000FFF714FF08BD00BFE463FF1F08B5034BE1
:10929000D3F8A800FFF70AFF08BD00BFE463FF1F73
:1092A00008B5034BD3F8A400FFF700FF08BD00BFCB
:1092B000E463FF1F08B5034BD3F8A000FFF7F6FEE9
:1092C00008BD00BFE463FF1F08B5034BD3F89C0043
:1092D000FFF7ECFE08BD00BFE463FF1F08B5034BBA
:1092E000D3F89800FFF7E2FE08BD00BFE463FF1F5C
:1092F00008B5034BD3F89400FFF7D8FE08BD00BFB4
:10930000E463FF1F08B5034BD3F89000FFF7CEFED0
:1093100008BD00BFE463FF1F08B5034BD3F88C0002
:10932000FFF7C4FE08BD00BFE463FF1F08B5034B91
:10933000D3F88800FFF7BAFE08BD00BFE463FF1F43
:1093400008B5034BD3F88400FFF7B0FE08BD00BF9B
:10935000E463FF1F08B5034BD3F88000FFF7A6FEB8
:1093600008BD00BFE463FF1F08B5024BD86FFFF7CD
:109370009DFE08BDE463FF1F08B5024B986FFFF721
:1093800095FE08BDE463FF1F08B5024B586FFFF759
:109390008DFE08BDE463FF1F08B5024B186FFFF791
:1093A00085FE08BDE463FF1F08B5024BD86EFFF7CA
:1093B0007DFE08BDE463FF1F08B5024B986EFFF702
:1093C00075FE08BDE463FF1F08B5024B586EFFF73A
:1093D0006DFE08BDE463FF1F08B5024B186EFFF772
:1093E00065FE08BDE463FF1F08B5024BD86DFFF7AB
:1093F0005DFE08BDE463FF1F08B5024B986DFFF7E3
:1094000055FE08BDE463FF1F08B5024B586DFFF71A
:109410004DFE08BDE463FF1F08B5024B186DFFF752
:1094200045FE08BDE463FF1F08B5024BD86CFFF78B
:109430003DFE08BDE463FF1F08B5024B986CFFF7C3
:1094400035FE08BDE463FF1F08B5024B586CFFF7FB
:109450002DFE08BDE463FF1F08B5024B186CFFF733
:1094600025FE08BDE463FF1F08B5024BD86BFFF76C
:109470001DFE08BDE463FF1F08B5024B986BFFF7A4
:1094800015FE08BDE463FF1F08B5024B586BFFF7DC
:109490000DFE08BDE463FF1F08B5024B186BFFF714
:1094A00005FE08BDE463FF1F08B5024BD86AFFF74D
:1094B000FDFD08BDE463FF1F08B5024B986AFFF786
:1094C000F5FD08BDE463FF1F08B5024B586AFFF7BE
:1094D000EDFD08BDE463FF1F08B5024B186AFFF7F6
:1094E000E5FD08BDE463FF1F08B5024BD869FFF72F
:1094F000DDFD08BDE463FF1F08B5024B9869FFF767
:10950000D5FD08BDE463FF1F08B5024B5869FFF79E
:10951000CDFD08BDE463FF1F08B5024B1869FFF7D6
:10952000C5FD08BDE463FF1F08B5024BD868FFF70F
:10953000BDFD08BDE463FF1F08B5024B9868FFF747
:10954000B5FD08BDE463FF1F08B5024B5868FFF77F
:10955000ADFD08BDE463FF1F01380B463A2800F259
:109560005C82DFE810F053024C0245023E023702F3
:109570003002290222021B02AE01A701A0019901BB
:1095800092018B0184017D0176016F016801610107
:109590005A0153014C0145013E01370130012901B7
:1095A00022011B0113010B010301FB00F300EB007F
:1095B000E300DB00D300CB00C300BB00B300AB0073
:1095C000A3009B0093008B0083007B0073006B0063
:1095D00063005B0053004B0043003B00BC4ABD49A5
:1095E000C2F8EC303B2004220CF074B8B848BA49F9
:1095F000C0F8E83004223A200CF06CB8B44AB749FD
:10960000C2F8E430392004220CF064B8B048B44900
:10961000C0F8E030042238200CF05CB8AC4AB14904
:10962000C2F8DC30372004220CF054B8A848AE4908
:10963000C0F8D830042236200CF04CB8A44AAB490C
:10964000C2F8D430352004220CF044B8A048A84910
:10965000C0F8D030042234200CF03CB89C4AA54914
:10966000C2F8CC30332004220CF034B89848A24918
:10967000C0F8C830042232200CF02CB8944A9F491C
:10968000C2F8C430312004220CF024B890489C4920
:10969000C0F8C030042230200CF01CB88C4A994924
:1096A000C2F8BC302F2004220CF014B88848964928
:1096B000C0F8B83004222E200CF00CB8844A93492C
:1096C000C2F8B4302D2004220CF004B88048904930
:1096D000C0F8B03004222C200BF0FCBF7C4A8D492E
:1096E000C2F8AC302B2004220BF0F4BF78488A4932
:1096F000C0F8A83004222A200BF0ECBF744A874936
:10970000C2F8A430292004220BF0E4BF7048844939
:10971000C0F8A030042228200BF0DCBF6C4A81493D
:10972000C2F89C30272004220BF0D4BF68487E4941
:10973000C0F89830042226200BF0CCBF644A7B4945
:10974000C2F89430252004220BF0C4BF6048784949
:10975000C0F89030042224200BF0BCBF5C4A75494D
:10976000C2F88C30232004220BF0B4BF5848724951
:10977000C0F88830042222200BF0ACBF544A6F4955
:10978000C2F88430212004220BF0A4BF50486C4959
:10979000C0F88030042220200BF09CBF4C4A69495D
:1097A000D3671F2004220BF095BF494866498367A1
:1097B00004221E200BF08EBF454A644953671D20CA
:1097C00004220BF087BF42486149036704221C2032
:1097D0000BF080BF3E4A5F49D3661B2004220BF08A
:1097E00079BF3B485C49836604221A200BF072BFA4
:1097F000374A5A495366192004220BF06BBF34488C
:1098000057490366042218200BF064BF304A5549BB
:10981000D365172004220BF05DBF2D4852498365A4
:10982000042216200BF056BF294A504953651520D3
:1098300004220BF04FBF26484D4903650422142033
:109840000BF048BF224A4B49D364132004220BF08B
:1098500041BF1F4848498364042212200BF03ABFDD
:109860001B4A46495364112004220BF033BF1848A9
:1098700043490364042210200BF02CBF144A4149D1
:10988000D3630F2004220BF025BF11483E498363A8
:1098900004220E200BF01EBF0D4A3C4953630D20DD
:1098A00004220BF017BF0A483949036304220C2035
:1098B0000BF010BF064A3749D3620B2004220BF08D
:1098C00009BF03483449836204220A200BF002BF17
:1098D000E463FF1F399100004D9100006191000089
:1098E00075910000899100009D910000B1910000E8
:1098F000C5910000D9910000ED9100000192000097
:1099000015920000299200003D9200005192000043
:1099100065920000799200008D920000A1920000F3
:10992000B5920000C9920000DD920000F1920000A3
:1099300005930000199300002D930000419300004F
:10994000559300006993000079930000899300000B
:1099500099930000A9930000B9930000C9930000F7
:10996000D9930000E9930000F993000009940000E6
:1099700019940000299400003994000049940000D3
:1099800059940000699400007994000089940000C3
:1099900099940000A9940000B99400001F4A20493E
:1099A0005362092004220BF095BE1C481D49036236
:1099B000042208200BF08EBE184A1B49D3610720F1
:1099C00004220BF087BE1548184983610422062043
:1099D0000BF080BE114A16495361052004220BF09A
:1099E00079BE0E4813490361042210460BF072BE83
:1099F0000A4A1149D360032004220BF06BBE0748CA
:109A00000E498360042202200BF064BE034A0C4915
:109A10005360012004220BF05DBE7047E463FF1F1A
:109A2000C9940000D9940000E9940000F994000062
:109A3000099500001995000029950000399500004E
:109A400049950000F0B55C699FEDE47AD0ED047AA9
:109A5000D0ED0C6AC0ED037A042CC0F88010C0ED84
:109A60000B6A80ED057A80ED0D7A00F0DF801588B5
:109A7000D0ED064AD0ED025A06EE105AB8EE460A6C
:109A8000B0EE674A70EE670AB6EE005AA4EEA04A3E
:109A9000CD006E1A37EEE52A74EE671A03EB8103E8
:109AA000A1EE857A00EB8604D3F8147174EE072AD0
:109AB0008434F4EEC22AF1EE10FA80ED057AC0ED9E
:109AC000042A00F1AE8037EEA57AF4EEC72AF1EE53
:109AD00010FAC4BF72EEE57AC0ED037A90ED003A59
:109AE000D0ED073AD0ED010AB0EE006AF0EE434A3D
:109AF000E5EE864AB0EE430A77EEE47AA7EEA30AD3
:109B0000B4EEE00AF1EE10FA08D5B4EEC03AF1EE88
:109B100010FA54BFF0EE430AF0EE400A6E1A00EB62
:109B2000860C9CF8986046B1DFF8B8E243F2844CAA
:109B30001EF80C60002E00F07281E7604FF0000EFE
:109B4000A74FD0ED0C6A90ED0D4A90ED0B1AC4EDC5
:109B5000040AC4F804E0A760528890ED0E2AD0ED04
:109B60000A2AD3F8244101EE902AB8EE617AF0EE89
:109B7000663A37EE663AF6EE004AE2EE033A6B1AC0
:109B800000EB830631EE620A73EEE65AF43675EEA8
:109B9000C47AA7EEA44A33EE845A80ED0D4AB4EE9F
:109BA000C05AF1EE10FA80ED0C5A40F12B8135EEDF
:109BB000221A80ED0B1A90ED084AD0ED0F1AD0ED65
:109BC000093AB0EE002AF0EE446AE2EE826AB0EEA4
:109BD000447A31EE661AA1EE217AB4EEE37AF1EE20
:109BE00010FA08D5B4EEC74AF1EE10FA54BFF0EE01
:109BF000443AF0EE473A691A00EB810090F80851B8
:109C00003DB1784F43F2844C17F80C20002A00F045
:109C1000058100237249C6ED043AF4607360B160B7
:109C2000F0BD72EEA57AC0ED037A57E71488568826
:109C30006C4DDFF8ACE106EE104A05EE906A43F297
:109C40008447F8EE464AB8EE655AEF5D03F58A7C24
:109C5000B0EE470AF0EE673A03F592730246002130
:109C6000F6EE000AB0EE004A74EEE71AD0ED066A8E
:109C700090ED021A5CF8044BB0EE672AA6EEA12A1A
:109C800073EEC12A72EE677A37EEC76AA6EE207AC3
:109C900072EE075A80ED057AF4EEE25AF1EE10FA10
:109CA000C0ED045A40F1A28075EE813AC0ED033A4E
:109CB000D0ED001A90ED072AD0ED012AF0EE616A8E
:109CC000E1EE046A33EEE61AF0EE613AE1EE023AB2
:109CD000F4EEE23AF1EE10FA08D5F4EEE31AF1EE02
:109CE00010FA54BFF0EE612AF0EE632A92F8986001
:109CF00006B13FB182ED220AC2F88CE0C2ED252AFE
:109D0000C2F89040D0ED0C7A90ED0E6AD0ED0D5A6D
:109D1000D0ED0B1A90ED0A1A53F8044B35EE677A22
:109D2000B0EE672AA6EE072A71EEC12A72EE673AF4
:109D300033EEE53AE3EE205A72EE257AC0ED0D5A85
:109D4000F4EEE27AF1EE10FAC0ED0C7A3AD577EE45
:109D5000811AC0ED0B1AD0ED085A90ED0F7AD0EDB4
:109D6000096AB0EE652AA1EE042AB0EE651A71EE1A
:109D7000C21AA1EE871AB4EEE61AF1EE10FA08D56F
:109D8000F4EEC15AF1EE10FA54BFF0EE656AF0EE4F
:109D9000416A92F8085105B13FB182ED3E0AC2F81E
:109DA000FCE0C2ED416AC2F800410131042902F130
:109DB0001C023FF435AFD0ED047A90ED057AD0ED7A
:109DC000033A51E731EE816AF4EEC67AF1EE10FA09
:109DD000C4BF77EEC11AC0ED0B1ABCE7000000004B
:109DE00000F07F45F82AFF1F0000000031EE237AC3
:109DF000F4EEC75AF1EE10FAC4BF75EEC13AC0EDE9
:109E0000033A55E772EE810AB4EEE05AF1EE10FA29
:109E1000C4BF35EE621A80ED0B1ACCE6F0BDB0EE91
:109E2000661A1FED0F4A97E6F0B55569042D00F04C
:109E3000D982D0F880300C88DE00F71A00EB870C4E
:109E400007EE104ADCF88440B8EE470AD4ED047AF5
:109E5000D4ED065A94ED056AD4ED036AD4ED023AC6
:109E600070EE670AB0EE675AA5EEA05AF6EE001A39
:109E700035EE672A76EEE34A72EE462AA2EEA16A32
:109E800035EE064A84ED056AB4EEE44AF1EE10FAC6
:109E900084ED044A00F1F68136EEA37AB4EEC74AA7
:109EA000F1EE10FAC4BF74EE636AC4ED036A94ED78
:109EB000000AD4ED077AF0EE005AB0EE406AA3EE45
:109EC000A56AB0EE405AF0EE460A76EEE06A94EDEE
:109ED000016AA6EEA75AB4EEC65AF1EE10FA08D5FA
:109EE000B4EEC50AF1EE10FA54BFB0EE406AB0EE1F
:109EF000456AF71A00EB870C8CED276A9CF89840AE
:109F0000002C00F01082E24F43F2844C17F80C4012
:109F1000002C40F00882F71AB1F802C000EB870469
:109F200005EE10CAD4F8F440B8EE451AD4ED041A80
:109F300094ED062AD4ED052A94ED033AD4ED020AF5
:109F400071EE613AB0EE614AA2EE234A02EB83075A
:109F5000F6EE004A34EE610AF0EE626A70EE627A62
:109F600087ED456AE7EEA46A73EE605A34EE266A1E
:109F7000C4ED056AB4EEE56AF1EE10FA84ED046A08
:109F800040F17A8336EE203A84ED033A94ED001ADC
:109F9000D4ED071AD4ED017AB0EE002AF0EE412A92
:109FA000E0EE822AF0EE413A33EE623AE3EE213AF5
:109FB000F4EEE73AF1EE10FA08D5B4EEE31AF1EE5A
:109FC00010FA54BFF0EE417AF0EE637AF41A00EB27
:109FD000840CCCED437A9CF80841002C00F05C81A5
:109FE000DFF8ACE243F2844C1EF80C40002C40F049
:109FF0005381C7ED497A8C88D0F8643100EE104A5D
:10A0000093ED044AD3ED064A93ED056AD3ED030AB6
:10A0100093ED023AB8EE405AB0EE441A75EE445A47
:10A02000B6EE007AA4EEA51A70EEC37A31EE442A99
:10A0300072EE462AA2EE876A71EE063A83ED056A51
:10A04000F4EEE73AF1EE10FAC3ED043A40F1BE81C6
:10A0500073EE830AC3ED030A93ED004AD3ED074A7A
:10A06000D3ED017AB0EE006AB0EE445AA3EE065A80
:10A07000B0EE441A70EEC50AA0EEA41AB4EEE71AC8
:10A08000F1EE10FA08D5B4EEC14AF1EE10FA54BF61
:10A09000F0EE447AF0EE417A90F87861C0ED5F7AA4
:10A0A0002EB17B4F43F2844C17F80C30C3B390EDC4
:10A0B0005D7A37EEC72AB5EEC02AF1EE10FA00F14C
:10A0C000188340F32383D0ED5B6AD0ED5C2A9FEDCB
:10A0D000713AD0ED5A3A36EEC70A36EEE24AB4EE9D
:10A0E000C30AF1EE10FA64EE024AD8BFB0EE430A9A
:10A0F00084EE806A36EE225AF4EEC56AF1EE10FA6A
:10A1000008DDF4EEC53AF1EE10FA54BFF0EE636AE2
:10A11000F0EE456AC0ED5D7AC0ED5C6AF0EE667AFD
:10A12000C988D0F88041C2ED4E7A00EE901A94EDC5
:10A13000041AD4ED065AD4ED051A94ED032A94EDD1
:10A14000026AB8EE607AB0EE413A77EE412AB6EE96
:10A15000000AA5EEA23A72EE467A33EE414A74EE58
:10A16000614AE4EE801A73EE216AC4ED051AF4EE3A
:10A17000E76AF1EE10FAC4ED046A40F11B8136EE95
:10A18000862A84ED032A94ED001AD4ED075AD4ED03
:10A19000017AF0EE001AB0EE417AA6EE217AB0EE26
:10A1A000413A32EE472AA2EE253AB4EEE73AF1EE12
:10A1B00010FA08D5B4EEC31AF1EE10FA54BFF0EE5F
:10A1C000417AF0EE437A90F89461C0ED667A2EB150
:10A1D0002F4F43F2844C17F80C30C3B390ED640A50
:10A1E00037EEC06AB5EEC06AF1EE10FA00F1748283
:10A1F00040F39382D0ED626AD0ED634A9FED254A29
:10A20000D0ED610A36EEC01A36EEE45AB4EEC41A46
:10A21000F1EE10FA65EE065AD8BFB0EE441AC5EE5C
:10A22000811A31EEA47AF4EEC76AF1EE10FA08DD75
:10A23000F4EEC70AF1EE10FA54BFF0EE606AF0EEE9
:10A24000476AC0ED647AC0ED636AF0EE667A042D69
:10A2500008BF0025C5EBC5018C000619C2ED4F7A79
:10A26000D6F89C70C2F8B0700444D4F80CC1C2F89F
:10A27000B4C0D0F87C31C2F8B830D0F89801C2F838
:10A28000BC00F0BD74EE236AC4ED036A0FE600BFA4
:10A29000F82AFF1FBD378635F41A00EB840C9CEDBD
:10A2A000417A77EEC74AF5EEC04AF1EE10FA00F1B6
:10A2B000468240F34F829CED3F0ADCED400A5FEDA1
:10A2C0000B6A70EE475A30EE606AF4EEE65AF1EE31
:10A2D00010FA26EE241AD8BFF0EE665AC1EE251AFF
:10A2E00031EEA02A8CED402AF41A00EB840C9CED90
:10A2F0003F3ADCED3E2AB4EEC23AF1EE10FA08DD48
:10A30000F4EEC22AF1EE10FA54BFB0EE623AB0EEAB
:10A31000423AF31A00EB8306C6ED417A86ED403AE5
:10A32000F0EE437A65E6F71A00EB870CDCED251AB0
:10A3300036EE612AB5EEC02AF1EE10FA00F1F48192
:10A3400040F30B82DCED232A9CED243A5FED2F3A9B
:10A3500032EEE14A72EEC34AB4EEE34AF1EE10FA8D
:10A3600024EE820AD8BFB0EE634AC0EE047A77EEDC
:10A37000835ACCED245AF41A00EB8407D7ED236AF4
:10A38000D7ED220AF4EEE56AF1EE10FA08DDF4EEFC
:10A39000E50AF1EE10FA54BFF0EE606AF0EE656A7D
:10A3A000F41A00EB840C8CED256ACCED246AB0EE37
:10A3B000666AB0E572EE060AF4EEE06AF1EE10FAB3
:10A3C000C4BF36EEC62A84ED032ADCE630EE830AEB
:10A3D000F4EEC03AF1EE10FAC4BF73EEC30AC3ED57
:10A3E000030A39E60F884C881FED564ADFF874C31C
:10A3F00003EE907A07EE104AF8EE634AB8EE475A39
:10A40000034602F5927E02F58A770026F6EE005AA0
:10A41000B0EE006AD3F8844094ED040AD4ED060A45
:10A4200094ED051AD4ED036A94ED023A74EEC01A65
:10A43000B0EE402AA0EEA12A36EEC37A72EE402A90
:10A4400072EEC17AA7EEA51A32EE010A84ED051A62
:10A45000B4EEC70AF1EE10FA84ED040A40F100816F
:10A4600070EE036AC4ED036A94ED001AD4ED071A86
:10A47000D4ED017AB0EE412AA3EE062AF0EE413A7D
:10A4800076EEC26AE6EEA13AF4EEE73AF1EE10FAA1
:10A4900008D5B4EEE31AF1EE10FA54BFF0EE417AAB
:10A4A000F0EE637A93F89840C3ED277A14B19CF8E4
:10A4B0000040C4B393ED257A77EEC72AF5EEC02AA3
:10A4C000F1EE10FA00F1EF8040F3F88093ED230AEB
:10A4D000D3ED240A93ED221A70EE471A30EE602A6B
:10A4E000F4EEC41AF1EE10FA62EE226AD8BFF0EE72
:10A4F000441AC6EEA13A33EEA03AB4EEC30AF1EE26
:10A5000010FAB0EE407A08DDB4EEC31AF1EE10FA9C
:10A5100054BFB0EE417AB0EE437AC3ED257A83EDB5
:10A52000247AF0EE477AE7EC017AD3F8F44094ED20
:10A53000040AD4ED060A94ED051AD4ED031A94ED3D
:10A54000023A35EE402AF0EE402AE0EE822A72EE20
:10A55000C03A31EEC30A33EEC17AA7EE251A72EE85
:10A56000817A84ED051AF4EEC07AF1EE10FAC4EDAA
:10A57000047A69D577EE831AC4ED031A94ED001AB4
:10A5800094ED072AD4ED017AF0EE412AE3EE062A93
:10A59000F0EE416A71EEE21AE1EE826AF4EEE76AE9
:10A5A000F1EE10FA08D5B4EEE61AF1EE10FA54BF47
:10A5B000F0EE417AF0EE667A93F80841C3ED437A03
:10A5C00014B19CF80040B4B3D3ED413A37EEE30A3E
:10A5D000B5EEC00AF1EE10FA5AD476DDD3ED3F0A9B
:10A5E00093ED401AD3ED3E1A30EEE37A30EEC12AF5
:10A5F000B4EEC47AF1EE10FA62EE002AD8BFB0EEE3
:10A60000447AC2EE876A36EE813AF4EEC30AF1EE7E
:10A6100010FAF0EE603A08DDF4EEC31AF1EE10FA2B
:10A6200054BFF0EE613AF0EE433AC3ED417AC3ED28
:10A63000403AF0EE637A0136042EEEEC017A03F133
:10A640001C037FF4E7AED6E471EE830AF4EEE07A01
:10A65000F1EE10FAC4BF77EEC31AC4ED031A8DE70A
:10A6600076EE830AB4EEE00AF1EE10FAC4BF70EEA3
:10A67000436AC4ED036AF7E633EE205AB4EEC56AC6
:10A68000F1EE10FAC4BF36EE603A84ED033A7DE491
:10A69000D3ED3E1A93ED401AD3ED3F0A33EEE17A43
:10A6A00031EE612AA4E793ED221AD3ED240A93ED4B
:10A6B000230A77EE411A30EEC12A11E793ED243ACE
:10A6C00093ED221A93ED230A17E793ED403AD3ED69
:10A6D0003E1AD3ED3F0A98E7D0ED610AD0ED634A08
:10A6E0009FED1F4AD0ED626A30EE601A34EEE05AF8
:10A6F0008CE5D0ED5A3AD0ED5C2A9FED193AD0EDB9
:10A700005B6A37EE630A32EEE34AE8E4D0ED5A3A88
:10A71000D0ED5B6A90ED5C5AEEE4D0ED610AD0EDCD
:10A72000626A90ED637A7EE59CED227A9CED243A94
:10A73000DFED0B3A31EEC74A73EE474A0CE69CED6B
:10A740003E5ADCED400ADFED066A77EE455A30EE00
:10A75000C56ABAE59CED402AC6E5DCED245A0AE656
:10A76000BD3786357C5FFF1F016990ED016AD0ED32
:10A77000005AD0ED086A0029CCBFF0EE467AF1EE1F
:10A78000467A77EEA57A10B4F4EEE76AF1EE10FAA5
:10A7900029DD4269F0EE000A002AD6EEA07A4FF0D9
:10A7A000010433D1BCEEE71A436AC0ED007A0461BC
:10A7B00011EE10CA63445A1C02F07F0403F07F03B9
:10A7C00000EB840100EB8300F8EE410A90ED0A0AE9
:10A7D00091ED0A1A5DF8044B77EEE07A71EE401ABB
:10A7E000A7EEA10A70479FED3F7A426936EE870ACD
:10A7F000F4EEC07AF1EE10FAA3BFB0EE005AD0EE3C
:10A80000057A4FF0FF340C46002ACBD0C2F100028B
:10A8100001EE902AB8EEE12ACABF446A84698369CE
:10A82000D0F81CC072EE252AD8BF2346F4EEE26AA7
:10A8300000EB8404F1EE10FAC4F828C0436227DC70
:10A840009FED283A76EE833AF4EEE32AF1EE10FA21
:10A8500040DBB0EE004AD3EE842A4FF0FF310024F3
:10A860000161C0ED002A4461B1EE466A76EE227ABB
:10A87000F4EEE76AF1EE10FA1BDDB0EE007AD6EEE8
:10A88000877A01210161C0ED007ABCEEE71A8FE7FB
:10A89000F0EE004AD6EEA42A01210022016176EEF4
:10A8A000227AC0ED002AF4EEE76AF1EE10FA426176
:10A8B000E3DC9FED0C5A76EE855AF4EEE57AF1EE84
:10A8C00010FAE0DBF0EE006A4FF0FF34D5EEA67A26
:10A8D0000461D8E700229142C0ED002A4261C5DC44
:10A8E000C2E700BF0000FC422DE9F041437D012B8F
:10A8F0008CB062D0046EC26D944208D300239C4693
:10A9000001F1FF3898450CD00CB0BDE8F081651C12
:10A910000444056694F81CC001F1FF38634698456D
:10A92000F2D1457D8DF808C0012D00F0A781076E9A
:10A93000C36D9F42C0F0DF8000228DF809209F4246
:10A9400080F05B827E1C074406663A7F37468DF8AE
:10A950000A209F4280F04A827E1C074406663B7FA5
:10A960008DF80B3004290DF1080E20D00EEB0801F4
:10A970000DF10B02002502248027012609E008F1D1
:10A9800001038044036698F81C3002F8013F9142AD
:10A990000DD0437D012B00F0B480D0F86080C36DF2
:10A9A0009845ECD3002302F8013F9142F1D1416870
:10A9B000704688470CB0BDE8F08100268DF8036032
:10A9C0009DF80330036942F21074DF783D0625D408
:10A9D00093F803805FEA086220D493F803C05FEA2B
:10A9E0000C651BD4DA78120618D4DD782F0615D43E
:10A9F000DE78360612D4DF783D060FD493F8038054
:10AA00005FEA08620AD4083CDFD19C7000BF03698A
:10AA100080229A7000BF012404756FE79C7804F0CF
:10AA2000E7029A7003691D79EEB28DF803609F7892
:10AA300047F008049C7003690222DA70036942F24D
:10AA40001074DD78AF071BD4DE78B60718D4DF7832
:10AA5000BF0715D493F803C05FEA8C7610D493F83F
:10AA600003805FEA88750BD4DA78920708D4DD7822
:10AA7000AF0705D4DE78B60702D4083CE1D1C4E7BD
:10AA80009C7804F0C7079F70026942F21073D57872
:10AA9000AD0640F1AD81D678B40640F1A98192F8B7
:10AAA00003C05FEA8C6540F1A38192F803805FEAFE
:10AAB000886440F19D81D478A70640F19981D778C8
:10AAC000BE0640F19581D578AD0640F19181D678EA
:10AAD000B40640F18D81083BD9D1937000BF026963
:10AAE0008024947000BF0125066905750227357919
:10AAF000F7709C4604E77E1C074406663A7F37469B
:10AB00001BE78DF807509DF80730036942F2107873
:10AB100093F803C01CF0800F2ED193F803C01CF0F3
:10AB2000800F29D193F803C01CF0800F24D193F833
:10AB300003C01CF0800F1FD193F803C01CF0800FDE
:10AB40001AD193F803C01CF0800F15D193F803C0FD
:10AB50001CF0800F10D193F803C01CF0800F0BD1B4
:10AB6000B8F10808D4D183F8028000BF03699F7050
:10AB700000BF0023067516E793F8028008F0E70C83
:10AB800083F802C0036993F804805FFA88FC8DF8AB
:10AB900007C093F8028048F0080C83F802C00369EC
:10ABA000DC70036942F2107893F803C01CF0020FC6
:10ABB00023D193F803C01CF0020F1ED193F803C0F9
:10ABC0001CF0020F19D193F803C01CF0020F14D12E
:10ABD00093F803C01CF0020F0FD193F803C01CF0D0
:10ABE000020F0AD193F803C01CF0020F05D193F8AD
:10ABF00003C01CF0020F00F0738193F8028008F08C
:10AC0000C70C83F802C0D0F8108042F2107C98F88C
:10AC100003309B062DD598F803309B0629D598F86C
:10AC200003309B0625D598F803309B0621D598F86C
:10AC300003309B061DD598F803309B0619D598F86C
:10AC400003309B0615D598F803309B0611D5BCF14F
:10AC5000080CDCD188F802C000BF03699F7000BFF8
:10AC6000D0F810800675634698F804C088F8034051
:10AC70008BE698F8043088F8034086E600248DF8C7
:10AC800006409DF80630036942F21075DF783F06F2
:10AC900000F1B580DA78160600F1B180DE7834066E
:10ACA00000F1AD8093F803E05FEA0E6700F1A78042
:10ACB00093F803C05FEA0C6600F1A180DC782406FB
:10ACC00000F19D80DF783F0600F19980DA78160662
:10ACD00000F19580083DD9D19D7000BF03698024A3
:10ACE0009C7000BF0127427D07750023012A8DF863
:10ACF000093040F0D48100258DF805509DF80530CD
:10AD0000036942F2107293F803C05FEA0C6700F126
:10AD10001E8193F803E05FEA0E6600F11881DC788B
:10AD2000270600F11481DF783E0600F11081DE78FD
:10AD3000340600F10C81DD782F0600F1088193F8CC
:10AD400003C05FEA0C6600F1028193F803E05FEA5A
:10AD50000E6400F1FC80083AD5D19A7000BF0369F7
:10AD600080279F7000BF0125447D05750023012CBD
:10AD70008DF80A3040F0908100228DF804209DF873
:10AD80000430036942F2107593F803C05FEA0C6760
:10AD900000F1AB8093F803E05FEA0E6600F1A58056
:10ADA000DC78270600F1A180DF783E0600F19D8067
:10ADB000DE78340600F19980DA78170600F1958084
:10ADC00093F803C05FEA0C6600F18F8093F803E00C
:10ADD0005FEA0E6400F18980083DD5D19D7000BF07
:10ADE000036980269E7000BF012202750023B7E52B
:10ADF000137902279C46D77082E50022A7E59D784B
:10AE000005F0E7069E70036993F804E05FFA8EFC94
:10AE10008DF806C09C7844F008079F7002690225EF
:10AE2000D570036942F21075DE78B4071DD493F82B
:10AE300003E05FEA8E7718D493F803C05FEA8C745E
:10AE400013D4DC78A70710D4DF78BE070DD4DA78E6
:10AE500094070AD4DE78B70707D493F803E05FEAD3
:10AE60008E7602D4083DDFD136E79D7805F0C70421
:10AE70009C70026942F21073D778BE0640F10281DD
:10AE8000D678B50640F1FE8092F803C05FEA8C6781
:10AE900040F1F88092F803E05FEA8E6640F1F280BC
:10AEA000D578AD0640F1EE80D478A70640F1EA806F
:10AEB000D778BE0640F1E680D678B50640F1E2804C
:10AEC000083BD9D1937000BF04698027A77000BFE9
:10AED00001260269067502251679D570427D05E7BF
:10AEE000B8F108087FF460AE3DE69D7805F0E70410
:10AEF0009C7003691F79FEB28DF804609A7842F065
:10AF000008059D7003690224DC70036942F2107524
:10AF1000DF78BC074DD4DE78B7074AD4DA789707D4
:10AF200047D493F803C05FEA8C7642D493F803E0E9
:10AF30005FEA8E743DD4DC78A7073AD4DF78BE0789
:10AF400037D4DE78B40734D4083DE1D146E79A78A7
:10AF500002F0E7049C7003691F79FEB28DF805606A
:10AF60009D7845F008029A7003690224DC70036939
:10AF700042F21072DF78BC074DD4DE78B7074AD4AE
:10AF8000DD78AF0747D493F803C05FEA8C7642D4EC
:10AF900093F803E05FEA8E743DD4DC78A7073AD4D7
:10AFA000DF78BE0737D4DE78B40734D4083AE1D16D
:10AFB000D3E69D7805F0C7029A70046942F21073D7
:10AFC000E778BE065AD5E678B50657D594F803C09B
:10AFD0005FEA8C6752D594F803E05FEA8E664DD540
:10AFE000E578AD064AD5E278970647D5E778BE06FC
:10AFF00044D5E678B50641D5083BE1D1A37000BF42
:10B0000004698022A27000BF012704690775022528
:10B010002679E570A4E49A7802F0C7059D7004696A
:10B0200042F21073E778BE0631D5E678B5062ED524
:10B03000E27897062BD594F803C05FEA8C6626D594
:10B0400094F803E05FEA8E6521D5E578AF061ED55A
:10B05000E778BE061BD5E678B50618D5083BE1D1E2
:10B06000A37000BF07698025BD7000BF012602697B
:10B07000067502241679D470447D78E6022523797A
:10B08000E5706DE402251379D570427D2EE602222B
:10B090002379E270447D6AE6076EC36D59E4076E5A
:10B0A000C36D4CE408B5044B1A681AB1014610464A
:10B0B000FFF71AFC08BD00BFE063FF1F4FF47A7270
:10B0C0007E4B02FB01F19942F0B400F2CC807C4C43
:10B0D000A14200F2CC807B4DA94200F2CA807A4E98
:10B0E000B14200F2CB80794FB94200F2CB80784B6D
:10B0F000994200F2CD80774CA14200F2CB804EF213
:10B10000E045A94200F2A68047F26F26B14288BF0F
:10B110004FF4807200F29F806F4F4FF400464FF45F
:10B120008072B94280F0A78053006C4FB7FBF3FCEC
:10B13000614580F0A5801344B7FBF3F5A94280F088
:10B14000A3801344B7FBF3F4A14280F09F80134423
:10B15000B7FBF3FC614580F09F801344B7FBF3F528
:10B16000A94280F09B801344B7FBF3F4A14280F026
:10B1700097801344B7FBF3FC614580F09380134440
:10B18000B7FBF3F5A94280F08F801344B7FBF3F7C8
:10B19000B94280F08B801344504CB4FBF3FC614502
:10B1A00080F086801344B4FBF3F5A94280F08280DE
:10B1B0001344B4FBF3F7B94253D21344B4FBF3FC8A
:10B1C000614579D21344B4FBF3F5A9423ED213444E
:10B1D000B4FBF3F2914228BF102238D2F024404D44
:10B1E0003E49404A4FF47A7707FB03F3B1FBF3F390
:10B1F0004360286820F008072F60296821F47F2C1D
:10B200002CF47F6343F460203043204328601668A9
:10B21000330714D41468270711D415682E070ED4E9
:10B2200017683D070BD411680C0708D4136818077A
:10B2300005D41068010702D416683307E7D5284AF9
:10B24000146844F008051560F0BC70470F22511EC9
:10B250000C01C4E780225308204CB4FBF2F71E0215
:10B260005FE70D22F3E71D4F0026012259E7022276
:10B27000F1E70422EFE713460024B0E70822EAE7EB
:10B280000222E4E71022E6E70322E0E70422DEE7F9
:10B290002022E0E74022DEE70522D8E70622D6E7B3
:10B2A0000722D4E70822D2E70922D0E70A22CEE714
:10B2B0000B22CCE70C22CAE70E22C8E7DF7072002F
:10B2C0006F383900379C1C001B4E0E000D270700FD
:10B2D00086930300C2C901000E270700000E27074E
:10B2E0002C100B4024100B402DE9F04107468846F6
:10B2F0000AF0C4FE194C1A4E054604E00AF0BEFEE0
:10B30000431BB34226D82368DB07F7D4154A1648F7
:10B31000C2F8008007600AF0B1FE144C104F0646D8
:10B3200004E00AF0ABFE851BBD4213D82568104B24
:10B330000E492B40002BF4D00E480A6802600A60C8
:10B3400006680B4C3440A4F10104B4FA84F7780980
:10B35000BDE8F0810020BDE8F08100BF24100B4063
:10B3600040420F0008100B400C100B4030100B40F7
:10B3700001000F000466FF1F2DE9F04F85B03F4F1D
:10B380000190029103920AF079FEDFF82CA13C4E65
:10B39000BB468146DAF800803A4D0AF06FFE04465B
:10B3A00004E00AF06BFE011BA94225D83368D907D7
:10B3B000F7D4354A3548C2F8008050600AF05EFE86
:10B3C000304C054604E00AF059FE401BA04213D859
:10B3D00039682F4B0B40002BF5D02E4CDBF80000CA
:10B3E0002060CBF800002268294B1340012B03D1C9
:10B3F000294D2968CA050FD40AF040FE214BC9EB3C
:10B4000000049C42C6D9019840F23312292105B0AC
:10B41000BDE8F04F09F026BE204D214F2B701A4891
:10B42000039B2049029E002222603B601E4A1F4B64
:10B4300006600A601E481F49B86319600AF01EFEC4
:10B44000104E074604E00AF019FEC21BB2420BD8A8
:10B450002B78002BF7D12468154D2540022D03D100
:10B46000012005B0BDE8F08F019840F23D12232184
:10B4700005B0BDE8F04F09F0F5BD00BF30100B403E
:10B4800024100B4040420F0008100B4000001A0D22
:10B4900001000F000466FF1F10100B400866FF1F1D
:10B4A00000100B4004100B40400001000C100B403A
:10B4B00002007F1111003A060C66FF1F2DE9F04FC4
:10B4C00093B080460AF0DAFDA44CA54E054605E08F
:10B4D0000AF0D4FD421BB24200F2DC80236813F074
:10B4E0000100F5D19F49A04A086010600AF0C6FD2E
:10B4F0009E4C9B4D064605E00AF0C0FD871BAF42FF
:10B5000000F2C88020689A4B984F0340002BF3D07C
:10B51000DFF884A23968CAF800103960DAF8002030
:10B52000934E1640012E40F0B5808C4EBB464FF036
:10B530000A090AF0A3FD8A4D044604E00AF09EFDC4
:10B54000021BAA4225D83068C207F7D48549864D28
:10B55000884B834C4FF4D5720A602B600AF08EFD45
:10B56000054604E00AF08AFD401BA04211D8386865
:10B570007F4A0240002AF5D0DBF80030CAF80030DC
:10B58000CBF80030DAF80010794D0D40012D00F0B5
:10B590000582B9F10109CCD198F81110764B002938
:10B5A00008BF4FF4401301930AF068FD6F4F6B4CD6
:10B5B000DFF8B0B10090B9460AF060FD684E05466C
:10B5C00004E00AF05BFD401BB04258D8206810F040
:10B5D0000101F6D1644B694ACBF800101A600AF0F9
:10B5E0004DFD5F4D064604E00AF048FD811BA9426F
:10B5F00045D838685E4901400029F5D0D9F80020C7
:10B60000CAF80020C9F80020DAF80060584B33402F
:10B61000012B34D10AF032FD514E054604E00AF008
:10B620002DFD431BB3422AD82068C307F7D44E4BE5
:10B63000019A5349CBF8002019600AF01FFD484DCC
:10B64000064604E00AF01AFD821BAA4217D83868A1
:10B65000474901400029F5D0D9F80020CAF8002058
:10B66000C9F80020DAF80030414E1E40012E06D104
:10B670000AF004FD00993A4D401AA84215D94046F7
:10B6800040F29112432109F0EDFC8346584613B075
:10B69000BDE8F08F40464FF4BF72202109F0E2FC74
:10B6A0008346584613B0BDE8F08F364B1A68002A1F
:10B6B00082DA354D196829601C68284F600044BF44
:10B6C000324C26700AF0DAFC254E054605E00AF0F9
:10B6D000D5FC401BB04200F26B81386810F00103CA
:10B6E000F5D1214A1F4C2A49236011600AF0C6FC9B
:10B6F0001E4E1B4D074605E00AF0C0FCC11BA942C7
:10B7000000F2568130681A4B184C0340002BF3D0DE
:10B710002268CAF800202260DAF80010144F0F40A7
:10B72000012F40F045810AF0A9FC0C4C0C4E054657
:10B7300005E00AF0A3FC431BB34200F249812068F4
:10B7400010F00103F5D1084A064F12493B60116021
:10B750000AF094FC054C024D064625E024100B40EF
:10B7600040420F0008100B400C100B4030100B40F3
:10B7700001000F0000001A080000304000001A37D6
:10B780000000022910100B40FC65FF1FF865FF1F29
:10B790000000090200001A030466FF1F0AF06EFC95
:10B7A000871BAF4200F214812068B24BB24F0340B6
:10B7B000002BF3D03A68CAF800203A60DAF800109B
:10B7C000AC4E0E40012E40F00381AC4CDFF8D89215
:10B7D0002568AB4EAB4C280C0704C9F800700AF082
:10B7E0004DFC054605E00AF049FC421BB24200F25E
:10B7F000F7802368D907F6D4A349A44CA44A0F6064
:10B8000022600AF03BFC9C4F9D4D064605E00AF085
:10B8100035FC841BAC4200F2E3803868954B9649B6
:10B820000340002BF3D00C68CAF800400C60DAF833
:10B830000020904E1640012E40F0D2808F4F954D43
:10B84000954B964938682A681F68096888F824105B
:10B85000040A060C050E130A88F82F4088F83000F9
:10B860003C0C100C88F82C2088F8287088F82E6082
:10B87000120E3E0A88F82D5088F82B300D0A3F0E24
:10B88000090C002388F8276088F8264088F825707E
:10B8900088F8235088F82A0088F8292088F8221090
:10B8A00088F83130D9F80070764E754D0AF0E6FB15
:10B8B000044605E00AF0E2FB001BA84200F2988073
:10B8C0003068C207F6D47049704B754A0F601A6031
:10B8D0000AF0D4FB684D6A4C064605E00AF0CEFB40
:10B8E000811BA14200F2848028686249624F0140B6
:10B8F0000029F3D03B68CAF800303B60DAF800203A
:10B900005C4E1640012E73D15C4D624C2868624B30
:10B91000624A21681B68126888F82000050A060C34
:10B920000C0A88F81F50050E080C88F8142088F8B7
:10B930001C1088F81830090E88F81E6088F81D5011
:10B940001E0A1D0C88F81B401B0E140A88F81A00EA
:10B95000120C002088F8191088F8176088F8210068
:10B9600088F8165088F8153088F8134088F81220A7
:10B97000D9F800104B484C4EFFF7B6FC00283FD0DA
:10B9800031684A48FFF7B0FC002841D1404640F2F8
:10B99000AB12402109F066FB834682E6374F3C68D4
:10B9A000B4F5D57F0CD1424E88F811500196FBE5D5
:10B9B000404640F29912212109F054FB834670E67B
:10B9C00040464FF4C272252109F04CFB834668E6DD
:10B9D00040464FF4CE72222109F044FB834660E6D4
:10B9E000404640F2A112262109F03CFB834658E66E
:10B9F00040464FF4D272272109F034FB834650E6CB
:10BA0000404640F2A712242109F02CFB834648E669
:10BA100002212848FFF768FC83460028B6D0264D4F
:10BA2000264B2968174C21F006022A60286840F04E
:10BA300002062E604FF010151D600AF01FFB8DE806
:10BA40000101D9F800800E4E0AF018FB054604E00B
:10BA50000AF014FB401BB0424FD82368DB07F7D431
:10BA6000094A1749C2F8008051600AF007FB044DEB
:10BA700006462CE001000F0030100B4010100B4068
:10BA800040420F0024100B4008100B400C100B40DC
:10BA90000000090914100B4018100B401C100B403B
:10BAA0000000090A00001B070C66FF1F00001A3780
:10BAB0000000304000001A0628100B4044100B40D4
:10BAC00000001A0D0AF0DAFA811BA94215D838686D
:10BAD000484B0340002BF5D04749474A0E68CAF847
:10BAE00000601660DAF80050424A44492A40012AB0
:10BAF00003D143480368D80537D40AF0BFFA009D44
:10BB0000404E421BB2429CD9DDF8048040F2331211
:10BB10002921404609F0A6FA00284FD146F2A81183
:10BB2000DFF81CA1DFF81C91374F384E384D394CE7
:10BB30000020CAF80000C9F80000386030602860B2
:10BB400020604046FFF7BAFA40F243424FF4886360
:10BB50004FF0010CCAF80020C9F800203B603260A9
:10BB60002A60226088F810C09BE52B4C2B4F2C4D8F
:10BB70003A70002602AB0E60DDF80480294923608C
:10BB80006FF07F442C602848284A294D0D60294ECB
:10BB90002949066011600AF071FA1A4D044604E062
:10BBA0000AF06CFA031BAB421CD838780028F7D196
:10BBB000DAF800701F4A3A40022A13D19DF8154066
:10BBC000A307ABD502AA1D494046FFF7D5FB0028C5
:10BBD000A4D09DF8187007F00F03012B9ED14CF2F2
:10BBE00050319DE740F23D122321404609F03AFAD8
:10BBF00092E700BF01000F0030100B400466FF1FEA
:10BC000010100B4040420F0008D004400CD00440FC
:10BC100010D0044014D0044000100B400866FF1FF1
:10BC200008100B4004100B4038100B400C100B4058
:10BC30004000010002007F1111003A06F1FFFF8071
:10BC400000D0044004D004402DE9F04F85B08DE8C9
:10BC50000E003C4FDFF82C91DFF800A13A4E039024
:10BC6000BB46D9F80080394D0AF008FA044604E0D2
:10BC70000AF004FA031BAB42F3D83368D907F7D4B0
:10BC8000334A3448C2F8008050600AF0F7F92F4C6C
:10BC9000054604E00AF0F2F9411BA142E1D83968F7
:10BCA0002D4B0B40002BF5D0DBF80000CAF800004C
:10BCB000CBF80000DAF80020274D28491540012D67
:10BCC000CFD1274C2368DA05CBD5264F26483D70C7
:10BCD000264D00222E780A600199016036BB009C37
:10BCE0006202029B1A4D224E2A601C042148224AFD
:10BCF0002249234D44F400733360056011600AF05B
:10BD0000BDF9124C064604E00AF0B8F9851BA542BD
:10BD10000ED838780028F7D1DAF80070184A3A407F
:10BD2000022A05D1012005B0BDE8F08F009AD8E7BE
:10BD300003984FF40272332105B0BDE8F04F09F0CB
:10BD400091B900BF30100B4024100B4040420F004F
:10BD500008100B4000001A0D01000F000466FF1FC1
:10BD600010100B400866FF1F00100B40F865FF1F06
:10BD700004100B4038100B400C100B4027003A19F0
:10BD800002007F110C66FF1FF0B5002A059C5FDBE7
:10BD9000002B5DDB7F285BDC3F2959DC7F2AA8BFB5
:10BDA0007F2220EAE0763F2BA8BF3F23B24221EA60
:10BDB000E1779E464CDB274B186807EB861500EBB6
:10BDC00085010D1F02F1010C0EF10101BE4539DBA9
:10BDD000FB437A1C0B448A4203F007006C6005F1B8
:10BDE00004032FD010B301281BD0022816D003283B
:10BDF00011D004280CD0052807D006281CBF43F812
:10BE0000044F013243F8044F013243F8044F01322A
:10BE100043F8044F013243F8044F013243F8044F12
:10BE2000013201328A4243F8044F0BD008328A4271
:10BE30005C609C60DC601C615C619C61DC6143F85F
:10BE4000204FF3D10136664505F58075BED1F0BDB2
:10BE5000F0BD00BFD063FF1F2DE9F04FADF5337D7E
:10BE6000C1EB411EBC9D9DF8F44205EB8106D6F85E
:10BE70000471BD1EEEB2022E0ED8032F0EF1040681
:10BE800000F09681042F00F01B83022F00F05482F3
:10BE90000DF5337DBDE8F08F03EB41039FEDC16AE3
:10BEA000DF8A07EE907AB8EE670AF7EE006A80EE56
:10BEB000067AB4EEE67AF1EE10FA00F161814FF005
:10BEC0001A080EF10605B84E47683368A844A8F171
:10BED0000206360203EB060E06F50079CEF8D070A6
:10BEE0004768CEF8D07199444668C9F8D060476871
:10BEF000CEF8D0734668CEF8D0644768C9F8D470DD
:10BF0000002CC5D002EB810ACC01DAF80C69B2A989
:10BF1000771C06F1020B07F07F070BF07F0B27441D
:10BF200006F1030C06F1040E02EB8707A34406F1A9
:10BF300005080CF07F0A0EF07F0906F1060C06F1E9
:10BF4000070E02EB8B0B9BED432AD7F80CB141F89F
:10BF500008BC06F07F0708F07F080CF07F0C0EF09D
:10BF60007F0EA244A144A044A444A644274402EB6B
:10BF70008A0A02EB890902EB880802EB8C0C02EBBF
:10BF80008E0E02EB8707DAF80CA1D9F80C91D8F8DD
:10BF90000C81DCF80CC1DEF80CE1D7F80C7101ED76
:10BFA000032A41F810AC41F8149C41F8188C41F870
:10BFB0001CCC41F8047C41F820ED0DF1C80B8B45F9
:10BFC00006F10806A4D1ADF104064FF0000EB1460B
:10BFD0007146013102EE901AB8EEE23A73EE033A7E
:10BFE000BCEEE34A14EE107A802F28BF80277745F5
:10BFF00040F2C38032AA02EB8E0A524632AC04EB06
:10C000008708F2EC014A9FED695ACAEB080CACF1C3
:10C01000040B424575EE247ACBF382044FD054B31F
:10C02000012C22D0022C1CD0032C16D0042C10D0B2
:10C03000052C0AD0062C04D0DAED015A77EEA57A49
:10C040000432B2EC016A77EE867AB2EC010A77EE3E
:10C05000807AF2EC016A77EEA67AB2EC017A77EE9A
:10C06000877AF2EC010A77EEA07AB2EC011A424527
:10C0700077EE817A23D09246FAEC011A92ED012AEA
:10C08000DAED012A92ED033A92ED044AD2ED054A27
:10C0900092ED065AD2ED073A77EEA15A203235EEEC
:10C0A000826A424536EE220A70EE036A36EE847AE0
:10C0B00077EE240A30EE851A71EE237ADBD1CEEBCF
:10C0C000070201EE902AB8EE612A3229C7EE822AD1
:10C0D000BE46FCEEE27A17EE904A49F8044F7FF430
:10C0E00078AF9FED303A9FED314AF7EE004AB3EE5C
:10C0F0000A5A22E0A844A8F1020212029C184768DA
:10C1000044F8217002F5807C9C4444684CF821403E
:10C1100002F5007B9B4447684BF8217002F540799B
:10C120009944446849F8214002F5806A9A4442687B
:10C130004AF8212001393FF4ABAE56F8047F03EEF4
:10C14000907AF8EE635A4FF01A0885EE836AB4EEDF
:10C15000E46AF1EE10FACDD5B5EEC06AF1EE10FA50
:10C1600008DDB0EE440AA6EE050AFCEEC06A16EE43
:10C17000908ABFE74FF00008BCE7DFED0C7A9EE73E
:10C18000DFED0A0AB4EEE07AF1EE10FA40F35682DF
:10C19000B3EE0A1AE7EE010AFCEEE01A11EE908AFD
:10C1A0008FE600BF00F07F45D063FF1F0000000056
:10C1B000604A15680EF1220100F6047C00F2847ECC
:10C1C0001224771ADEF80430FA4302F007070EF162
:10C1D000040223B105EB0628436848F82430731C99
:10C1E000994200F09B80002F4CD0012F3FD0022FAE
:10C1F00034D0032F29D0042F1ED0052F13D0062FA3
:10C2000008D052F8047F27B105EB032B47684BF8A1
:10C210002470013352F8047F27B105EB03294768E6
:10C2200049F82470013352F8047F27B105EB032A43
:10C2300047684AF82470013352F8047F27B105EBB0
:10C240000328476848F82470013352F8047F27B167
:10C2500005EB032B47684BF82470013352F8047F39
:10C2600027B105EB0329476849F82470013352F8D8
:10C27000047F27B105EB032A47684AF8247001338D
:10C2800099424BD05768043227B105EB0328476821
:10C2900048F824705768013327B105EB032B476832
:10C2A0004BF82470976803F1010927B105EB092ABF
:10C2B00047684AF82470D76803F1020827B105EBF4
:10C2C000082B47684BF82470176903F1030927B15D
:10C2D00005EB092A47684AF82470576903F10408F6
:10C2E00027B105EB082B47684BF82470976903F1D9
:10C2F000050927B105EB092A47684AF82470D2F8E6
:10C300001C809F1D1C32B8F1000F04D005EB072BD9
:10C3100047684BF8247007339942B3D10EF1780E79
:10C32000F44504F101047FF44CAF0DF5337DBDE815
:10C33000F08F00BFD063FF1F604B1D680EF122011C
:10C3400000F2847C00F1040E2324771ADEF8043016
:10C35000FA4302F007070EF1040223B105EB0628A9
:10C36000436848F82430731C994200F09B80002FEA
:10C370004CD0012F3FD0022F34D0032F29D0042FCF
:10C380001ED0052F13D0062F08D052F8047F27B1F6
:10C3900005EB032B47684BF82470013352F8047FF8
:10C3A00027B105EB0329476849F82470013352F897
:10C3B000047F27B105EB032A47684AF8247001334C
:10C3C00052F8047F27B105EB0328476848F824702A
:10C3D000013352F8047F27B105EB032B47684BF874
:10C3E0002470013352F8047F27B105EB0329476815
:10C3F00049F82470013352F8047F27B105EB032A72
:10C4000047684AF82470013399424BD05768043288
:10C4100027B105EB0328476848F8247057680133B3
:10C4200027B105EB032B47684BF82470976803F19D
:10C43000010927B105EB092A47684AF82470D76833
:10C4400003F1020827B105EB082B47684BF824706D
:10C45000176903F1030927B105EB092A47684AF870
:10C460002470576903F1040827B105EB082B4768CE
:10C470004BF82470976903F1050927B105EB092AE8
:10C4800047684AF82470D2F81C809F1D1C32B8F10E
:10C49000000F04D005EB072B47684BF824700733D7
:10C4A0009942B3D10EF1780EF44504F101047FF402
:10C4B0004CAF0DF5337DBDE8F08F00BFD063FF1F9B
:10C4C000604A14680EF12205002100F6047E771BF5
:10C4D000DEF80430FA4302F0070701310EF10402DE
:10C4E00023B104EB0629436849F82130731C9D42AF
:10C4F00000F09B80002F4CD0012F3FD0022F34D072
:10C50000032F29D0042F1ED0052F13D0062F08D0BB
:10C5100052F8047F27B104EB032A47684AF82170D8
:10C52000013352F8047F27B104EB0328476848F829
:10C530002170013352F8047F27B104EB032B4768C5
:10C540004BF82170013352F8047F27B104EB032C20
:10C5500047684CF82170013352F8047F27B104EB8F
:10C560000329476849F82170013352F8047F27B145
:10C5700004EB032A47684AF82170013352F8047F1C
:10C5800027B104EB0328476848F8217001339D4226
:10C590004BD05768043227B104EB032B47684BF8A4
:10C5A00021705768013327B104EB032C47684CF81E
:10C5B0002170976803F1010927B104EB092A476844
:10C5C0004AF82170D76803F1020827B104EB082B61
:10C5D00047684BF82170176903F1030C27B104EB8E
:10C5E0000C29476849F82170576903F1040A27B1FB
:10C5F00004EB0A28476848F82170976903F1050B96
:10C6000027B104EB0B2C47684CF82170D2F81C9032
:10C610009F1D1C32B9F1000F04D004EB072A4768B4
:10C620004AF8217007339D42B3D110290EF1780EDC
:10C630007FF44DAF0DF5337DBDE8F08F4FF000086E
:10C640003FE400BFD063FF1F2DE9F04F8BB0BC4F1C
:10C65000049000F55B504A1C0430DFF83093DFF89B
:10C66000F8A2B84E01920090BB46D9F80080B64DB2
:10C6700009F004FD044604E009F000FD021BAA4293
:10C68000F3D83168C907F7D4B048B14BC0F800807F
:10C69000436009F0F3FCAC4C054604E009F0EEFC05
:10C6A000401BA042E1D83A68AA4911400029F5D0C0
:10C6B000DBF80030CAF80030CBF80030DAF80000C0
:10C6C000A44DA5490540012DCFD1A44C2268D20527
:10C6D000CBD5A34FA3483D70A34D00232E780B600C
:10C6E00000990160002E40F06084019C630297482D
:10C6F0009E4A9F499F4C03609F4EA04B4FF481354B
:10C7000015600E60236009F0B9FC8F4E044605E009
:10C7100009F0B4FC011BB14200F24A8438780028C9
:10C72000F6D1DAF80070944A3A40022A40F0408488
:10C73000049F0099924D742243F2B03807F5867039
:10C7400008F0E4FE3E887C8857F80830DFED8D6AFB
:10C7500093ED047A196D1A6F186BD86204EE906A23
:10C7600005EE104A43F28446B8EE640A15F806E076
:10C77000854ED964F8EE450ADA66F0EE663AF0EED8
:10C78000477AB0EE664A83ED037AC3ED056AC3EDDE
:10C790000D6AC3ED156AC3ED1D6A1A4607F5A87C3C
:10C7A00007F5B0780421F6EE005AB0EE006A30EEDC
:10C7B000471AD3ED062A93ED023A5CF8044BB0EE2B
:10C7C000472AA2EE812A77EEC36A32EE477A77EEE5
:10C7D000634AE4EEA53A32EE235AC3ED053AB4EECD
:10C7E000E65AF1EE10FA83ED045A40F19C8075EEA2
:10C7F000037AC3ED037A93ED001AD3ED072AD3ED44
:10C80000016AB0EE412AA3EE062AB0EE413A77EE75
:10C81000C27AA7EEA23AB4EEE63AF1EE10FA08D5E3
:10C82000B4EEC31AF1EE10FA54BFF0EE416AF0EE26
:10C83000436A92F8985015B1BEF1000F07D082ED0F
:10C84000224AC2F88C60C2ED256AC2F8904093ED8E
:10C850000C7AD3ED0E4A93ED0D5A93ED0B1A93ED2E
:10C860000A2A58F8040B70EEC73AF0EE477AE4EE65
:10C87000A37A71EE422A77EEC71A71EEC56AA6EE68
:10C88000A55A37EE857A83ED0D5AB4EEE27AF1EED1
:10C8900010FA83ED0C7A3AD537EE021A83ED0B1AB3
:10C8A00093ED085AD3ED0F3AD3ED091AF0EE452A6D
:10C8B000E2EE062AF0EE457A31EE621AE1EE237AD4
:10C8C000F4EEE17AF1EE10FA08D5B4EEE75AF1EEA3
:10C8D00010FA54BFF0EE451AF0EE671A92F808719C
:10C8E00017B1BEF1000F07D082ED3E4AC2F8FC60DE
:10C8F000C2ED411AC2F80001013902F11C024BD00D
:10C9000093ED047AD3ED053AD3ED037A4FE771EE58
:10C91000024AB4EEE47AF1EE10FAC4BF37EE421ADE
:10C9200083ED0B1ABCE773EE273AB4EEE35AF1EE4F
:10C9300010FAC4BF75EE437AC3ED037A5BE700BF1C
:10C9400030100B4024100B4040420F0008100B40E9
:10C9500000001A0D01000F000466FF1F10100B40AD
:10C960000866FF1F00100B40F865FF1F04100B4006
:10C9700038100B400C100B4002007F1137003A12A8
:10C98000F82AFF1F0000000000F07F450C66FF1F23
:10C99000AE47813F00F07F45049E93ED140AB6F840
:10C9A00004A0D3ED160A93ED156AD3ED136AD3ED07
:10C9B000123AD6F8744104EE10AAF8EE445AB0EEDA
:10C9C000405A75EEC04AB6EE002AA0EEA45A36EEE2
:10C9D000E37A35EE401A31EE463AA3EE026A75EE7E
:10C9E000067A83ED156AF4EEC77AF1EE10FAC3ED1C
:10C9F000147A40F1CE8277EEA36AC3ED136A93ED09
:10CA0000100AD3ED170A93ED112AB0EE006AF0EE8A
:10CA1000405AE3EE865AB0EE405A76EEE56AA6EE4C
:10CA2000A05AB4EEC25AF1EE10FA08D5B4EEC50A17
:10CA3000F1EE10FA54BFB0EE402AB0EE452A93F85A
:10CA40007821002A00F0CF81BEF1000F40F0CB81A9
:10CA5000049F93ED1C3AF988D3ED1E1AD3ED1D3ACD
:10CA600093ED1B4AD3ED1A2AD7F8786101EE101A1C
:10CA7000F8EE417AB0EE430A37EEC37AB6EE006ABA
:10CA8000A1EE870A34EE622A70EE435A75EEE34A4D
:10CA9000E4EE863A30EE235AC3ED1D3AB4EEC25AA4
:10CAA000F1EE10FA83ED1C5A40F1678235EE224A0E
:10CAB00083ED1B4A93ED183AD3ED1F1A93ED197AC3
:10CAC000F0EE003AF0EE437AE2EEA37AF0EE430A9B
:10CAD00034EE674AE4EE210AF4EEC70AF1EE10FAEA
:10CAE00008D5B4EEE03AF1EE10FA54BFB0EE437A56
:10CAF000B0EE607A93F89441002C00F06981BEF1A9
:10CB0000000F40F0658104985FED5F6AD0ED544AF4
:10CB10001FED602AD0ED585A24EEA65AFDEEE52A04
:10CB2000B4EEC25AF1EE10FAD8BFBDEEC55A12EEFD
:10CB3000907AD4BF15EE100A40F6FF7079110144C7
:10CB400041F27D06B14200F31682C34D21EAE17243
:10CB500005EB8209D9F800400498DFEDC01A90ED8A
:10CB6000553A9FEDBF0A90ED591A046763EE217A9A
:10CB7000FDEEC13AF4EEC07AF1EE10FAD8BFFDEE48
:10CB8000E77A13EE903A8246D4BF17EE90AA40F6A9
:10CB9000FF7A5F11574441F27D018F4200F3E98132
:10CBA000AD4C27EAE77504EB850BDBF800600498D1
:10CBB0009FEDAA6AD0ED560ADFEDA94A90ED5A4AD8
:10CBC000466760EE865ABDEEC47AF4EEE45AF1EEA2
:10CBD00010FAD8BFFDEEE55A17EE102A8446D4BFEE
:10CBE00015EE90CA40F6FF7C5311634441F27D0775
:10CBF000BB4200F3BC81984923EAE37401EB84084B
:10CC0000D8F80060049DDFED956A95ED575AD5ED93
:10CC10005B2A9FED933AAE6725EE261ABDEEE22A17
:10CC2000B4EEC31AF1EE10FA12EE100AD8BFBDEE40
:10CC3000C11A4FEA6012D4BF11EE100A40F6FF701D
:10CC4000104441F27D03984200F38F81824E20EA26
:10CC5000E07106EB810ADAF80070049C04F5A6582E
:10CC600004F5E750A446E767454604F5E657424613
:10CC700004460C3207F1140B083410350CF59E777E
:10CC8000002002920694059507970190079E56F89A
:10CC9000043F079613F0FF04039400F0F580042C82
:10CCA00003D8059A039C00211170A51E022D00F2E5
:10CCB000A580039F032F00F05381042FF0EE081A84
:10CCC000F7EE003A08BFF0EE613ACDED003A049875
:10CCD000019E644900F59E5E4FF40A7CDEF80890E0
:10CCE00033468A220CFB06966FF00800344606F1A4
:10CCF00014074FF0FF3A02FB03F8002534E09FEDE4
:10CD0000617A74EE075AF0EE004AB4EEE56AF1EE8D
:10CD100010FA04DB95EEA46A4FF0FF33336101355E
:10CD20000020802D84ED006A9FED4F5A386065D059
:10CD300006EE905A9DED001ADFED4C1ADFED4C7AAD
:10CD4000B8EEE62A22EE013A63EE213A83EEA70A14
:10CD500030EE454A14EE100A0CF05AFC41EC100B70
:10CD60000BF01EF951EC100B636A5A1E02F07F03A0
:10CD7000A36100223F4B0CF0EDFA35A3D3E9002369
:10CD80000CF09AFC00223C4B0CF096FC0CF056FF89
:10CD9000E061C7F800A0A169E069414409EB810C9A
:10CDA000F7EE000ACCF82800A269626296ED000A4C
:10CDB00096ED084A30EE206AB4EEC64AF1EE10FA5B
:10CDC0009DDDF0EE002A012194EE226A3161A6E792
:10CDD00000252A4A83ED647AC3F88C61C3F8845134
:10CDE000C3F888218FE60025244883ED5D2AC3F827
:10CDF0007041C3F86851C3F86C0129E6029E96F8A9
:10CE00000090A9F10204022C02D8039F012F45D9FA
:10CE1000019E029C069F059A9DF80C0004F8010BE8
:10CE2000013610370132042E019602940BF1040BE7
:10CE3000069705927FF42AAF114D049E2968099147
:10CE4000099BC6F8E4300BB0BDE8F08FAFF300806B
:10CE50000000000000FEAF4038E20100AE47813F15
:10CE600000F07F45FFFFEFBFDB0FC93FDB0F4940FD
:10CE70000000FE420000F03F0000E03F00F07F4570
:10CE80002C66FF1F0000FC42029D059995F800A04A
:10CE9000AAF102030122022B0A70B9D80498019961
:10CEA000069B00F59E560836D6F800E04FF40A7847
:10CEB0004FF0140C08FB01E400208A2704EB0C055A
:10CEC000C3F800C0224681464FF0FF3807FB01F748
:10CED0004FEAC11CF7EE000AB0EE006A4FF0010AFB
:10CEE00014E05FED182A37EE225AF4EEC54AF1EE4F
:10CEF00010FA04DBD5EE064A4FF0FF332361013010
:10CF00008028C2ED004AC5F8009081D0DBF80030DF
:10CF1000516A034403F07F03634406EB8303013942
:10CF2000D3F80C31D36101F07F019161C5F8008025
:10CF30009369D1693B440EEB830399629169516215
:10CF4000D4ED005A94ED087A75EEA04AB4EEE47A76
:10CF5000F1EE10FAC5DDD7EE064AC4F810A0CEE710
:10CF6000F0EE007ACDED007AB1E6174F75E6164E79
:10CF700048E6154E1BE6144CEEE534EE221AB4EEEC
:10CF8000C15AF1EE10FAC4BF35EE624A83ED1B4A76
:10CF900090E536EEA34AF4EEC47AF1EE10FAC4BF7F
:10CFA00077EEE36AC3ED136A29E5019BFFF79FBBA8
:10CFB000049D05F552504FF4F4723121083008F009
:10CFC00051F8FFF7B5BB00BF00005C452DE9F04FFD
:10CFD00081460024012580F83C4080F83D400464EF
:10CFE00044648464C46487B02146C9F85040C9F8D9
:10CFF0005440C9F8584089F85E4089F8964089F84D
:10D000005C5089F85D503C2298300DF087F9D54B83
:10D01000C9F8D440186805902D21D34B059889F89C
:10D02000DC4089F8DD40C9F8E440C9F8E84089F8F7
:10D030000C4189F80D4189F80E51C9F820414FF093
:10D040007E55C9F82441C9F82841C9F82C41C9F8CE
:10D050004041C9F84441C9F84841C9F84C41C9F8B0
:10D060009810C24EC24FC9F8D86063210F22052420
:10D07000C9F89C20C9F8A040C9F8E000C9F8A4503C
:10D08000C9F8A850C9F80051C9F80451C9F81011DD
:10D09000C9F83011C9F81411C9F8341103F5A07E8C
:10D0A000C9F81811C9F83811C9F81C11C9F83C1190
:10D0B0001A689E681D69D3F818C01C6A986A196BB3
:10D0C000D3F838A007EBC20807EBC606D8F804B0BF
:10D0D0005A68CBF8002007EBC5087568DA682A6043
:10D0E00007EBCC0CD8F804505E692E60DCF8042005
:10D0F000DD69156007EBC40407EBC00066685C6A75
:10D1000034604268DD6A156007EBC1015C6B4E68F4
:10D1100007EBCA0A3460D86BDAF8041040339E4536
:10D120000860C5D1934B934C5D6B9E6B2A68206B56
:10D130009149C9F8841116430223002289F88831E5
:10D1400089F8902189F89121C9F89421C9F8D8214A
:10D15000C9F8DC212E60C9F88C010270D9F88C5115
:10D16000864E6A70D9F88C41854DA270D9F88C0131
:10D17000FF21C170D9F88C315A71D9F88C415020F7
:10D18000A071D9F88C11CA71D9F88C4194F802E0D9
:10D190000EF07F03A370D9F88C01964609F5C27191
:10D1A0001222C270F446F04600914FF0FF304FF06B
:10D1B000010B744A0BFA0EF40021A3E0CAF5C31A5E
:10D1C0000AF52063984202D91846F0468C465388E7
:10D1D00004FB03F3B6FBF3FAAA4501F1010100F2E7
:10D1E000A880CAF5C31A0AF52063984202D91846E6
:10D1F000F0468C46938804FB03F3B6FBF3F3AB4293
:10D2000001F1010A40F2A280A3F5C313A3F5206344
:10D21000984205D9D446F046002B00F0F38018461A
:10D22000D38804FB03F3B6FBF3F3AB4201F1020A2C
:10D2300040F2AA80A3F5C313A3F52063984205D951
:10D24000D446F046002B00F0DD801846138904FB1D
:10D2500003F3B6FBF3F3AB4201F1030A40F29F8004
:10D26000A3F5C313A3F52063984205D9D446F0462D
:10D27000002B00F0C7801846538904FB03F3B6FB6C
:10D28000F3F3AB4201F1040A40F29480A3F5C31317
:10D29000A3F52063984205D9D446F046002B00F050
:10D2A000B1801846938904FB03F3B6FBF3F3AB425A
:10D2B00001F1050A40F28980A3F5C313A3F52063A9
:10D2C000984205D9D446F046002B00F09B801846C2
:10D2D000D38904FB03F3B6FBF3F3AB4202F10E0276
:10D2E00001F1060A7CD9A3F5C313A3F52063984284
:10D2F00005D9D446F046002B00F08480184607314B
:10D30000402979D0538804FB03F3B6FBF3FAAA450E
:10D3100002F102027FF652AFAAF5C313A3F5206310
:10D3200098427FF654AFF0468C46002B6AD01846E0
:10D330004DE7AAF5C313A3F5206398427FF65AAFD1
:10D34000F0468C46002B5DD0184653E7C3F5C31357
:10D3500003F5206398427FF663AFD4461846F04643
:10D360005EE700BF2C66FF1FF8E001006F12033B71
:10D37000FC2E02004C2B0200C4DF01000087930347
:10D38000FF691800922B0200C3F5C31303F5206355
:10D3900098427FF65BAFD4461846F04656E7C3F591
:10D3A000C31303F5206398427FF666AFD446184650
:10D3B000F04661E7C3F5C31303F5206398427FF697
:10D3C00071AFD4461846F0466CE7C3F5C31303F5B6
:10D3D000206398427FF67CAFD4461846F04677E744
:10D3E000C3F5C31303F52063984288D90731402958
:10D3F000D4461846F04685D1BEF1020F02D00EF198
:10D40000010ED6E60CF03F02D9F88C01E44942EA5D
:10D410008814E3B24370D9F88C516E7946F020023B
:10D420006A71D9F88C41607940F080036371D9F852
:10D430008C51DC48AE7846F08002AA7099F888A139
:10D440000AEB4A0400EBC40C4FF0010BDCF80C5063
:10D450006B099E0006F1604808F5614E05F01F0259
:10D46000D14D009B00240BFA02F0CEF80000AB6017
:10D470000820C9F88411C9F8E44189F8E841C9F8DD
:10D48000EC4108F023F92146064607F08DFFD9F854
:10D490008C11C9F8E4618D78C448C54A05F0FE03D3
:10D4A0008B70D9F8E4613179017099F888A1BD4891
:10D4B000D9F8E4510AEB4A0C00EBCC082B79D8F8E8
:10D4C000106003F1804A0AF5043506F03F0141F08F
:10D4D00080002C702870D9F8E4E199F888C1B14E29
:10D4E0009EF804100CEB4C0306EBC3084D1101F140
:10D4F000100AB04ED8F8140046F82A00AB0003F129
:10D50000604C0CF5614801F01F01DEF800000BFAD9
:10D5100001F5C8F80050B0F81CE01FFA8EFA4AF086
:10D5200008038383868B009BB1B241F002059E4EB7
:10D530008583194609F5FC70B360F3F793FF40202B
:10D5400009F10A0109F10C024123C9F80C02C9F8DA
:10D550001812442045214FF0430A09F10E084FF0FC
:10D56000420C09F1100E272609F11205C9F8102204
:10D57000C9F81432262209F11403C9F83C02C9F88B
:10D58000641209F10200242189F80642C9F81CA29C
:10D59000C9F844A2C9F86CA2C9F82082C9F8488227
:10D5A000C9F87082C9F824C2C9F84CC2C9F874C25B
:10D5B000C9F828E2C9F850E2C9F878E2C9F82C6243
:10D5C000C9F85462C9F87C62C9F83052C9F8585297
:10D5D000C9F88052C9F83422C9F85C22C9F8383237
:10D5E000C9F86032C9F86802C9F80892C9F84092CF
:10D5F000C9F88422C9F88C12232109F10400C9F862
:10D6000094122521C9F89002C9F89C1209F108006A
:10D610001621C9F89802C9F8C41209F106001F21A1
:10D62000C9F8A002C9F8CC1209F11E002021C9F8DE
:10D63000C802C9F8D41209F120001321C9F8D00298
:10D64000C9F8DC1209F122000F21C9F8D802C9F883
:10D65000041309F124005849C9F8E00209F1160041
:10D66000C9F88832C9F8A4A2C9F8A882C9F8ACC21E
:10D67000C9F8B0E2C9F8B462C9F8B852C9F8BC2216
:10D68000C9F8C032C9F8E4A2C9F8E882C9F8ECC206
:10D69000C9F8F0E2C9F8F462C9F8F852C9F8FC22F6
:10D6A000C9F80033C9F80803C9F8403303C9424B2D
:10D6B000C9F824A3C9F830E3C9F834634FF0100A5D
:10D6C0004FF0110E09F11A06C9F82883C9F82CC3C6
:10D6D000C9F83853C9F83C23C9F80CA3C9F814E3B6
:10D6E000C9F8186309F11808122509F11C0209F597
:10D6F000537C03F1080E4FF00406DFF8CCA0C9F804
:10D700001083C9F81C53C9F8202389F8446389F8A9
:10D7100045B3C9F848A38CE803009EE8030009F567
:10D72000557888E80300254989F85C43C9F8CC4559
:10D73000C9F8D0450C68224A224DC9F8605344F01C
:10D74000006009F55278C2F800800860AB6823F0E9
:10D750000C06AE60A96841F00404AC60686A40F051
:10D7600004036B626E6A26F0030169626C6A44EA24
:10D770000B006862EB6843F00806EE60A96841F0B0
:10D780000304AC60A86840F02003AB60EE6846F08C
:10D790000401E9602C6A14F0400009F5037C15E0EF
:10D7A000D0DF01004C2B0200EC65FF1F1A80004007
:10D7B000F8FB02200002FF1FD4DF01003C80044080
:10D7C000E464FF1F00B003408CDF010000F05B86C3
:10D7D0002B6A23F040065C462E62AB4B5D6A45F037
:10D7E000C0015962586AA849000614D55E6A30061D
:10D7F00011D55D6A2E060ED5586A05060BD55E6AF0
:10D80000300608D55D6A2E0605D5586A050602D58C
:10D810005E6A3006E6D44B6A0B691CB10C6A44F0B0
:10D8200040030B62984E994BF56CB06C716C346C84
:10D8300028440144F06BB56B0C44954920440544E1
:10D8400003C96C0844F4004509F5BB6BF562C9F8DF
:10D85000D4A5C9F848338BE803009EE8030009F516
:10D86000BC6A8AE803008B4C8B482668C9F8EC0533
:10D8700046F000610125002689F8E855C9F8586886
:10D88000C9F85C682160846824F00C0181608668B6
:10D8900046F004048460416A41F004064662446A2A
:10D8A00024F00301416209F2D4515160426A2A43D3
:10D8B0004262C66846F00804C460826842F003060B
:10D8C0008660846844F020028260C66846F00404E2
:10D8D000C460026A12F0400618BF066A6E4A1CBF96
:10D8E00026F040060662506A40F0C00408BF354684
:10D8F0005462566A684816F080061BD0546A14F0C9
:10D90000800617D0566A16F0800613D0546A14F0B9
:10D9100080060FD0566A16F080060BD0546A14F0B9
:10D92000800607D0566A16F0800603D0546A14F0B9
:10D930008006DED1426A009602691DB1056A45F093
:10D9400040020262544A554DD66C906C546C30447F
:10D950000444106CD66B2044946B06443444600835
:10D9600040F4004609F5517ED66209F5066BC9F808
:10D97000D435CDF80490E2464D26F14610E04346FA
:10D98000D3F8842203EBC20C0132C3F88422CCF812
:10D990001C00CCF820E00AF1080ACA4500F0828099
:10D9A000D8459AE80140F6D015F800C00CF01F03E6
:10D9B0001F2BE4D1C1EB0B04394AA30802FB03F38C
:10D9C00013F0030C0C462AD00C7D06FB04520B46C8
:10D9D000145C04F01F021F2A01F52374D0D1BCF19E
:10D9E000010F1CD0BCF1020F0CD0234601F5A3643B
:10D9F00093F814C006FB0C5212F800C00CF01F0282
:10DA00001F2ABDD1234604F5237493F814C006FBE6
:10DA10000C5212F800C00CF01F021F2AB0D15C4556
:10DA2000234604F5237CB6D0227D06FB0252125C0D
:10DA300002F01F021F2AA3D19CF8143006FB0352E8
:10DA4000634612F800C00CF01F021F2A04F5A36CF5
:10DA500096D194F82C3506FB0352634612F800C0A9
:10DA60000CF01F021F2A04F2A47C89D194F8B83765
:10DA700006FB035204F52364135C03F01F021F2A04
:10DA800063467FF47DAFCAE700B003409CDF01002E
:10DA9000D4DF01003080044000B00B40B02A020007
:10DAA0000BB31A05DDF80490F149C9F86818002590
:10DAB00014244FF4FA760520C9F86048C9F8646860
:10DAC000C9F86C08C9F8705889F8745889F87558FD
:10DAD000022108F097FAE64BC9F880380620C9F809
:10DAE0007848C9F87C68C9F8885889F88C5889F84A
:10DAF0008D58C9F88408022108F084FADC4AC9F874
:10DB000098281920C9F89048C9F89468C9F8A0580D
:10DB100089F8A45889F8A558C9F89C08022108F08A
:10DB200071FA6FF0004617230E20C9F8A848D04CB0
:10DB3000C9F8C83889F8B658C9F8B868C9F8C0082B
:10DB40000221C9F8BC48C9F8C44808F05BFA0221B0
:10DB500099F8C80808F056FA386F012500F50071E9
:10DB6000C9F8AC1889F8B458D7F8B87089F8B5581E
:10DB700007F50072C9F8B028022008F0A1FAD9F818
:10DB8000AC6899F8B488337813EA080F05D099F88F
:10DB9000B64844F0010089F8B608D9F8B05899F8A9
:10DBA000B5182F780F4205D099F8B62842F0020632
:10DBB00089F8B66809F6AC0B59460E20FBF7CCFC89
:10DBC00059461720FBF7C8FCA948AA4BC9F8F0082A
:10DBD00000241B20C9F8D838C9F8E838C9F8CC485F
:10DBE000C9F8D048C9F8D448C9F8DC48C9F8E048B1
:10DBF000C9F8E448C9F8F408012108F003FA082537
:10DC00009B49C9F8F8182846C9F8FC58012108F0C2
:10DC1000F9F9974FC9F800791A20C9F804090121C8
:10DC200008F0F0F909F6081C4FF0000A9FED926A1F
:10DC3000924E8F49CCF80860072340F2DC52CCF8B2
:10DC400000A0CCF804A01846C9F81449C9F818492E
:10DC5000C9F82019C9F81C29C9F82439012109F685
:10DC6000381B8DED016A08F0CDF99DED010A89F8A8
:10DC70002C49F7EE007A322200234FF07C5709F549
:10DC80001368C8E900230121CBED017ACBED067AB8
:10DC90008BED020ACBF800A0CBF80CA0CBF810A0BB
:10DCA000CBF814700220C9F85449C9F85849C9F88A
:10DCB0005C49CDED027A08F0A5F9284608F096F8FF
:10DCC0009FED6F0A6F4E022008F0A0F8012568480A
:10DCD000C9F86449C9F86009C9F8680902212046F1
:10DCE000C9F86C5908F08EF9022199F86C0908F00E
:10DCF00089F909F5176BDDED020A9DED011ACBF8E4
:10DD000000A009F5196309F51B6109F51D62CBF83F
:10DD10000CA0CBF81870CBF810A0CBF814A0CBED6A
:10DD2000010A8BED021ACBED070A09F6F81CC3F8BD
:10DD300000A0C3F80CA09F61C3F810A0C3F814A002
:10DD4000C3ED010A83ED021AC3ED070A09F6142890
:10DD5000C1F800A0C1F80CA08F61C1F810A0C1F8F3
:10DD600014A0C1ED010A81ED021AC1ED070A09F6FE
:10DD70004C20976109F52367C2F800A0C2F80CA0F7
:10DD8000C2F810A0C2ED010A82ED021AC2F814A076
:10DD9000C2ED070AC9F8F049C9F8F4B9CCF800A0F7
:10DDA000CCF808A0CCF80CA0CCED010A89F8084A00
:10DDB000C9F810BA09F6682CC8F800A0C8F808A07D
:10DDC000C8F80CA0C8ED010A89F8244AC9F82CBA91
:10DDD00009F68428C7F800A0C7F808A0C7F80CA067
:10DDE000C7ED010A89F8404AC9F848BAC0F800A04E
:10DDF000C0F808A0C0F80CA0C0ED010A09F52A601F
:10DE000089F85C4AC9F8643ACCF800A0CCF808A0BC
:10DE1000CCF80CA0CCED010A89F8784AC9F8803A10
:10DE20003768C8F800A0C8F808A0C8F80CA0C8ED6A
:10DE3000010A89F8944AC9F89C3AC0F800A0C0F8D1
:10DE400008A0C0F80CA0C0ED010AC9F8B83A09F65C
:10DE5000BC2309F6D82C09F6F42889F8B04A47F40F
:10DE60000007C3F800A0C3F808A0C3F80CA00BE09B
:10DE7000ACDF0100010000800AD7233C000096437C
:10DE8000C0E164483C800440C3ED010AC9F8D41ADB
:10DE9000B34989F8CC4ACCF800A0CCF808A0CCF85B
:10DEA0000CA0CCED010AC9F8F02A89F8E85AC8F8A4
:10DEB00000A0C8F808A0C8F80CA0C8ED010A89F8AD
:10DEC000045B37600F68A74CA74AA84BDFEDA86A30
:10DED0009FEDA87ADFF8A88227F002004FF4803780
:10DEE0000860C9F80C2B2760906840F00207976023
:10DEF000326842F4000030600E684FF4003226F0C1
:10DF000002070F60C9F8103B226099684EF6602244
:10DF100041F0020009F59E5411EE10CA10EE907AFD
:10DF2000986056461C34AA461A6009F6143E09F653
:10DF30003C30002340F8286C40F824CC40F8207C8A
:10DF400040F81C8C40F818AC40F80C6C40F8086C99
:10DF500040F8143C40F8103C40F8043C02469D1C3C
:10DF6000591C03EE905ADD1C04EE105A02EE901A72
:10DF70001D1D591D01EE903A04EE905A05EE101A3F
:10DF80009D1DD91D05EE905A06EE101AB8EEE13A25
:10DF9000F8EEE27AB8EEC51AF8EEE51AF8EEC62AFF
:10DFA000B8EEE32AB8EEC40AF8EEE40A23EE263A05
:10DFB00062EE263A20EE264A60EEA64A21EE260AB6
:10DFC00061EEA60A22EEA61A27EEA62A63EE071A2B
:10DFD000154663EE872A62EE077A24EE073A64EE6E
:10DFE000873A20EE075A60EE875A21EE076A083317
:10DFF000E5EC011A802BC2ED017AC5ED012A02F190
:10E00000200202ED053A42ED043A02ED035A42EDD8
:10E01000025A02ED016AA2D100F50A70A04288D12D
:10E02000CEF553660C369FED545ADFED543A019607
:10E030004B4609F5336471464FF0000A4FF0FF3547
:10E040004FF08A0808FB0AF6802003F61437F7EE33
:10E05000006AB0EE002A4FF001084FF0000C3FE0DC
:10E0600074EEA30AB4EEE00AF1EE10FAA4BF90EE4B
:10E07000820A0D61013887ED000AD3F8382B013A86
:10E0800002F07F02C3F82C2B84ED005AD3F82C2B1E
:10E09000C3F8285B94ED001A32440EEB820282ED45
:10E0A0000A1AD3F82C2BC3F8382BD1ED001AD1ED76
:10E0B000082A71EEA67AF4EEE72AF1EE10FA37DCC0
:10E0C00032EEA33AF4EEC37AF1EE10FA02DBD3EEAD
:10E0D000027A0D610138C7ED007AC3F828CB31D040
:10E0E000D3F8382B013A02F07F02C3F82C2B84EDD1
:10E0F000005AD3F82C2BC3F8285B94ED007A3244F5
:10E100000EEB820282ED0A7AD3F82C2BC3F8382B5F
:10E1100091ED004AD1ED084A34EE260AF4EEC04AE9
:10E12000F1EE10FA9CDD94EE820AC1F81080A1E7AE
:10E13000D2EE827A0138C1F81080C7ED007AC3F8B8
:10E1400028CBCDD10AF1010ABAF1040F03F50A7305
:10E1500004F50A7416D0019F3944494470E700BFA2
:10E160000070034004E100E00071034010710340BF
:10E1700000F07F450000003C000000000000FC4271
:10E18000C637BE37C14DDFF830A32E68C049DAF874
:10E190000430D1F800C0BF4ADAF8008009F59E5477
:10E1A00041F2C83733430C34BB4E49F807E041F223
:10E1B000CC3E2071CCEB02022B60356849F80E8012
:10E1C00044F201030195C8F80030002A6ED00E46D3
:10E1D000012756F8083FCCEB030C62458E46C1F090
:10E1E0005980AC48C21A1D463846002A5ED00E46F9
:10E1F000022756F8103F5D1BAA42C1F04B80A6468D
:10E20000A44CE21A38461F46002A4ED0451C01EBAA
:10E21000C50651F835309E4CDF1BBA42C1F037803D
:10E220003F2D1F4601F087809A4AD21A2846002ABD
:10E230003BD005F1010C01EBCC0651F83C30DF1B63
:10E24000BA42C1F02480934EF21A60461F4662B370
:10E25000431C01EBC30651F83330DF1BBA42C1F057
:10E2600016808C48C21A1F46A81CF2B105F1030C97
:10E2700001EBCC0651F83C30DF1BBA42C1F00780FD
:10E28000844CE21A1F4660467AB1431C01EBC30678
:10E2900051F833307E4CDF1BBA42C0F0F8877D4C1A
:10E2A000E21A281D1F46002AB0D1744601EBC000B7
:10E2B00043680199794A7A4E41F0625545F4001756
:10E2C0001F43C8F80C700223C8F8006014600022D5
:10E2D00023746261082007F0F9F90021064607F06F
:10E2E00063F870483179E66041F2D035017019F871
:10E2F0000570E3686C4A93F80480DFF8C0E16C268F
:10E3000006FB07AC08F18040DCF8101000F504357E
:10E3100001F03F0747F080034FF000062E702B708E
:10E32000E16815680A68908B87B247F00808A2F880
:10E330001C800A795D4F531102F1100C9E0047F8C2
:10E340002C5006F1604000F5614502F01F030122E8
:10E35000096802FA03F62E608F8BB8B209F59F5850
:10E3600040F002038B83454641F2E4304FF0000158
:10E37000217441F2EC36CEF800404D4949F80010C6
:10E380000C3541F2F43E18231C20C8F8083049F837
:10E390000610686009F5A05649F80E101D21C8F84E
:10E3A0001810C44641F2FC33043604F118081E214B
:10E3B0003F4849F80300B045CCF8201000F08080B9
:10E3C0003C4FC8EB060C5FEA0C713B4653D4114638
:10E3D00098F80400019207F015FE55F8082C00216A
:10E3E0009368404698470A2007F06AFE55F8083CB3
:10E3F00001999A684046904755F8080B04F12008A7
:10E40000036838E098F8040007F0FCFD55F8083C74
:10E4100000219A68404690470A2007F051FE55F8BF
:10E42000080C01218368404608F1080898474645D2
:10E4300005F108054FF0010142D055F8082C13688A
:10E44000BB4240F01F8798F8040007F0DBFD55F849
:10E45000080C00218268404690470A2007F030FEF1
:10E4600055F8081C40468B680121984755F8080B61
:10E47000036808F10808BB424FF00101C2D0012136
:10E4800040469847C2E70446FFF7A7B93C800440DE
:10E49000FC2C0200E0211101142C02002066FF1F59
:10E4A00000003F801A800040081EFF1F0002FF1F6F
:10E4B000ACDF010091090000242C02001066FF1F50
:10E4C00041F2D0356C2619F8057006FB07A2103210
:10E4D00051680A2902F1040300F024879D680A2D7F
:10E4E00002F10C0A00F01F871E690A2E02F1140ABD
:10E4F00000F019879F690A2F02F11C0A00F01387A8
:10E500001D6A0A2D02F1240A00F00D879E6A0A2E68
:10E5100002F12C0A00F007871F6B0A2F02F1340A60
:10E5200000F001879D6B0A2D02F13C0A00F0FB868A
:10E530001E6C0A2E02F1440A00F0F5869F6C0A2F29
:10E5400002F14C0A00F0EF861A6D0A2A03F1500A14
:10E5500000F0E9860020A063092900F0DA869868B7
:10E56000092803F1080E00F0D5861D69092D03F175
:10E57000100E00F0CF869E69092E03F1180E00F0F0
:10E58000C9861F6A092F03F1200E00F0C386986A1E
:10E59000092803F1280E00F0BD861D6B092D03F13B
:10E5A000300E00F0B7869E6B092E03F1380E00F096
:10E5B000B1861F6C092F03F1400E00F0AB86986CFA
:10E5C000092803F1480E00F0A5861D6D092D03F101
:10E5D000500E00F09F860022E263142900F090861E
:10E5E0009D68142D03F1080C00F08B861E69142E13
:10E5F00003F1100C00F085869F69142F03F1180CAD
:10E6000000F07F86186A142803F1200C00F0798648
:10E610009D6A142D03F1280C00F073861E6B142ED6
:10E6200003F1300C00F06D869F6B142F03F1380C52
:10E6300000F06786186C142803F1400C00F0618626
:10E640009D6C142D03F1480C00F05B861E6D142E9A
:10E6500003F1500C00F0558600222264152900F0C9
:10E6600046869E68152E03F1080800F041861F6952
:10E67000152F03F1100800F03B869869152803F167
:10E68000180800F035861D6A152D03F1200800F0EA
:10E690002F869E6A152E03F1280800F029861F6B2D
:10E6A000152F03F1300800F02386986B152803F12D
:10E6B000380800F01D861D6C152D03F1400800F090
:10E6C00017869E6C152E03F1480800F011861F6D09
:10E6D000152F03F1500800F00B86002262640A290E
:10E6E00000F0FC859F680A2F03F1080A00F0F78507
:10E6F00018690A2803F1100A00F0F1859D690A2DB6
:10E7000003F1180A00F0EB851E6A0A2E03F1200AB5
:10E7100000F0E5859F6A0A2F03F1280A00F0DF85E3
:10E72000186B0A2803F1300A00F0D9859D6B0A2D79
:10E7300003F1380A00F0D3851E6C0A2E03F1400A5B
:10E7400000F0CD859F6C0A2F03F1480A00F0C785C1
:10E75000186D0A2803F1500A00F0C1850022A26456
:10E76000092900F0B2859868092803F1080E00F025
:10E77000AD851D69092D03F1100E00F0A7859E6976
:10E78000092E03F1180E00F0A1851F6A092F03F16D
:10E79000200E00F09B85986A092803F1280E00F0EE
:10E7A00095851D6B092D03F1300E00F08F859E6B52
:10E7B000092E03F1380E00F089851F6C092F03F133
:10E7C000400E00F08385986C092803F1480E00F094
:10E7D0007D851D6D092D03F1500E00F07785002217
:10E7E000E264142900F068859D68142D03F1080C7B
:10E7F00000F063851E69142E03F1100C00F05D8596
:10E800009F69142F03F1180C00F05785186A14281B
:10E8100003F1200C00F051859D6A142D03F1280CA2
:10E8200000F04B851E6B142E03F1300C00F0458573
:10E830009F6B142F03F1380C00F03F85186C1428DF
:10E8400003F1400C00F039859D6C142D03F1480C48
:10E8500000F033851E6D142E03F1500C00F02D8551
:10E8600000222265152900F020859E68152E03F1EF
:10E87000080100F019851A69152A03F1100100F04A
:10E8800013859F69152F03F1180100F00D85186A93
:10E89000152803F1200100F007859D6A152D03F16D
:10E8A000280100F001851E6B152E03F1300100F0E8
:10E8B000FB849A6B152A03F1380100F0F5841F6C74
:10E8C000152F03F1400100F0EF84986C152803F137
:10E8D000480100F0E9841D6D152D03F1500300F08F
:10E8E000E48409F5A25E09F5A35C09F5A15A009834
:10E8F00060654FF000084FF07E5509F59E544FF0CB
:10E900007C53514FCAF80850CAF81C50CAF80C7012
:10E91000CAF81830CAF80480CAF81080CAF81480FF
:10E9200004F58A70CEF80450CEF80870CEF8143092
:10E93000CEF81850CEF82050CEF82470CEF83030F3
:10E94000CEF83450CEF80080CEF80C80CEF810808F
:10E95000CEF81C80CEF82880CEF82C800021CCF890
:10E960002070CCF81C50CCF82C30CCF83050CCF8BF
:10E970001880CCF82480CCF828804FF400620BF08B
:10E98000CDFC0020C4F81409C4F81809C4F81C0907
:10E99000C4F8200909F5E75A09F5E85C41F6F8479B
:10E9A00041F6085604F1640341F6E84541F618546F
:10E9B000142049F80500CAF80C80CAF8108049F8FC
:10E9C0000700CAF81C80CAF8208049F80600CCF875
:10E9D0000C80CCF8108049F8040009F5A4501430DC
:10E9E00009F5A551DFF870E0184E194C194FCCF815
:10E9F0001C808342CCF82080C1F81080C1F81C80B4
:10EA0000C1F82080C1F814E08F614E628C62C0F8BA
:10EA10000080C0F804E08760C0F80C80C0F8108067
:10EA2000466184611AD032462546C3F80080C3F897
:10EA300004E09F60C3F80C80C3F810805A619D61A8
:10EA40001C339842F1D109E00AD7233CA4707D3FE2
:10EA5000D3A0803F0000204100F07F4509F5E95533
:10EA6000083541F6285A0124002749F80A7005F1B3
:10EA700008006C6039464FF4F0620BF04FFC2C62DA
:10EA80006C62AC62C5F89040C5F89440C5F8A440EB
:10EA9000C5F8A840C5F80441C5F82441C5F8784137
:10EAA000C5F8A041C5F8F041C5F81842C5F8644260
:10EAB000C5F89442C5F8D842C5F81043C5F850438C
:10EAC000C5F88843C5F80444C5F83C44C5F87C44FF
:10EAD000C5F8B444C5F8F844C5F82845C5F87445E8
:10EAE000C5F89C45C5F8EC45C5F81446C5F8684618
:10EAF000C5F88846C5F8E44605F5F160C5F8E8466E
:10EB00003946C5F8F846C5F8FC46C5F86447C5F867
:10EB10006847C5F86C474FF4F0620BF0FFFBC5F88F
:10EB20009447C5F89847C5F8D047C5F80848C5F8D0
:10EB30001448C5F84448C5F84C48C5F88048C5F89D
:10EB40008C48C5F8B848C5F8C848C5F8F448C5F8B1
:10EB50000849C5F83049C5F84049C5F86C49C5F8B9
:10EB60008049C5F8A449C5F8BC49C5F8E449C5F8C9
:10EB7000F849C5F81C4AC5F8344AC5F8584AC5F8DA
:10EB8000744AC5F8944AC5F8AC4AC5F8D04AC5F8E5
:10EB9000EC4AC5F80C4BC5F8284BC5F8644B05F694
:10EBA0000870C5F8804B3946C5F8A04BC5F8BC4B7A
:10EBB000C5F8E04BC5F8F84BC5F8184CC5F8344C0F
:10EBC000C5F8584CC5F8704CC5F8944CC5F8A84C1D
:10EBD000C5F8D04CC5F8E84CC5F80C4DC5F8204D2B
:10EBE000C5F84C4DC5F85C4DC5F8844DC5F8984D39
:10EBF000C5F8C44DC5F8D44DC5F8004EC5F80C4E47
:10EC0000C5F8404EC5F8484EC5F8784EC5F8844E54
:10EC1000C5F8BC4EC5F8F44EC5F8F84E4FF4F06296
:10EC20000BF07CFB41F22C0641F2040C41F2240E65
:10EC300041F24C0009F550521832C5F8104FC5F892
:10EC4000384FC5F8604FC5F8844FC5F88C4FC5F8EC
:10EC5000AC4FC5F8B44FC5F8D44FC5F8DC4FC5F874
:10EC6000FC4F41F2540845F80C40009245F80E4024
:10EC700041F2740AAC5141F27C012C5041F29C02E9
:10EC800041F2A40C41F2C40E41F2CC0641F2E8007C
:10EC900045F8084045F80A4041F2F8086C5041F246
:10ECA000101AAC5041F2701145F80C4041F2881234
:10ECB00045F80E4005F5895CAC5141F2381E2C50E8
:10ECC00041F2481605F58B5045F8084045F80A40D2
:10ECD00009F53B58CCF8004041F2B01A45F80E4017
:10ECE00041F2102CAC5141F2282E046005F58E56ED
:10ECF0006C5009F53C50AC5041F2E81105F59052CA
:10ED0000C8F8004045F80A4041F23828346041F222
:10ED1000502A046041F2B0266C5041F2DC201460AD
:10ED200005F5935145F80C4041F2782245F80E4024
:10ED300041F2882C05F5955E45F8084045F80A40F3
:10ED400041F2EC280C6041F2043AAC5041F26431DB
:10ED500045F80C4041F27C32CEF8004041F2143CC0
:10ED6000AC5141F22C3E2C5041F23C3641F2543031
:10ED700045F8084045F80A4041F28C3845F80C4007
:10ED800041F2A43A45F80E4041F2044CAC5141F234
:10ED90001C4E2C5041F2B4366C5041F2CC30AC5089
:10EDA00041F2DC3141F2F43245F8084045F80A40BE
:10EDB00041F22C48AC5141F2444A2C5041F2A44655
:10EDC0006C5005F5A650AC5041F2544145F80C404A
:10EDD00041F26C4245F80E4041F27C4C41F2944EB7
:10EDE00045F8084045F80A4041F2C8486C5041F2E5
:10EDF000E84AAC5005F5AA5145F80C4005F5AB5270
:10EE000045F80E4041F2F04CAC5141F2105E046006
:10EE100009F5495641F2385045F8084045F80A408E
:10EE200041F2685845F80C4041F2885A45F80E40C6
:10EE300034602C5041F290560C6041F2B050146096
:10EE400041F2B85109F54C5205F5AF5C45F8084060
:10EE500009F54E5345F80A4005F5B05EAC5141F254
:10EE600008682C5041F22C6A6C5041F254601460D6
:10EE700041F27C6143F2B032CCF8004043F21846D4
:10EE800043F2144CCEF8004045F8084045F80A40DB
:10EE90002C506C5049F802B01F6783F8747083F8E7
:10EEA0007570C3F88C7083F89070AB4B09F80C70D8
:10EEB00009F80670009D58686F70A74906689B683E
:10EEC0000968A64A6A6009F5505E0EF1200C43F20B
:10EED000204A3343A24D49F80A508CF804708CF84C
:10EEE0000C708CF80D70CCF81070CEF87470CEF8F1
:10EEF00078700360CCF808100F70DCF80800994EA9
:10EF00004770DCF80830984D9F70DCF80810FF223D
:10EF1000CA70DCF808004771DCF80830502199719C
:10EF2000DCF80820D771DCF8080090F802B00BF08C
:10EF30007F038370DCF808100098019409F5505E97
:10EF40000EF1140B083012220BF104030290CA7068
:10EF5000BE46B84603934FF0FF30844ABC400021C0
:10EF600098E0CAF5C333A033834202D21846B846AC
:10EF70008E46538804FB03F3B6FBF3FAAA4501F16E
:10EF8000010100F29D80CAF5C333A033834202D24F
:10EF90001846B8468E46938804FB03F3B6FBF3F39A
:10EFA000AB4201F1010A40F29780A3F5C333A03BC5
:10EFB000834205D2D646B846002B00F0D9801846C9
:10EFC000D38804FB03F3B6FBF3F3AB4201F1020A6F
:10EFD00040F28C80A3F5C333A03B834205D2D646D2
:10EFE000B846002B00F0C4801846138904FB03F3D5
:10EFF000B6FBF3F3AB4201F1030A40F28180A3F5C3
:10F00000C333A03B834205D2D646B846002B00F05E
:10F01000AF801846538904FB03F3B6FBF3F3AB420E
:10F0200001F1040A75D9A3F5C333A03B834205D28D
:10F03000D646B846002B00F09B801846938904FB07
:10F0400003F3B6FBF3F3AB4201F1050A6AD9A3F56A
:10F05000C333A03B834205D2D646B846002B00F00E
:10F0600087801846D38904FB03F3B6FBF3F3AB4266
:10F0700002F10E0201F1060A5DD9A3F5C333A03BEC
:10F08000834204D2D646B846002B71D018460731C9
:10F0900040295BD0538804FB03F3B6FBF3FAAA457F
:10F0A00002F102027FF65DAFAAF5C333A03B8342B3
:10F0B000BFF45FAFB8468E46002B59D0184658E7CC
:10F0C000AAF5C333A03B8342BFF465AFB8468E4672
:10F0D000002B4DD018465EE7C3F5C333A0338342FF
:10F0E000BFF46EAFD6461846B84669E7C3F5C333DA
:10F0F000A0338342BFF479AFD6461846B84674E7CA
:10F10000C3F5C333A033834284D2D6461846B846EB
:10F1100080E7C3F5C333A03383428FD2D646184667
:10F12000B8468BE7C3F5C333A03383429AD2D646A1
:10F130001846B84696E7C3F5C333A0338342A6D238
:10F1400007314029D6461846B846A3D1022F0FD022
:10F150000137019C01E700BF4C2B0200A50900000C
:10F16000C4DF0100008793039F860100922B0200F9
:10F1700043F228410EF03F0259F8013042EA88106C
:10F18000C5B25D70DCF80860777947F020047471CF
:10F19000DCF80820507940F080035371DCF8085007
:10F1A000684AAE7846F08007AF709CF804A00AEB7E
:10F1B0004A0402EBC40E0120DEF80C305D09AE00FB
:10F1C00006F1604808F5614703F01F0400FA04F2F5
:10F1D0003A605D4D009F029E2E60002387F86830E4
:10F1E000DCF80840A37000BFDCF80820574E584DEB
:10F1F000584CC5F800B080279770DCF80820564DB1
:10F20000137059F8017097F802A04AF04002BA70E2
:10F2100059F801700399316002268CF80D6097F857
:10F22000068009F5525C624609F55B5643F2304AA6
:10F23000083248F007010CF13C0E043643F28848CE
:10F24000B97149F80A5043F6CC0743F6D0058BF85C
:10F2500070308BF871308BF872304FF0FF3149F815
:10F2600008301372D360137453748EF8040286F856
:10F270000402484649F80710226049F8051007B013
:10F28000BDE8F08F012140469847FFF7E0B875468A
:10F29000A6462C46314F1F44BA4296BF0EEBC00023
:10F2A00073684368FFF705B80B461E7906F03F0206
:10F2B00017040097FFF715BB9C469CF8047007F0F5
:10F2C0003F0005042565FFF7CDBA9E469EF8046011
:10F2D00006F03F073804E064FFF783BA9A469AF8CD
:10F2E000045005F03F063704A764FFF739BA984683
:10F2F00098F8040000F03F052E046664FFF7EFB9AC
:10F300009C469CF8047007F03F0005042564FFF755
:10F31000A5B99E469EF8046006F03F073804E063F6
:10F32000FFF75BB99A469AF8045005F03F06370498
:10F33000A763FFF711B97146A6460C46DEF8FC310B
:10F34000FEF7B7BF4C2B0200EC65FF1FE063FF1F09
:10F35000C02AFF1F0066FF1FA5B0000020DEEEFEE2
:10F360004FF4FA6202FB00F007EE900AB8EE677AFB
:10F37000F7EE006A86EE870A0E4BD3F80C1B70B4CA
:10F3800041F2C8368D689B590B4CB4FBF0F025F068
:10F3900001028A6003F50A64086083ED030A03F53D
:10F3A0000A739C42F9D18E6846F001058D6070BCED
:10F3B000704700BFF82AFF1F008793032DE9F04F25
:10F3C000203A8DB0D3B26B2B099000F26882B2481C
:10F3D00050F8230090F800E0B04EB14CB368B26A28
:10F3E000D6F820B00593099BF569776A08902668DE
:10F3F0000BEB020000245A1C0233069007942F44A2
:10F4000001F1020801F1010C0A920B9310461C460F
:10F41000099A02970023019604914EFA03F111F024
:10F42000010F27D0019E954206EB002706EB02292B
:10F43000039706EB042A3CDDA54240F3D2808542C7
:10F4400018DC0299814215DD049EB34503DC069960
:10F45000B14200F39682E34503DC069E664500F365
:10F460006982D84506DB069EB04503DA039F0599FD
:10F4700047F828100133062B02F1030200F10300C4
:10F4800004F10304C9D107980499029F019E013039
:10F490000828079008F1030801F103010CF1030C9F
:10F4A00000F0E081089C0A9814F801EF08940B9C86
:10F4B000AEE702998C424EDBAC4280F2F38085428B
:10F4C00000F3A680914240F3DE81049FBB45BA461B
:10F4D00026DC0699B94223DD029E059F49F82A7071
:10F4E000864227DD039E049F059946F8271002995E
:10F4F00091421FDC0299814240F3C181E34540F310
:10F500006B82029E9642ACDDD845B3DB069FB845C0
:10F51000B0DA029E059949F828108642A6DCA9E7D0
:10F52000029F874206DD049EB34540F3B3810299F2
:10F530009142DFDDE345DDDC069E6645DADD029EB5
:10F54000059949F82C10864240F32B820399059FB8
:10F5500041F82C70D5E7AC4276DA854258DC91420E
:10F5600040F38A81049FBB45BA461FDC0699B94225
:10F570001CDD029E059F49F82A70864220DD039E0D
:10F58000049F059946F827100299914218DC0299C8
:10F59000814240F37481E34540F30F82029E96421C
:10F5A0007FF75FAFD845FFF665AFAFE7029F8742B1
:10F5B00006DD049EB34540F3058202999142E6DDE3
:10F5C000E345E4DC069E6645E1DD029E059949F8C7
:10F5D0002C10864240F3DE810399059F41F82C7080
:10F5E000DCE7029EA64200F3AC8085423FF742AFC3
:10F5F00086427FF73FAF049FBB453FF72CAF06998C
:10F60000B9427FF728AF039E059946F8271022E7F5
:10F6100091427FF72FAF049FBB45BA4603DC0699A2
:10F62000B94200F34481E34503DC069E664500F3DE
:10F630003A81D845FFF61EAF069FB845BFF61AAF10
:10F64000059949F8281015E7814200F3B4809142EA
:10F6500040F3D380049FBB4540F33781E3450BDC87
:10F66000069F674508DD059E49F82C60029F0599B5
:10F670004AF82C10974273DDD845FFF6FBAE069E84
:10F68000B045BFF6F7AE059949F82810D14605995F
:10F6900049F82810EEE600BF00290200C42AFF1F27
:10F6A000D063FF1FA842B3DB914240F3DE80049F8A
:10F6B000BB45BA462ADC0699B94227DD029E059F62
:10F6C00049F82A70B0422BDA039E049F059946F848
:10F6D00027100299914223DC0299884280F2C88067
:10F6E000E34540F37481029E96427FF7BAAED84557
:10F6F000FFF6C0AE069FB845BFF6BCAE029E0599A8
:10F7000049F82810B042FFF6B1AEB3E6029FB84206
:10F7100006DA049EB34540F34B8102999142DBDD4A
:10F72000E345D9DC069E6645D6DD029E059949F87B
:10F730002C10B04280F22A810399059F41F82C7069
:10F74000D1E7854215DD049EB34503DC069FB74231
:10F7500000F30F81E34503DC069E664500F30D814F
:10F76000D845FFF687AE069EB045BFF683AED146BC
:10F770008DE7864255DD049FBB4540F3B680E345E7
:10F7800037DC069E664534DD0399059F41F82C70F1
:10F790000299059F4AF82C708142E1DDD845FFF6B9
:10F7A00069AE069EB045BFF665AE0399059F41F868
:10F7B0002870D1466BE7914203DD049EB34540F3C8
:10F7C000AF80854245DC049EB34540F3C480029E71
:10F7D000964202DDE34540F39980854233DCE34500
:10F7E00040F3AD800299914201DDD84563DA85424C
:10F7F000B6DCD845FFF63EAED3E7049EB34509DC40
:10F80000069FB74206DD059F4AF82670029E964283
:10F810003FF724AFE345A3DC069961453FF726AFE8
:10F820009EE7049FBB4508DC0699B94205DD059EAD
:10F830004AF82760029F8742A1DCE34590DC0699E5
:10F840006145A5DC8CE7E345CCDC069F67457EDCA3
:10F85000C8E7049FBB45BADC069F049EB74200F38D
:10F860008480B4E70DB0BDE8F08F8842FFF651AF59
:10F8700091427FF7FFAD3AE781423FF79AAE91425E
:10F880007FF7F8AD40E681423FF74DAE91427FF7FA
:10F89000F1AD39E60699B1427FF749AE22E651480B
:10F8A0004FF0000E98E5059949F82C10C1E6059F28
:10F8B00049F82A70B7E6069EB04598DA059F49F8E0
:10F8C000287085427FF771AF4DE70699B9427FF7FF
:10F8D000C5AE3E46059949F82710059F4AF826709F
:10F8E000029E96423FF7BAAE94E70699B9427FF777
:10F8F00046AF039E0599B146059E49F827104AF880
:10F900002760029F87423FF73AAF96E7069F674519
:10F910007FF763AF059E49F82C60854213DD94E7BD
:10F920000699B1427FF74DAF059949F826108542F7
:10F9300015DD91E7039F059947F82C1091E506998D
:10F9400061457FF74FAF039E059946F82C10059F40
:10F950004AF82C7046E7069FB7427FF738AF039E00
:10F96000049F059946F827103E4605994AF8261047
:10F970002DE7059F4AF82670ECE6059F4AF82C70A3
:10F98000EEE6BA4605994AF8261064E596423FF736
:10F99000AEAE6FE596423FF7B7AD86423FF761AD39
:10F9A00068E596423FF7B0AD86427FF763AD58E514
:10F9B0000699B1427FF7B1AE86E6069F67457FF7AD
:10F9C000EDAD09E60699B1427FF7F7ADD7E5069FA1
:10F9D00067457FF788AEAFE6069F67457FF791AD35
:10F9E000B4E500BFA82502002DE9F04F203AD3B2BC
:10F9F0006B2B85B000F28180434C54F8232017789C
:10FA0000424BDFF810E19C6ADE695D6AD3F8208022
:10FA10009B6802939246DEF800300393421C08EB89
:10FA2000040B06EB050E01F1010C4FF000090192E9
:10FA300014460246002300903CE0724509DA414535
:10FA400007DB594505DA039D029805EB022545F8C9
:10FA50002100B44254DBA64549DD414507DB594549
:10FA600005DA039D029805EB042545F8210096422E
:10FA70000FDC72450BDAE04507DCE34505DD039D4D
:10FA8000029805EB022545F82C00A6420BDCA645A2
:10FA900009DDE04507DCE34505DD039D029805EB44
:10FAA000042545F82C000133062B04F1020402F171
:10FAB00002020ED047FA03F0C007F4D59642BCDD2F
:10FAC000A642C8DD0133062B04F1020402F1020252
:10FAD000F0D109F10209B9F1100F00980CF1020CF4
:10FAE00001F1020106D01AF8017F019CA1E79642BC
:10FAF000BFDDD8E705B0BDE8F08F054A00277FE7F6
:10FB00007245B8DBCFE700BF00290200C42AFF1FFF
:10FB1000A8250200D063FF1F203AD2B22DE9F04F92
:10FB20006B2A96BF8A4B8B4A53F822208A4B8B4F05
:10FB30001B68FC697D6A3E6AD7F828B0BF688BB045
:10FB4000013A019200F1010903EB002200F10208E1
:10FB5000049203EB092200F1030C059203EB082247
:10FB6000039700F1040E471D069203EB0C22B344E9
:10FB7000079203EB0E2203EB072308922544019A18
:10FB8000099301F1080ACDF808B001905378D8071D
:10FB900002F1010207D50198A04204DBA84202DA73
:10FBA0008E4240F3CB80980706D54C4504DC4D458A
:10FBB00002DD8E4240F3B880580706D5444504DC88
:10FBC000454502DD8E4240F3A580180706D5644501
:10FBD00004DC654502DD8E4240F39280D80605D5EF
:10FBE000744503DC754501DD8E427FDD9B0605D53E
:10FBF000BC4203DCBD4201DD8E426FDD5378D80785
:10FC000001F1010102F1010206D50198A04203DBD6
:10FC1000A84201DA8E4258DD980705D54C4503DC31
:10FC20004D4501DD8E4247DD580705D5444503DCCF
:10FC3000454501DD8E4236DD180705D5644503DCF8
:10FC4000654501DD8E4225DDD80605D5744503DC0A
:10FC5000754501DD8E4214DD9B060CD5BC420ADCE5
:10FC6000BD4208DD8E4206DC029B8B4203DD099813
:10FC7000039B40F8213001318A4587D10BB0BDE8A4
:10FC8000F08F02988842E7DD0898834603984BF886
:10FC90002100E1E702988842D6DD07988346039861
:10FCA0004BF82100D0E702988842C5DD06988346CC
:10FCB00003984BF82100BFE702988842B4DD05980D
:10FCC000834603984BF82100AEE702988842A3DDF3
:10FCD0000498834603984BF821009DE7029B8B42D2
:10FCE0008CDD0998039B40F8213087E70298884211
:10FCF0007FF77CAF0898834603984BF8210075E79F
:10FD0000029888427FF76AAF0798834603984BF8BA
:10FD1000210063E7029888427FF757AF0698834631
:10FD200003984BF8210050E7029888427FF744AFD0
:10FD30000598834603984BF821003DE702988842D6
:10FD40007FF731AF0498834603984BF821002AE7E8
:10FD500000290200A8250200D063FF1FC42AFF1F4C
:10FD60002DE9F04F9E4FD7F83080D7F800A07C687F
:10FD7000B8F1000F8DB0054640F3D980B8F1030FFC
:10FD800055DC28460AF03CFB2B78002B58D0002885
:10FD90004FF00006B8BF6FF00040B446691E4FF048
:10FDA000010E11F8012F32B990B911F8012F4FF05F
:10FDB000FF30002AF8D00A2A03D01F2AF1D90636CC
:10FDC000EFE7B445B8BFB4460EF1010E0026E8E7F0
:10FDD000F96A01F1080966450EFB09FBD7F80C909A
:10FDE000B8BF664608FB06F6B9F1010F039608FB9B
:10FDF0000BF02DD0B9F1020F04BF039EC6EB0A0A27
:10FE00003E69012E2CD0022E08BF241AFA697E6AA0
:10FE100004929619B2451146DFF8C4E104DA039A58
:10FE20000AEB020C614520DB0DB0BDE8F08F032327
:10FE300028463B6398460AF0E3FA2B78002BA6D1BC
:10FE4000D7F80C900393B9F1010F4FEAC800D1D154
:10FE5000039A3E6902EBD271012EAAEB610AD2D15C
:10FE600000EBD07BA4EB6B04D0E7DEF82020DEF8BB
:10FE70002810069211448C42D6DA20448242D3DA0A
:10FE8000002BD1D0DEF82C209EF814000790083209
:10FE900008FB02F20592A2EBC8001A464B1E0A9319
:10FEA000059BCDF824A0013E1C44C11A0B96089175
:10FEB000CDF81490A2469B460A2ACBEB0A012E46A7
:10FEC00000F08C801346002001E00A2B6FD01F2B1E
:10FED00016F8013F88BF0130002BF6D100EB40003F
:10FEE00044000598012808FB04F36AD0022870D06A
:10FEF000099C079858BB0899B8F1020F01EB0A0951
:10FF000019D0B8F1030F46D142B909E0204649465D
:10FF1000FFF754FA15F8012F12340AB10A2AF5D165
:10FF20003278DA44002A3FF47FAF3546C4E7012037
:10FF30003863804625E7002AF2D00A2AF0D020460E
:10FF40004946FFF751FD0C3415F8012FF3E7B86966
:10FF5000009023440B985A1E8242A8BF024606987E
:10FF60008142B8BF01460A980AF1FF338342A8BF15
:10FF700003460498A042B8BF2046FBF705FF089A45
:10FF8000B8F1020F02EB0A092A78D4D0B8F1030FB6
:10FF9000BAD0002AC4D00A2AC2D020464946FFF768
:10FFA000BBFD15F8012F0634002AF4D1B8E700EBA9
:10FFB0004004630008FB03F30598012806F10106DD
:10FFC00094D1039CE01A099C00EBD07904EB6904FE
:10FFD0008FE7039C0998E41A04448AE70023EBE7BF
:10FFE000C42AFF1F0FB410B582B004AB074C53F8FE
:10FFF000042B0193402120460AF0AAFA2046FFF77D
:020000021000EC
:10000000AFFE02B0BDE8104004B070477C2AFF1F6D
:100010002DE9F04F15785669C34F8FB004469069AB
:100020000692002DC14AC24D049118BF0646606871
:10003000A86098464FF0020018BF174638210123E8
:10004000042EE86069602B6300F0EF81069DDFF805
:10005000EC9205F1340B4FF0000A1E25DBED000A8F
:10006000B348BDEEE01A5645056011EE101AB148CE
:1000700000F06E81FFF7B6FF0AF1010ABAF1040F32
:1000800005F11F050BF1040BE8D1A94EAA48002782
:10009000F7603760FFF764FE069D95F8589095F875
:1000A000D220CDF820904846079220B995F8597093
:1000B000002F00F06C81079E012E00F0EA819F4D19
:1000C000079928680A900A9BC3F30802B2F5807F5B
:1000D00094BF4FF0000B4FF0010B069882468A4404
:1000E0009AF8D0700997022F00F08C81B8F80A6056
:1000F0009FED936A01EE906AB8EE612AF7EE006A0E
:1001000082EE067AB4EEE67AF1EE10FA00F1C481DE
:100110004FF00B0A4FF00A094FF0090C0821062096
:10012000052604274FF0030E0723B8F80C80854DF1
:10013000DFED834A2A68656842F8235004EE108A8E
:10014000B8EE445A02EB8E0E6568CEF80051C5EE4B
:10015000245A02EB87076568C7F8005102EB860650
:100160006768C6F8007102EB80006568C0F800514E
:1001700002EB83036668C3F8006102EB81016768E4
:10018000C1F8007102EB8C0C6068CCF8000102EB46
:1001900089096568C9F80051F7EE007A02EB8A0A0E
:1001A000F4EEE75A6368CAF80031F1EE10FA00F194
:1001B00093814FF00B0A4FF00A094FF0090808200D
:1001C000062605274FF0040E4FF0030C072102EB23
:1001D000810101F5FE4365681D6002F5FC43656819
:1001E00043F82C50656843F82E50656843F8275053
:1001F000676843F8267001F5FC4C6668CCF800602F
:10020000616843F82010606843F82800656843F887
:100210002950676843F82A70BBF1000F00F0CD80C9
:10022000049BDFED471AD3F80C699FED476A9FEDF9
:10023000472A033602F5407302F5FA420592F7EEBB
:10024000006A039629E0606843F82B00606843F871
:100250002A00606843F82900606843F82800606855
:1002600043F82200626843F82120616843F82C10AB
:10027000606843F82E00626843F82720676843F8F7
:100280002670666843F825600599039D03F5807321
:1002900001359942039500F090800399049D01F087
:1002A0007F0005EB800B9BED437AFCEEC72A0C2503
:1002B000B8EE623A0B26C3EE213A0A274FF0090E38
:1002C0004FF0080C072106224FF005084FF00409F3
:1002D0004FF0030A4FF0020BF4EEE63AF1EE10FA9B
:1002E000B1D5F5EEC03AF1EE10FA54DDB0EE424A67
:1002F000A3EE864AFCEEC44A14EE900A14EE901A5D
:1003000000EB0B0E00EB0A0700EB090600EB0805FB
:1003100000F1010CA0F1050BA0F1040AA0F1030902
:10032000A0F10208421E8EE750240200542402006D
:10033000C42AFF1F582402005C2402002C66FF1F01
:1003400000F07F45D063FF1F000024C20000404240
:10035000FFF748FED9F800300C930C99C1F308025E
:10036000B2F5807F38460AD8D9F80030069A0B9348
:100370000B99536DC91AB1F5C87FBFF47DAE754AAC
:100380007449136805330B60FFF7EAFC74E64FF01D
:10039000010B0799A1E63525342633274FF0320E9D
:1003A0004FF0310C30212F224FF02E084FF02D0945
:1003B0004FF02C0A4FF02B0B45E7089818B9069A16
:1003C00092F85970DFB1079E012E18D0624B256854
:1003D00019680D910D98C0F30802FF2A98BF65684F
:1003E000099C002C74D0012C00F0938000275B48FE
:1003F0003E46584B1E605F609D60FFF7B1FC0FB03A
:10040000BDE8F08F049F00265D4681463146019588
:10041000CDF8009043463A4620460136FBF71CFDD6
:10042000042EF3D10FB0BDE8F08F069A4A4E02F1C8
:10043000340B4FF01E0ADC465546B1469346E24661
:10044000FAEC017A434946480D60BDEEE70A1F35D4
:1004500010EE101AFFF7C6FD30680C900C9BC3F32A
:100460000802B2F5807F384609D8D9F800100B9100
:100470000B9BDBF85420991AB1F5C87F06D2354B97
:10048000344A196805311160FFF76AFC9A2DD7D1FB
:10049000FBE5B346314620E6B5EEC07AF1EE10FA40
:1004A0003BDDDFED302A9FED303AA7EE223AFCEE3D
:1004B000C33A13EE903AA3F1040EDF1E9E1E581E9F
:1004C000591C03F1020C03F1030903F1040A2CE6A1
:1004D0002648032776268CE7F5EEC05AF1EE10FA8F
:1004E00029DD9FED200ADFED200AE5EE800ABCEE53
:1004F000E01A11EE101AA1F1040CA1F1030E8F1EE7
:100500004E1E481C01F1020801F1030901F1040A21
:100510005DE603273E4616486BE74FF0340A4FF07E
:1005200033094FF0320C31212F202E262D274FF08A
:100530002C0E3023F9E54FF0340A4FF033094FF019
:10054000320831202F262E274FF02D0E4FF02C0C85
:1005500030213CE6C42AFF1F2C66FF1F64340200D2
:1005600058240200000024C2000040424824020037
:100570004C2402002DE9804800F5E95785B03E463D
:100580000446DFF8E881764D0192894608370C363B
:1005900000F5FC7A02E0012005F092FDD4F8F83174
:1005A00093F864100029F6D14FF40042D8F8000007
:1005B00009F0B4FED8F800E03A6831680EF5FC4B5B
:1005C0000BF1580B0EF5567C0CF1480063465A604F
:1005D0009A60DA601A615A619A61DA611A6243F8C4
:1005E000242F8342F3D10CF5807CE345ECD10EF54A
:1005F000157B0EF52972CBF80410CBF80810CBF858
:100600000C10CBF81010CBF81410CBF81810CBF856
:100610001C10CBF82010CBF824104BF8281F5A459B
:10062000E9D1CEF858120EF5FA40CEF85813CEF8AC
:1006300058140EF5A063CEF85815CEF85816C3F826
:100640005817C3F85818C3F85819C3F85812C3F804
:100650005813C3F85814C3F85815C3F8581603F5BF
:1006600000639842EBD10EF5FC430EF5FD42543386
:10067000243259609960D960196159619961D961D1
:100680001962596243F8281F9342F2D1CEEB000C55
:100690000EF58073ACF5807B9842CEF8A412CBF3B4
:1006A00002223ED04AB3012A21D0022A1BD0032ABB
:1006B00015D0042A0FD0052A09D0062A1CBFC3F87A
:1006C000A41203F5807303F58073C3F8A411C3F873
:1006D000A41203F58073C3F8A41203F58073C3F862
:1006E000A41203F58073C3F8A41203F58073C3F852
:1006F000A41203F58073984213D0C3F8A417C3F86B
:10070000A418C3F8A419C3F8A412C3F8A413C3F817
:10071000A414C3F8A415C3F8A41603F50063984203
:10072000EBD1104908680390039BC3F3080E002225
:1007300001233F201821BEF5807F2A6185E8030050
:10074000EB602B6302D94846FFF70AFB212201998F
:1007500005486A60FFF746FC5046F6F75FFB1AE76C
:10076000C42AFF1F2C66FF1F60240200D063FF1FF6
:100770000EB42DE9F04F82B00BAB044604F5E957F7
:1007800053F8042B764800933E46402109F0E0FEE2
:10079000DFF8D481DFF8D4A1724D08370C3604F5A8
:1007A000FC7902E0012005F08BFCD4F8F83193F8D5
:1007B00064100029F6D14FF40042D8F8000009F087
:1007C000ADFDD8F800E03A6831680EF5FC4B0BF14E
:1007D000580B0EF5567C0CF1480063465A609A603F
:1007E000DA601A615A619A61DA611A6243F8242F59
:1007F0008342F3D10CF5807CE345ECD10EF5157BFB
:100800000EF52972CBF80410CBF80810CBF80C10B9
:10081000CBF81010CBF81410CBF81810CBF81C1034
:10082000CBF82010CBF824104BF8281F5A45E9D1FB
:10083000CEF858120EF5FA40CEF85813CEF85814E8
:100840000EF5A063CEF85815CEF85816C3F8581711
:10085000C3F85818C3F85819C3F85812C3F85813F6
:10086000C3F85814C3F85815C3F8581603F50063B5
:100870009842EBD10EF5FC430EF5FD425433243281
:1008800059609960D960196159619961D96119629A
:10089000596243F8281F9342F2D1CEEB000C0EF5BB
:1008A0008073ACF5807B9842CEF8A412CBF3022281
:1008B0003ED04AB3012A21D0022A1BD0032A15D0E8
:1008C000042A0FD0052A09D0062A1CBFC3F8A41297
:1008D00003F5807303F58073C3F8A411C3F8A41261
:1008E00003F58073C3F8A41203F58073C3F8A41250
:1008F00003F58073C3F8A41203F58073C3F8A41240
:1009000003F58073984213D0C3F8A417C3F8A41852
:10091000C3F8A419C3F8A412C3F8A413C3F8A41409
:10092000C3F8A415C3F8A41603F500639842EBD1ED
:10093000DAF8001001910198C0F30802B2F5807F47
:100940000AD901233F2120220548EB6085E80600F3
:100950002B612B63FFF704FA4846F6F75FFA21E7AD
:100960003C2AFF1FC42AFF1FD063FF1F2C66FF1FF6
:100970002DE9F04F924D934A934E8FB02B46182796
:100980001E211C241D20AB420D91069208920A9252
:100990000C92079709940B900DEB07080DF13009A5
:1009A0004FF0020117D198F8040005F02BFBD8F89E
:1009B0000030DA68B24215D198F8040005F014FB53
:1009C000A0B1C14500F0D88058F8087F3B68AB4221
:1009D0004FF00201E7D040469847D8F80030DA6877
:1009E000B242E9D0404690470028EAD1774E784994
:1009F000784D794C794B7A4ADFF83CC2DFF800E257
:100A00002027377030270F70502640212E7020701D
:100A1000197015687349744F744E45F04064146042
:100A20000B68734D734C02F5232A0AF62C0B43F422
:100A300000320A604FF08071CCF80000D846CEF842
:100A400000003860306028602060CBF80010D8F8D3
:100A500000006949C5011BD5D8F80070FA0117D507
:100A6000D8F80060F70113D5D8F80030DE010FD5B3
:100A7000D8F80050ED010BD5D8F80040E40107D5B7
:100A8000D8F80020D00103D5D8F80000C201DED488
:100A90000F68DFF884B1594A27F008060E600B682A
:100AA00023F47F2525F47F6443F28C4944F46120CC
:100AB00040F2771740F090064BF809700E6011680D
:100AC0000C0714D413681B0711D415682F070ED414
:100AD000146826070BD41068050708D417683C076C
:100AE00005D41668300702D411680907E7D5424BD0
:100AF000434F1A68DFF840C13B483C493C4E3D4CEF
:100B0000404D42F008021A6040F24342CCF8002007
:100B10003A604FF4886707600A6030483A493260AB
:100B200022603A4E2E6060244FF4003204700A6056
:100B30001D6845F000671F601868000114D519682A
:100B40000F0111D51E6836010ED51C6825010BD585
:100B50001A68140108D51D68280105D51F683901D8
:100B600002D518680201E7D42948FAF7A7FC38B97A
:100B700028492948FFF7FCFD28492748FFF7F8FDD9
:100B8000274FDFF8B0A01D4EB946264B264DD3F8AF
:100B9000008005F073FA044604E005F06FFA031BC9
:100BA000AB42F2D83168C907F7D4204A2048C2F8CE
:100BB0000080506005F062FA1B4C054643E000BF20
:100BC00091090000ACDF01009909000000E400E099
:100BD00001E400E030E400E018E400E051E400E06B
:100BE00000D800403080044008D004400CD00440BD
:100BF00010D0044014D004402C100B4024100B40A3
:100C000004D0044034100B4008E100E00B007F11D9
:100C1000805FFF1F80240200F82AFF1F6424020067
:100C200030100B400C66FF1F40420F0008100B40B5
:100C300000001A0D0466FF1F00D0044005F01EFAE4
:100C4000421BA242A1D83968AE4B0B40002BF5D015
:100C5000D9F80000CAF80000C9F80000DAF800204E
:100C6000A84DA94C1540012D8FD1A8490B68DA0574
:100C70008BD5DFF8E892A64889F80050002525605A
:100C8000A44AA54CA54EA64F04604FF48131A54B54
:100C9000A548156031601363386005F0EFF9A34D86
:100CA000044605E005F0EAF9011BA94201F2D187EB
:100CB00099F80020002AF5D1DAF80060994F374002
:100CC000022F41F0C68743F2BC4E994B5BF80E00F1
:100CD000984C984202F03A8004F55358964F44F8E5
:100CE0000E3043F2C446012342F28E65A551C8F886
:100CF000003038463C2243F2C8450021059709F0F0
:100D00000DFB2D2308F11802635108F1140C43F276
:100D1000CC4543F2D0481046039205230F2262517E
:100D200044F80830854F864ECDF808C04FF07E5409
:100D3000CCF80040046083487C4DD0F8008005F07A
:100D40009DF9044604E005F099F9001BA842F2D889
:100D50003268D307F7D46F497B4BC1F800804B60F2
:100D600005F08CF9714C054604E005F087F9411B4C
:100D7000A142E0D83868634A0240002AF5D06F4BA0
:100D80006E4D1968CAF800102960DAF800405D4A13
:100D90005D492240012ACED15C480368D805CAD5F6
:100DA0005B4F89F8002000265A4D5C4A5C4B5A4C38
:100DB0000E605C483C604FF48131644F2E601160DE
:100DC00028631F6005F05AF9584E054605E005F006
:100DD00055F9411BB14201F2478799F80040002CB8
:100DE000F5D1DAF800204F4B1340022B41F03C873D
:100DF0004FF4007200215648564D009543F2C864E6
:100E0000049009F08BFA43F2C66043F2CC6163238D
:100E10004FF0010C0BF800C04BF804304BF80130D8
:100E200043F2D06543F2E86843F2EC6243F2F060CB
:100E300043F2D46443F2F4614BF805303F4F404E27
:100E40004BF8083000254BF802304BF800304BF8D7
:100E500004304BF80130019501350195394B334D84
:100E6000D3F8008005F00AF9044604E005F006F91D
:100E7000031BAB42F2D83268D107F7D42549324878
:100E8000C1F80080486005F0F9F8284C054604E0F8
:100E900005F0F4F8421BA242E0D83A68194B13401F
:100EA000002BF5D02548254D0168CAF800102960AF
:100EB000DAF80040134B14482340012BCED1134ADB
:100EC0001168CA05CAD589F80030009B104D049AF4
:100ED0000024046018782A60002841F035860199C2
:100EE0004D020C480D4C1C4B05604FF481320D49EE
:100EF000164D22601960A56005F0C0F80B4D044640
:100F000034E000BF01000F000466FF1F10100B400B
:100F100000100B4008100B40B45FFF1F04100B4083
:100F20000C100B4002007F1137003A1240420F00B4
:100F30004B45454EF82AFF1FC05FFF1F30100B4086
:100F400024100B400C66FF1F00001A0D27003A19F1
:100F5000BC61FF1FF865FF1F38100B400866FF1FBC
:100F600005F08CF8011BA94201F2F18599F80030D7
:100F7000002BF5D1DAF80000C24A0240022A41F003
:100F8000E685019D1F2D7FF467AF029ED6ED007AA6
:100F9000B7EE007AF4EEC77AF1EE10FA01F1F483BD
:100FA000B0EE080AF4EEC07AF1EE10FA01F3EC8329
:100FB00000270398D0ED000AB7EE001AF4EEC10A3C
:100FC000F1EE10FA01F15B83F0EE081AF4EEE10A9B
:100FD000F1EE10FA01F35383002F41F05383059C87
:100FE000A94FAA4E0FCC07F1980EAEE80F000FCC18
:100FF000AEE80F000FCCAEE80F00DBF89C5094E891
:10100000070006EBC50C8EE807009CF80580DBF8AE
:10101000CC359CF804208BF8042201208BF8058243
:101020008BF806027BB397F85CE3D7F8D015984DA0
:1010300007EB8E0407EBC106D4F85423D6F86443BB
:10104000D7F860734D2303FB0E5C51098E001CF82A
:1010500004803D6806F1604E02F01F0200FA02F1C2
:101060000EF5614408F01F0045F040031F283B6067
:10107000216008D05FEA086401F123861026FE6033
:1010800040F040023A60DBF8D47582497B687E48C4
:101090008B4241F0BD85D0F858688EB390F8E87562
:1010A000D0F85C187A4DD0F8EC2500EB870C00EBFB
:1010B000C108DCF8E065D8F8F0454D2303FB075E76
:1010C000700987001EF804C0156807F1604101F53A
:1010D000614406F01F0601230CF01F0745F0400095
:1010E000B3401F2F106023600AD05FEA0C604ABF34
:1010F000D468102424F0100447F04005D460156033
:101100000A2004F0DDFFBBF80460BBF80020BBF848
:101110000240BBF806806048604D43F2B03102EEF9
:10112000102A02EE904A5BF801205D49506005EEFE
:10113000906A05EE108AB8EE427AF8EE627AF8EE1E
:10114000655AB8EE455A02F1840302F1F40400270F
:10115000544E1760A342576117625763176457656F
:101160001766506250645066916091629164916616
:1011700082ED037A82ED047A966196639665D56175
:10118000D563D565C2ED0B7AC2ED0C7AC2ED135A68
:10119000C2ED145A82ED1B5A966782ED1C5A5767AE
:1011A000D56708D05F60986083ED047A83ED037A99
:1011B0001C339C42F6D102F5B277BC4200F0B880F5
:1011C000381BA0F11C06384B3349C4ED047AB5082E
:1011D00004F11C064FF0000E03FB05F5B742C4ED09
:1011E000037A05F00700C4F804E0A16000F0A080D5
:1011F00000285BD001283AD0022830D0032826D01E
:1012000004281CD0052812D0062808D0C6F804E00F
:10121000B160C6ED047AC6ED037A04F13806C6F86B
:1012200004E0B160C6ED047AC6ED037A1C36C6F858
:1012300004E0B160C6ED047AC6ED037A1C36C6F848
:1012400004E0B160C6ED047AC6ED037A1C36C6F838
:1012500004E0B160C6ED047AC6ED037A1C36C6F828
:1012600004E0B160C6ED047AC6ED037A1C36C6F818
:1012700004E0B160C6ED047AC6ED037A1C36B742CD
:1012800056D013E002007F11F82AFF1F78E001001A
:10129000B02A0200750B000000F07F4587D4843F20
:1012A000BAE814420AD7233CB76DDB36C6F804E02F
:1012B000B160C6ED047AC6ED037AC6F820E071622B
:1012C000C6ED0B7AC6ED0A7AC6F83CE03164C6ED8D
:1012D000127AC6ED117AC6F858E0F165C6ED197AB2
:1012E000C6ED187AC6F874E0B167C6ED207AC6ED8F
:1012F0001F7AC6F890E0C6F89410C6ED277AC6EDBE
:10130000267A06F1A80C06F1C408E036B742CCF8FC
:1013100004E0CCF80810CCED047ACCED037AC8F8E0
:1013200004E0C8F80810C8ED047AC8ED037ABDD10E
:10133000DBF85000E34FC2ED5D5A00240428C2EDF3
:101340005C5A82ED645A82ED635AC2F86841C2F871
:101350008441C2F86C71C2F8887141F04982DA4D5B
:10136000DFEDDA3ADA4FA5F1100613460024B6EEA7
:10137000004AF0EE004AD3F8841091ED040AD1ED52
:10138000060A91ED051AD1ED032A91ED022A37EEF6
:10139000406AF0EE401AE0EE861A72EEC20A71EE72
:1013A000C06A36EEC10AA0EE041A31EE816A81ED00
:1013B000051AB4EEE06AF1EE10FA81ED046A41F12B
:1013C000588076EE022AC1ED032A91ED003AD1ED64
:1013D000071A91ED016AF0EE436AE2EE246A32EEFA
:1013E000E62AF0EE432AE2EE212AF4EEC62AF1EED6
:1013F00010FA08D5B4EEE23AF1EE10FA54BFB0EEAE
:10140000436AB0EE626A93F8981083ED276A09B1D7
:101410003978B1B3D3ED250A36EE603AB5EEC03A6D
:10142000F1EE10FA01F1F98341F30B84D3ED232A95
:10143000D3ED241A93ED222A72EEE06A32EEE11A1D
:10144000F4EEE36A21EE030AF1EE10FAD8BFF0EEF3
:10145000636AC0EE260A30EEA13AF4EEC32AF1EE3A
:1014600010FA08DDB4EEC32AF1EE10FA54BFF0EE24
:10147000422AF0EE432A83ED256AC3ED242AB0EE1A
:10148000626AA6EC016AD3F8F41091ED041A91EDAA
:10149000062AD1ED056A91ED030AD1ED022A77EE15
:1014A000C10AF0EE411AE2EE201A30EE622A31EE65
:1014B000C16A36EE661AE1EE046A71EEA60AC1ED63
:1014C000056AF4EEC20AF1EE10FAC1ED040A40F129
:1014D000C38730EEA20A81ED030A91ED003AD1ED07
:1014E000071AB0EE436AA2EEA46AF0EE432A30EE89
:1014F000460A91ED016AE0EE212AF4EEC62AF1EEE9
:1015000010FA08D5B4EEE23AF1EE10FA54BFB0EE9C
:10151000436AB0EE626A93F8081183ED436A09B139
:101520003978B1B3D3ED410A36EE603AB5EEC03A40
:10153000F1EE10FA01F15A8341F37B83D3ED3F2A98
:10154000D3ED401A93ED3E2A72EEE06A32EEE10AE4
:10155000F4EEE36A60EE030AF1EE10FAD8BFF0EEA3
:10156000636A80EEA61A31EE213AF4EEC32AF1EE58
:1015700010FA08DDB4EEC32AF1EE10FA54BFF0EE13
:10158000422AF0EE432A83ED416AC3ED402AB0EED1
:10159000626A0134042CA5EC016A03F11C037FF498
:1015A000EAAED2F86411D1ED047AD1ED063A91EDAC
:1015B000054AD1ED031A91ED021A75EEE75AF0EEE5
:1015C000674AE3EEA54AB6EE002A74EEE76A71EECA
:1015D000C12A36EEC40AA0EE024A34EE843A81ED06
:1015E000054AB4EEE23AF1EE10FA81ED043A41F127
:1015F000728273EE011AC1ED031AD1ED007AD1EDBA
:10160000073A91ED017AB0EE004AF0EE675AE1EE4A
:10161000045AB0EE672A71EEE51AA1EEA32AB4EEE1
:10162000C72AF1EE10FA08D5F4EEC27AF1EE10FAFC
:1016300054BFB0EE677AB0EE427A92F8783182ED1C
:101640005F7A2BB143F284441BF80450002D41D043
:1016500092ED5D0A77EE400AF5EEC00AF1EE10FA5F
:1016600001F1218341F34883D2ED5B4A92ED5C1A8C
:101670009FED163AD2ED5A2A74EEC07A34EEC16A62
:10168000F4EEC37AF1EE10FA66EE203AD8BFF0EE2F
:10169000437A83EEA74A74EE015AF4EEE54AF1EE7E
:1016A00010FA08DDF4EE652AF1EE10FA4CBFF0EE08
:1016B000654AF0EE624A82ED5D7AC2ED5C4AB0EEB8
:1016C000647A07E000F07F45582CFF1FBD37863550
:1016D0007C5FFF1FD2F880618BED5D7AD6ED041A36
:1016E00096ED062A96ED050AD6ED030AD6ED023AE6
:1016F00075EE616AB0EE615AA2EE265AB6EE003A75
:1017000075EE612A70EEE35A72EEC07AA7EE830A94
:1017100035EE004A86ED050AB4EEE54AF1EE10FA20
:1017200086ED044A41F1E48174EE230AC6ED030A12
:10173000D6ED001A96ED072AD6ED017AB0EE000A32
:10174000F0EE616AE3EE806AB0EE611A70EEE60ACE
:10175000A0EE821AB4EEE71AF1EE10FA08D5F4EE14
:10176000C11AF1EE10FA54BFF0EE617AF0EE417A50
:1017700092F89471C2ED667A002F00F0878643F2EA
:1017800084411BF80130002B40F08086F0EE670AA0
:101790000428CBED5E0AEC4E00F0B686C0EBC00725
:1017A000B9005318D2F87CC1D3F89CE0C6F8ECE03D
:1017B0000A44D2F80C4196F83C20C6F8F040C6F82E
:1017C000F4C0C6ED3E7A22B1DBF85400042800F0E4
:1017D000AE860BEB800E9EED540ADFEDDC6A9EEDCB
:1017E000584A9FEDDB3A20EE261ABDEEC45AB4EEFD
:1017F000C31AF1EE10FA15EE105AD8BFBDEEC11A99
:101800004FEA6517D4BF11EE105A40F6FF753D44FC
:1018100041F27D018D4201F38881CE4A25EAE57CC3
:1018200002EB8C031C680BEB80000467BBF81E60A6
:10183000DBED447ADFEDC81ADFEDC85A9FEDC82A08
:101840009BED1C1ADFEDC76A02EE906AF8EEE73AEC
:10185000F8EE624A23EEA14A24EEA56A24EE060AB7
:10186000A0EE021AB4EEE61AF1EE10FA41F115817B
:101870009FEDBD5AB4EEC51AF1EE10FAD8BFB0EE26
:10188000451ABBF82050DBED455ADFEDB32ADFEDFA
:10189000B31A9FEDB34ADBED1D6A9FEDB26A8BED83
:1018A000181A03EE105AB8EEE52AF8EE433A62EE43
:1018B000227A63EEA14A27EEA40AE0EE046AF4EE6F
:1018C000C66AF1EE10FA41F124819FEDA71AF4EEF9
:1018D000C16AF1EE10FAD8BFF0EE416ABBF822708F
:1018E000DBED461ADFED9C2A9FED9C5ADFED9C4A0A
:1018F0009BED1E4ACBED196A03EE107AF8EEE15A21
:10190000B8EE432A65EEA23A62EE057ADFED956AFB
:1019100023EEA70AA0EE244AB4EEE64AF1EE10FA4E
:101920000AD59FED916AB4EEC64AF1EE10FAD4BF23
:10193000F0EE466AF0EE446ABBF82410DBED471A7D
:101940009FED863ADFED842ADFED854A9BED1F0A85
:101950009FED844ACBED1A6A01EE101AF8EEE15AB7
:10196000B8EE415A65EEA23A25EE032A62EE237ADA
:10197000A7EEA40AB4EEC40AF1EE10FA41F1C58054
:101980009FED796AB4EEC60AF1EE10FAD8BFB0EE58
:10199000460ABBF81640DBED4C2A9FED6F1A9FED0F
:1019A0006F3ADBED483A8BED1B0A06EE904AB8EE33
:1019B000E25AF8EE661A65EE015A21EE832AF8EE35
:1019C000E34A65EE827AB7EE004AE4EE817AF4EEFD
:1019D000C47AF1EE10FA01F1E680F0EE447ABBF839
:1019E00018209BED4D3ADFED5C6A9FED5C1A9BED94
:1019F000492ACBED207A06EE102AF8EEC32AB8EE7B
:101A0000465A62EEA61A65EE015AF8EEC23A21EE87
:101A1000A54AF7EE004AA3EEA64AB4EEE44AF1EE78
:101A200010FA01F1B580B0EE644ABBF81A809BED64
:101A30004E6ADFED496A9FED491ADBED4A5A8BED9C
:101A4000214A00EE108AB8EEC63AF8EE402A23EE9C
:101A5000265A62EE811AF8EEE53A25EE212AF7EED3
:101A6000004AA3EEA62AB4EEE42AF1EE10FA01F140
:101A70008480BBF81CE09BED4F1ADFED376A9FEDC9
:101A8000370ADBED4B1ACBED224A04EE10EAB8EE32
:101A9000C16AF8EE447A66EE262A27EE803AB8EE5E
:101AA000E12A23EE225AF7EE003AA2EE265AB4EECD
:101AB000E35AF1EE10FA01F15580BBF808C0DFEDF2
:101AC000275ACBED233A70EEA00A04EE90CABFEE7F
:101AD000004AA0EEA54AB8EE640AF7EE006A60EE8E
:101AE000257A27EE841AA7EE251AB4EEE61AF1EE4F
:101AF00010FA01F11D809FED1D7A1D4BBBF80A60A5
:101B00001C4F1D4D1D491E4C9F6103EE106A1A4665
:101B10000020F8EE432A42F8040B8BED367A9C60E5
:101B200001205D611160C3ED032AC3ED042A154F46
:101B3000154E04F0C5FA154B154DD3F8008004F08E
:101B40009DFA04462BE000BFF82AFF1FAE47813FF5
:101B500000F07F4538E20100B57E253C0108803960
:101B600000445E4500205F4500005C416F12033E6B
:101B70003034FF1FD3A0803FA4707D3F00F07F452D
:101B80000000204130100B4024100B400C66FF1F5A
:101B900040420F0004F072FA031BAB42CBD830680E
:101BA000C107F7D4AE4AAF49C2F80080516004F0D3
:101BB00065FAAD4C054604E004F060FA421BA2420F
:101BC000B9D83868A94B0340002BF5D0A849A84ADA
:101BD0000D68CAF800501560DAF80000A34BA5495B
:101BE0000340012BA7D1A44D2A68D205A3D50098A4
:101BF00089F800300678A14F994DA14AA1480023E9
:101C00000B60002E049939600CBF4FF478541F24E8
